:100000000C946B310C949C310C949C310C949C316D
:100010000C949C310C94DB8F0C949C310C949C318F
:100020000C946C930C949C310C9492B20C949C3173
:100030000C949C310C949C310D943E470D94E253EA
:100040000C949C310C94A7C90C949C310C949C3159
:100050000C949C310C949C310C949C310D94122284
:100060000C949C310D945D4F0C949C310C949C31FC
:100070000C949C310C949C310C949C310C949C31CC
:100080000C949C310C949C310C949C310C949C31BC
:100090000D94194F0C949C310C949C310C949C3110
:1000A0000C949C310C949C310C949C310C949C319C
:1000B0000C949C310C949C310C949C310C949C318C
:1000C0000C949C310C949C310C949C310D942153D4
:1000D0000C949C310C949C310C949C310C949C316C
:1000E0000C949C31A54AAB4AB14ABC4AC74A4C4B16
:1000F000D24ADB4AE44AEF4AFA4A054B154B204BF9
:100100004C4B2B4B364B414B6EA275A227A2F5A14F
:10011000C5A1BAA497A271A30DA46BA445B149B11E
:100120004FB158B171B18EB1CBB102B29EDFB4DF25
:10013000C7DFD4DFDEDF0CE02DE033E041E044E058
:1001400046E050E061E072E068018C014E018801F8
:1001500040019E015A015C0144018A019A013E015D
:1001600062016A019E01A601700182013A016E01DD
:100170007401320154015E0192019C0186012C013F
:100180007E01084AD73B3BCE016E84BCBFFDC12F28
:100190003D6C74319ABD56833DDA3D00C77F11BE78
:1001A000D9E4BB4C3E916BAAAABE000000803F057B
:1001B000A84CCDB2D44EB93836A9020C50B99186AC
:1001C00088083CA6AAAA2ABE000000803F07634216
:1001D00036B79BD8A71A39685618AEBAAB558C1DDE
:1001E0003CB7CC5763BD6DEDFD753EF6177231BF60
:1001F000000000803F08000000BE922449123EAB80
:10020000AAAA2ABECDCCCC4C3E00000080BEABAA30
:10021000AAAA3E00000000BF000000803F000000CE
:100220000000084178D3BB4387D1133D190E3CC36E
:10023000BD4282AD2B3E68EC8276BED98FE1A93EED
:100240004C80EFFFBE01C4FF7F3F000000000000B4
:100250000D94338B0D942B140D94AF290D94288C91
:100260000D94818D0D945D290D9477200D94A08CB3
:100270000D9432260D9437290D942D5E0D945B203C
:100280000D9438200D942A8D0D944D200D947E8B65
:100290000D9481200D9422A10D94C38C0D942E20D9
:1002A0000D94478D0D94B28C0D9479290D94D21331
:1002B0000D947B200D9443200D9447200D947F29AD
:1002C0000D94648D0D945F200D941F890D940D8DF8
:1002D0000D943C200D9463200D94FF200D9445292E
:1002E0000D946D200D94058B0D944B290D94EE8B80
:1002F0000D94CCAC0D940F210D94F08C0D94C62967
:100300000D94D28C0D9471200D94CE4E0D94A12994
:100310000D9432200D9451200D943F200D94A1890D
:100320000D94B54E0D9485290D94B28A0D94C18B10
:100330000D94538A0D9455200D9493290D94762095
:100340000D9486200D94D78A0D949E8D0D9469206E
:100350006E616E00696E66004E414E494E495459B9
:10036000494E46CDCCCC3D0AD7233C17B7D1387780
:10037000CC2B329595E6241FB14F0A000020410096
:1003800000C84200401C4620BCBE4CCA1B0E5AAEE0
:10039000C59D7400407A10F35A00A0724E180900EF
:1003A00010A5D4E80000E87648170000E40B5402DA
:1003B0000000CA9A3B000000E1F505000080969815
:1003C00000000040420F000000A086010000001065
:1003D0002700000000E803000000006400000000A7
:1003E000000A00000000000100000000002C76D888
:1003F00088DC674F0823DFC1DFAE59E1B1B796E56E
:10040000E3E453C63AE651997696E8E6C28426EBD1
:10041000898C9B62ED407C6FFCEFBC9C9F40F2BAE4
:10042000A56FA5F490055A2AF75C936B6CF9676D7C
:10043000C11BFCE0E40D47FEF520E6B500D0ED90D1
:100440002E0300943577050080841E080000204E9E
:100450000A000000C80C333333330F986E12831137
:1004600041EF8D2114893BE65516CFFEE6DB18D10E
:10047000844B381BF77C1D901DA4BBE424203284E0
:10048000725E228100C9F124ECA1E53D2763646915
:100490006E6F70737578585B00256420627974659F
:1004A00073207772697474656E20746F20454550AF
:1004B000524F4D2061742061646472657373203003
:1004C0007825303478004433202D20526561642F24
:1004D000577269746520454550524F4D0A002043BC
:1004E0006F756E7420583A20005344207072696E04
:1004F00074696E67206279746520004E6F7420699C
:100500006E206661726D206D6F64652E00416374AC
:100510006976652045787472756465723A20004981
:100520006E76616C696420657874727564657200BA
:100530005A204F666673657400556E6B6E6F776EEA
:1005400020636F6D6D616E643A2022004D32303051
:1005500020496E76616C6964206578747275646593
:100560007220007A5F6D61783A20007A5F6D696E63
:100570003A2000795F6D61783A2000795F6D696E8D
:100580003A2000785F6D61783A20006F70656E00E8
:1005900054524947474552454400785F6D696E3A69
:1005A00020005265706F7274696E6720656E6473A7
:1005B000746F7020737461747573000053494C45F7
:1005C0004E54004E4F524D414C002553204D4F4448
:1005D000453A2050657263656E7420646F6E653AAB
:1005E0002025643B207072696E742074696D6520EB
:1005F00072656D61696E696E6720696E206D696EE6
:10060000733A2025640A00456E642066696C652093
:100610006C69737400426567696E2066696C652059
:100620006C6973740025643A2025640A000A5049F5
:100630004E44412074656D70657261747572653ADF
:1006400020252E3166205A20736869667420286D33
:100650006D293A20252E3366000A537465703A20BE
:1006600025642F360A000A537465703A2025642FDA
:10067000362028736B6970706564290A50494E44AE
:10068000412074656D70657261747572653A2025DC
:1006900064205A20736869667420286D6D293A3089
:1006A0000A000A5A45524F3A20252E33660A007333
:1006B000746172742074656D7065726174757265B1
:1006C0003A20252E31660A0025642020252E326628
:1006D00000255320583A20252E356620593A2025EA
:1006E0002E3566205A3A20252E35660A00536C6551
:1006F00065702E2E2E004E6F7420696E206661721A
:100700006D206D6F64652E0025640045303A2564C8
:100710002052504D0A50524E303A25642052504DCE
:100720000A002564004175746F0020452F443D0088
:10073000416476616E6365204B3D004D323230205E
:1007400053256900255346696C616D656E7420738D
:10075000657474696E67733A2044697361626C658D
:10076000640A00255346696C616D656E742073657B
:100770007474696E67733A0A25532020204D323015
:10078000302044252E32660A00255352657472616A
:1007900063743A20533D4C656E67746820286D6D14
:1007A0002920463A537065656420286D6D2F6D29A8
:1007B000205A3A205A4C69667420286D6D290A2502
:1007C000532020204D3230372053252E32662046CC
:1007D000252E3266205A252E32660A25535265632D
:1007E0006F7665723A20533D4578747261206C656E
:1007F0006E67746820286D6D2920463A53706565D0
:100800006420286D6D2F6D290A25532020204D323C
:1008100030382053252E32662046252E32660A2592
:10082000534175746F2D526574726163743A20532D
:100830003D3020746F2064697361626C652C2031D7
:1008400020746F20696E74657270726574206578AB
:1008500074727564652D6F6E6C79206D6F7665733B
:10086000206173207265747261637473206F7220EB
:100870007265636F7665726965730A25532020205F
:100880004D323039205325640A0025535049442005
:10089000686561746265642073657474696E6773FA
:1008A0003A0A25532020204D3330342050252E3253
:1008B000662049252E32662044252E32660A002500
:1008C000535049442073657474696E67733A0A25FE
:1008D000532020204D3330312050252E32662049C0
:1008E000252E32662044252E32660A002553537485
:1008F0006570732070657220756E69743A0A2553AD
:1009000020204D39322058252E32662059252E328E
:1009100066205A252E32662045252E32660A25533A
:100920004D6178696D756D20666565647261746589
:1009300073202D206E6F726D616C20286D6D2F738A
:10094000293A0A255320204D3230332058252E32A3
:10095000662059252E3266205A252E3266204525DE
:100960002E32660A25534D6178696D756D20666576
:1009700065647261746573202D20737465616C7495
:100980006820286D6D2F73293A0A255320204D3297
:1009900030332058252E32662059252E3266205AB3
:1009A000252E32662045252E32660A25534D617864
:1009B000696D756D20616363656C65726174696FE3
:1009C0006E202D206E6F726D616C20286D6D2F73FF
:1009D00032293A0A255320204D3230312058256CD7
:1009E000752059256C75205A256C752045256C7528
:1009F0000A25534D6178696D756D20616363656C7F
:100A000065726174696F6E202D20737465616C74FA
:100A10006820286D6D2F7332293A0A255320204D06
:100A20003230312058256C752059256C75205A2597
:100A30006C752045256C750A2553416363656C65AB
:100A4000726174696F6E3A20533D616363656C65D2
:100A5000726174696F6E2C20543D726574726163AB
:100A60007420616363656C65726174696F6E0A25D9
:100A70005320204D3230342053252E326620542509
:100A80002E32660A2553416476616E636564207672
:100A900061726961626C65733A20533D4D696E20E5
:100AA000666565647261746520286D6D2F73292CED
:100AB00020543D4D696E2074726176656C206665C8
:100AC00065647261746520286D6D2F73292C204236
:100AD0003D6D696E696D756D207365676D656E74CA
:100AE0002074696D6520286D73292C20583D6D6137
:100AF00078696D756D205859206A65726B20286D74
:100B00006D2F73292C20205A3D6D6178696D756DAC
:100B1000205A206A65726B20286D6D2F73292C2056
:100B200020453D6D6178696D756D2045206A65725F
:100B30006B20286D6D2F73290A255320204D3230EC
:100B4000352053252E32662054252E32662042252C
:100B50002E32662058252E32662059252E326620E8
:100B60005A252E32662045252E32660A2553486FB7
:100B70006D65206F666673657420286D6D293A0A6D
:100B8000255320204D3230362058252E32662059EC
:100B9000252E3266205A252E32660A00462564200C
:100BA00025640A004D4D55203C3D202746256420F4
:100BB0002564270A00504944204175746F74756E8E
:100BC000652066696E6973686564212050757420BC
:100BD000746865206C617374204B702C204B692005
:100BE000616E64204B6420636F6E7374616E747306
:100BF0002066726F6D2061626F766520696E746F1A
:100C000020436F6E66696775726174696F6E2E68D6
:100C100000504944204175746F74756E652066619B
:100C2000696C6564212074696D656F75740020407E
:100C30003A00543A00423A00504944204175746FDA
:100C400074756E65206661696C6564212054656DFC
:100C5000706572617475726520746F6F2068696762
:100C60006800204B643A2000204B693A2000204B5A
:100C7000703A200020436C617373696320504944CB
:100C800020002054753A2000204B753A2000206D3A
:100C900061783A2000206D696E3A200020643A2085
:100CA0000020626961733A200020453A00205A3AD8
:100CB0000020593A0020453A00205A3A0020593A7B
:100CC00000583A00005A30005A310059300059316A
:100CD00000583000583100456E642073746F707393
:100CE0002064696167002E0044656C6574696F6EED
:100CF000206661696C65642C2046696C653A200049
:100D000046696C652064656C657465643A004E6F75
:100D100074205344207072696E74696E670050725B
:100D2000696E742073617665640053442070726943
:100D30006E7420706175736564000A002F000A00EC
:100D40002F2F20616374696F6E3A63616E63656C07
:100D50000043524153485F43414E43454C00435288
:100D60004153485F5245434F564552004352415309
:100D7000485F5245434F56455200222832290054BD
:100D8000004475706C6963697420542D636F6465E9
:100D90002069676E6F7265642E0A004475706C6915
:100DA00063697420542D636F64652069676E6F7288
:100DB00065642E0A00496E76616C69642054206374
:100DC0006F64652E00556E6B6E6F776E204D2063DD
:100DD0006F64653A202573200A006E6F2076616C7F
:100DE000696420636F6D6D616E64002C20002C209F
:100DF000002C20006E2F61002C20002C20002C20C5
:100E0000006E2F61002F00503A0057616974206610
:100E10006F722050494E444120746172676574209E
:100E200074656D70657261747572653A004C414EFF
:100E3000472053454C20464F524345440022283119
:100E4000290030303030303030302D303030302DDF
:100E5000303030302D303030302D30303030303098
:100E60003030303030300020555549443A003100A0
:100E70002045585452554445525F434F554E543ABD
:100E8000005072757361206933204D4B3300204D43
:100E9000414348494E455F545950453A00312E3040
:100EA00000206261736564206F6E204D61726C6911
:100EB0006E204649524D574152455F55524C3A6853
:100EC000747470733A2F2F6769746875622E636F3C
:100ED0006D2F707275736133642F50727573612D4D
:100EE0004669726D776172652050524F544F434F7F
:100EF0004C5F56455253494F4E3A004649524D5762
:100F00004152455F4E414D453A50727573612D46D1
:100F100069726D7761726520004D31313320530065
:100F200020423A0020453A00543A0020413A00203D
:100F3000503A002042403A0020403A00202F003A28
:100F400000205400202F0020423A00202F006F6B19
:100F500020543A002569206D696E2C202569207384
:100F6000656300496E76616C6964204D20636F642F
:100F7000653A202573200A00556E6B6E6F776E20E0
:100F80004720636F64653A202573200A004D65731E
:100F90006820626564206C6576656C696E67206E9A
:100FA0006F74206163746976652E000A002020004A
:100FB0000A4D6561737572656420706F696E747334
:100FC0003A000A5A20736561726368206865696730
:100FD00068743A20002C004E756D20582C593A2028
:100FE00000206D6963726F6E73004578636573737B
:100FF00069766520626564206C6576656C696E67EC
:1010000020636F7272656374696F6E3A20004732B5
:10101000382057300050494E44412070726F62654D
:101020002063616C6962726174696F6E20737461B0
:10103000727400473238205730004D323400534527
:10104000545F43484F505F005345545F53544550DD
:101050005F005345545F574156455F00544D435F11
:101060000043524153485F005072657373206B6EAA
:101070006F6220746F2070726568656174206E6F96
:101080007A7A6C6520616E6420636F6E74696E7528
:10109000652E00506C6561736520707265737320F6
:1010A000746865206B6E6F6220746F20756E6C6F54
:1010B00061642066696C616D656E740052656D6F68
:1010C0007665206F6C642066696C616D656E742056
:1010D000616E6420707265737320746865206B6E36
:1010E0006F6220746F207374617274206C6F61641E
:1010F000696E67206E65772066696C616D656E74D8
:101100002E00616E642070726573732074686520B0
:101110006B6E6F6200496E736572742066696C61F4
:101120006D656E7400436F6C6F72206E6F74206318
:101130006F72726563740046696C616D656E7420D0
:101140006E6F74206C6F61646564004368616E67E4
:10115000656420636F72726563746C793F004C6FD5
:101160006164696E6720636F6C6F72004368616EC3
:10117000676520737563636573732100506C6561E7
:101180007365206F70656E2069646C657220616E96
:10119000642072656D6F76652066696C616D656E41
:1011A00074206D616E75616C6C792E0057617320CF
:1011B00066696C616D656E7420756E6C6F6164201C
:1011C0007375636365737366756C3F00506C65611E
:1011D000736520757067726164652E004E657720B7
:1011E0006669726D776172652076657273696F6E7C
:1011F00020617661696C61626C653A00576169745F
:10120000696E6720666F722050494E4441207072AB
:101210006F626520636F6F6C696E67004372617304
:10122000682064657465637465642E205265737507
:101230006D65207072696E743F004372617368203F
:1012400064657465637465642E00457874727564B2
:1012500065720043686F6F7365206578747275649A
:1012600065723A0043686F6F73652066696C616DE3
:10127000656E743A004E6F206D6F76652E00576173
:10128000697420666F7220757365722E2E2E00535E
:101290006F6D652070726F626C656D20656E636F37
:1012A000756E74657265642C205A2D6C6576656C5C
:1012B000696E6720656E666F72636564202E2E2EE0
:1012C00000537461626C6520616D6269656E7420A3
:1012D00074656D70657261747572652032312D327E
:1012E0003643206973206E656564656420612072F1
:1012F00069676964207374616E6420697320726524
:101300007175697265642E00506C65617365207239
:10131000756E2058595A2063616C696272617469F4
:101320006F6E2066697273742E0073746172740A32
:10133000006164635F696E69740A001B5B324A1B5B
:101340005B313B31484F726967696E616C20507246
:101350007573612069331B5B323B33485072757380
:101360006120526573656172636800466163746FE2
:10137000727920524553455400466562203132202F
:101380003230313900436F6D70696C65643A20000A
:10139000286E6F6E652C2064656661756C742063C1
:1013A0006F6E6669672900466562203132203230EF
:1013B00031392032313A34393A35370020332E353D
:1013C0002E322D313939390A002055706C6F616425
:1013D00020696E2070726F677265737300205A3ACD
:1013E0000020593A0020583A0043524153485F4484
:1013F0004554454354454458590043524153485F6E
:101400004445544543544544590043524153485F71
:10141000444554454354454458004D3239005072B8
:10142000757361206933204D4B33204F4B2E0042A2
:101430006C61636B6F7574206F6363757272656442
:101440002E205265636F766572207072696E743FEC
:101450000053656C66746573742077696C6C2062E8
:10146000652072756E20746F2063616C69627261B1
:1014700074652061636375726174652073656E7352
:101480006F726C657373207265686F6D696E672E1D
:10149000005468657265206973207374696C6C20F0
:1014A00061206E65656420746F206D616B65205AE4
:1014B0002063616C6962726174696F6E2E20506C7A
:1014C0006561736520666F6C6C6F7720746865204A
:1014D0006D616E75616C2C2063686170746572203B
:1014E00046697273742073746570732C207365631E
:1014F00074696F6E2043616C6962726174696F6EAA
:1015000020666C6F772E005072696E746572206869
:101510006173206E6F74206265656E2063616C6913
:10152000627261746564207965742E20506C656107
:10153000736520666F6C6C6F7720746865206D61D1
:101540006E75616C2C2063686170746572204669E9
:101550007273742073746570732C2073656374697F
:101560006F6E2043616C6962726174696F6E206690
:101570006C6F772E004F6C642073657474696E67AE
:101580007320666F756E642E2044656661756C7499
:10159000205049442C204573746570732065746332
:1015A0002E2077696C6C206265207365742E00575D
:1015B00061726E696E673A20626F7468207072693A
:1015C0006E746572207479706520616E64206D6F31
:1015D00074686572626F61726420747970652063EB
:1015E00068616E6765642E005761726E696E673A56
:1015F000207072696E7465722074797065206368FA
:10160000616E6765642E005761726E696E673A207D
:101610006D6F74686572626F617264207479706551
:10162000206368616E6765642E0045787465726E2C
:10163000616C2053504920666C61736820573235C5
:10164000583230434C206E6F7420726573706F6E29
:1016500064696E672E0043726173684465746563E4
:10166000742044495341424C4544004372617368BD
:1016700044657465637420454E41424C45442100E5
:101680002020506C616E6E657242756666657242AE
:10169000797465733A20002046726565204D656D4A
:1016A0006F72793A2000207C20417574686F723A1D
:1016B0002000204C61737420557064617465643A35
:1016C000200020536F6674776172652052657365E0
:1016D0007400205761746368646F67205265736596
:1016E00074002042726F776E206F7574205265739C
:1016F0006574002045787465726E616C2052657364
:10170000657400506F7765725570006572726F7204
:101710002077726974696E6720746F2066696C65E2
:1017200000656E6473746F7073206869743A20008A
:10173000446F6E6520736176696E672066696C65BB
:101740002E006F6B0058595A2063616C6962726198
:1017500074696F6E20616C6C2072696768742E20EA
:10176000536B65772077696C6C20626520636F72BC
:10177000726563746564206175746F6D617469630B
:10178000616C6C792E0058595A2063616C696272E1
:101790006174696F6E20616C6C2072696768742E69
:1017A00020582F5920617865732061726520736C11
:1017B000696768746C7920736B657765642E204760
:1017C0006F6F64206A6F62210058595A2063616C00
:1017D0006962726174696F6E206F6B2E20582F5989
:1017E0002061786573206172652070657270656E26
:1017F000646963756C61722E20436F6E67726174E9
:10180000756C6174696F6E73210058595A20636159
:101810006C6962726174696F6E206661696C65647F
:101820002E2052696768742066726F6E742063613F
:101830006C6962726174696F6E20706F696E74207A
:101840006E6F7420726561636861626C652E00580A
:10185000595A2063616C6962726174696F6E2066A7
:1018600061696C65642E2046726F6E742063616CD2
:101870006962726174696F6E20706F696E74732033
:101880006E6F7420726561636861626C652E0058CA
:10189000595A2063616C6962726174696F6E206667
:1018A00061696C65642E20506C6561736520636F9F
:1018B0006E73756C7420746865206D616E75616CF3
:1018C0002E0058595A2063616C6962726174696FA5
:1018D0006E20636F6D70726F6D697365642E205238
:1018E000696768742066726F6E742063616C6962E8
:1018F000726174696F6E20706F696E74206E6F74A0
:1019000020726561636861626C652E0058595A20C7
:1019100063616C6962726174696F6E20636F6D7070
:10192000726F6D697365642E2046726F6E742063EA
:10193000616C6962726174696F6E20706F696E7438
:1019400073206E6F7420726561636861626C652ECE
:101950000058595A2063616C6962726174696F6ED4
:10196000206661696C65642E204265642063616C49
:101970006962726174696F6E20706F696E7420772E
:101980006173206E6F7420666F756E642E00506CEC
:101990006561736520706C61636520737465656C47
:1019A000207368656574206F6E2068656174626578
:1019B000642E0044697374616E6365206265747798
:1019C00065656E20746970206F6620746865206E8E
:1019D0006F7A7A6C6520616E642074686520626538
:1019E00064207375726661636520686173206E6F31
:1019F00074206265656E20736574207965742E208D
:101A0000506C6561736520666F6C6C6F77207468CD
:101A100065206D616E75616C2C2063686170746502
:101A2000722046697273742073746570732C20730E
:101A3000656374696F6E204669727374206C617996
:101A400065722063616C6962726174696F6E2E00E9
:101A5000506C6163652061207368656574206F66F2
:101A600020706170657220756E646572207468659F
:101A7000206E6F7A7A6C6520647572696E67207467
:101A800068652063616C6962726174696F6E206F52
:101A900066206669727374203420706F696E747387
:101AA0002E20496620746865206E6F7A7A6C6520F6
:101AB0006361746368657320746865207061706524
:101AC000722C20706F776572206F6666207468656F
:101AD000207072696E74657220696D6D65646961EC
:101AE00074656C792E00506C656173652072656D4C
:101AF0006F766520737465656C2073686565742006
:101B000066726F6D20686561746265642E0049734A
:101B100020737465656C207368656574206F6E2032
:101B2000686561746265643F00206F66203400530D
:101B30006561726368696E67206265642063616CC9
:101B40006962726174696F6E20706F696E740020D3
:101B50006F662039004D6561737572696E6720721A
:101B600065666572656E636520686569676874207F
:101B70006F662063616C6962726174696F6E207058
:101B80006F696E7400506C6561736520636C65618C
:101B90006E20746865206E6F7A7A6C6520666F724D
:101BA0002063616C6962726174696F6E2E20436C90
:101BB00069636B207768656E20646F6E652E0041E7
:101BC00075746F20686F6D650078797A63616C5FFA
:101BD0006D656173737572655F656E7465720A0019
:101BE00078797A63616C5F73706972616C382063B5
:101BF000783D25642063793D2564207A303D256455
:101C000020647A3D2564207261646975733D2564A2
:101C10002061643D25640A0078797A63616C5F73A2
:101C200065617263685A206E6F207369676E616CBC
:101C30000A20783D256C6420793D256C64207A3D2E
:101C4000256C640A00204F4E2D5349474E414C20CD
:101C5000617420783D256420793D2564207A3D25F6
:101C6000642061643D25640A0078797A63616C5F61
:101C70007365617263685A20783D256C6420793DF4
:101C8000256C64207A3D256C640A000A00253032F8
:101C9000780078797A63616C5F7363616E5F7069F5
:101CA00078656C735F33327833322063783D256416
:101CB0002063793D2564206D696E5F7A3D2564203F
:101CC0006D61785F7A3D25640A0020253264202505
:101CD000640A000A002530327800206D696E3D25C7
:101CE00064206D61783D2564206469663D25640A41
:101CF000006D61785F633D253264206D61785F6CB3
:101D00003D25640A006D61785F633D2564206D6147
:101D1000785F723D2564206D61785F6D61746368E2
:101D20003D25640A0020783D256420793D25642006
:101D30007A3D25640A00207061747465726E2066B5
:101D40006F756E642061742025642025640A00008C
:101D500000F000F801FC03FE07FE07FE07FE07FC8B
:101D600003F801F000000073697A656F6628746FEC
:101D700074616C293D25640A0073697A656F662871
:101D8000626C6F636B5F627566666572293D256480
:101D90000A0078797A63616C5F6D6561737375723F
:101DA000655F6C656176650A00706F696E743D25CC
:101DB0006420783D256420793D2564207A3D2564A2
:101DC0000A0058025802584D584DB004F055F055CD
:101DD000B00478797A63616C5F66696E645F62658E
:101DE000645F696E64756374696F6E5F73656E734B
:101DF0006F725F706F696E745F787920783D256CC3
:101E00006420793D256C64207A3D256C640A0020AD
:101E10003C20005741524E494E473A2046726F6E61
:101E20007420706F696E74206E6F742072656163C8
:101E30006861626C652E205920636F6F7264696EF1
:101E40006174653A0000000040410000C04000009D
:101E50005C430000C04000005C43000046430000BB
:101E6000404100004643497465726174696F6E3A7F
:101E7000200043616C6962726174696F6E206661F3
:101E8000696C65642120436865636B207468652014
:101E90006178657320616E642072756E2061676180
:101EA000696E2E0020423A0020453A00543A00491B
:101EB0004E5434007265636F7665725F6D6163685E
:101EC000696E655F73746174655F61667465725F86
:101ED000706F7765725F70616E69632C20696E69DF
:101EE0007469616C20007265636F7665725F6D6105
:101EF0006368696E655F73746174655F616674655C
:101F0000725F706F7765725F70616E69632C2069B4
:101F10006E697469616C2000473932204500505267
:101F20005553412075766C6F004734205330004D77
:101F300032362053256C75004D3130362053004D1C
:101F40003832004731204625640047312045322A87
:101F500064656661756C745F7265747261637469DF
:101F60006F6E2046343830004731205A0020463208
:101F70003030300020590047312058004D383300B0
:101F8000506F736974696F6E207265616420667248
:101F90006F6D20656570726F6D3A004D323320258C
:101FA00073002E67636F0046656564726174653AFD
:101FB00000473120452D64656661756C745F7265FC
:101FC0007472616374696F6E204634383000473133
:101FD0002045352046313230004D3833004D3139FF
:101FE0003020532564004D3130392053256400479B
:101FF000323820582059004731205A32352046388F
:102000003030002046004731205A0020460047313A
:102010002045004D383300627573793A2070617540
:1020200073656420666F7220696E707574006275E6
:1020300073793A2070617573656420666F722075DC
:1020400073657200627573793A2070726F6365739D
:1020500073696E67006F6B0A0055564C4F202D2038
:10206000656E642025640A007374707325640A0029
:10207000776F726C6420636F6F7264696E617465F0
:10208000733A2028252E33662C20252E33662C20EB
:10209000252E3366290A00706879736963616C20A4
:1020A000636F6F7264696E617465733A2028252EC0
:1020B00033662C20252E33662C20252E3366290AE4
:1020C0000043757272656E7420706F73205A5F41A1
:1020D0005849533A252E33660A43757272656E74F9
:1020E00020706F7320455F415849533A252E33665F
:1020F0000A0041667465722077616974696E6720B1
:10210000666F722074656D703A0A43757272656EFF
:102110007420706F7320585F415849533A252E330D
:10212000660A43757272656E7420706F7320595F12
:10213000415849533A252E33660A005265636F763B
:102140006572696E67207072696E742020202000AD
:102150006F6B0A0073746172740A004D4D55322022
:102160006669726D776172652076657273696F6EEC
:1021700020696E76616C69642E2052657175697292
:1021800065642076657273696F6E3A206275696C5A
:1021900064206E756D626572202564206F72206800
:1021A00069676865722E004D4D55203D3E20276FB2
:1021B0006B270A002564004D4D55207265747279B5
:1021C00020617474656D7074206E722E2025640A0F
:1021D000004D4D55203D3E20276F6B270A00410AD8
:1021E000004D4D55203C3D202741270A004D3630FB
:1021F00030004D363030204155544F004653454E47
:10220000534F525F5245434F5645520025686875FB
:102210000050300A0053330A004D4D55203C3D20FC
:10222000275333270A0052300A004D4D55203C3DBC
:1022300020275230270A004525640A004D4D5520BD
:102240003C3D2027452564270A0055300A004D4DA6
:1022500055203C3D20275530270A0043300A004DC9
:102260004D55203C3D20274330270A004C25640A69
:10227000004D4D55203C3D20274C2564270A005435
:1022800025640A004D4D55203C3D202754256427E8
:102290000A004D4D55202D20454E41424C454400ED
:1022A000256868750050300A0050300A004D4D55C1
:1022B0002076657273696F6E2076616C6964004D7B
:1022C0004D55203D3E202725646F6B270A0025755C
:1022D0000053320A004D4D55203C3D2027533227F4
:1022E000004D4D55203D3E202725646F6B270A0089
:1022F0002575004D4D55206E6F7420726573706F9B
:102300006E64696E67202D2044495341424C454418
:102310000053310A004D4D55203C3D2027533127B5
:10232000004D4D55203D3E20277374617274270087
:102330006D6D755F6765745F726573706F6E7365E1
:1023400028292072657475726E696E673A2025645B
:102350000A006D6D755F6765745F726573706F6E8F
:102360007365202D20626567696E206D6F76653A12
:1023700025640A00556E6C6F6164696E672066693A
:102380006E697368656420320A00556E6C6F616413
:1023900020320A00556E6C6F6164696E6720666951
:1023A0006E697368656420310A00556E6C6F6164F4
:1023B00020310A006D6D755F6765745F72657370BB
:1023C0006F6E7365202D20626567696E206D6F7674
:1023D000653A25640A004D4D55207374617274731B
:1023E00020726573706F6E64696E670A004D4D559B
:1023F000206E6F7420726573706F6E64696E670A09
:10240000000000803F555585410000803F0000C816
:102410004100000040555505420000C03F00004803
:10242000420000204055558542000070C1ABAAA66D
:1024300042000060C10000A0410000C0C0000020B8
:102440004100002041ABAA3A41000020C15555D5BA
:1024500040000048C2555505424D373031204530C7
:10246000004D373031204531004D37303120453275
:10247000004D373031204533004D37303120453461
:10248000004D373031204534004D37303120453351
:10249000004D373031204532004D37303120453145
:1024A000004D3730312045300046696C616D656EF6
:1024B00074206E72206F7574206F662072616E6773
:1024C0006521004164646974696F6E616C206C6F92
:1024D000616420617474656D7074206E722E2025A5
:1024E000640A00506C656173652075706461746581
:1024F000206669726D7761726520696E20796F75EB
:1025000072204D4D55322E2057616974696E6720D7
:10251000666F722072657365742E004D4D55204FA5
:102520004B2E20526573756D696E672E2E2E004DF1
:102530004D55204F4B2E20526573756D696E672087
:10254000706F736974696F6E2E2E2E004D4D55207D
:102550004F4B2E20526573756D696E672074656DE3
:1025600070657261747572652E2E2E004669782032
:1025700074686520697373756520616E6420746882
:10258000656E20707265737320627574746F6E204F
:102590006F6E204D4D5520756E69742E005072651A
:1025A000737320746865206B6E6F6220746F207285
:1025B0006573756D65206E6F7A7A6C652074656DD4
:1025C00070657261747572652E004D4D55206E6593
:1025D000656473207573657220617474656E7469C7
:1025E0006F6E2E00506C656173652072656D6F763D
:1025F000652066696C616D656E7420616E6420741F
:1026000068656E20707265737320746865206B6EE8
:102610006F622E00456A656374696E672066696C37
:10262000616D656E74004D4D55206C6F6164206660
:1026300061696C65642020202020002563253364B7
:102640002F2564256300746D63323133305F686F0A
:102650006D655F656E74657228617865735F6D6125
:10266000736B3D307825303278290A00746D6332FF
:102670003133305F686F6D655F6578697420746DA4
:1026800063323133305F73675F686F6D696E675FA8
:10269000617865735F6D61736B3D3078253032789A
:1026A0000A00726573756C742076616C75653A20EA
:1026B00025640A0020693D25326420636E743D253F
:1026C00032642076616C3D2532640A00636C757358
:1026D000746572733A0A0020693D25326420737470
:1026E00065703D2532640A00736F727465642073EF
:1026F000616D706C65733A0A003A2000202020203A
:1027000020202020202020202020202020202000E9
:10271000203A2000202020202020202020202020BF
:1027200020202020202020200020202020202020C9
:1027300020202020202000257300544D43204452A7
:1027400049564552204F56455254454D5000253369
:10275000642E25303175256325642563005A2533A1
:10276000642E25303275005A2D2D2D2E2D2D00254D
:10277000632533642525002D2D2D002533686864DD
:102780000025335325337325250020534400202092
:102790002000555342002025753E257500203F3E00
:1027A000257500204625750020463F002046302034
:1027B000200025632D2D3A2D2D2020002563253363
:1027C00075682025632563002563253032753A2519
:1027D000303275256325630050494E4441204865D9
:1027E0006174696E670054656D702E2063616C2E94
:1027F000202020202020202020200043616C6962BE
:10280000726174696F6E20646F6E650043616C69FC
:1028100062726174696E67205A0042656420646F59
:102820006E65004265642048656174696E670048A2
:10283000656174696E6720646F6E652E004865611E
:1028400074696E6700256920686F75727320256949
:10285000206D696E757465730054494D454F55542C
:102860003A004D3131300046756C6C205258204290
:102870007566666572006673656E736F725F7374FA
:102880006F705F616E645F736176655F7072696EB1
:10289000740A006673656E736F725F726573746F2E
:1028A00072655F7072696E745F616E645F636F6E94
:1028B00074696E75650A0044495341424C45440AA7
:1028C00000454E41424C4544004653656E736F725D
:1028D0002025530A00504154393132355F696E6901
:1028E000743A256868750A00504154393132355FB1
:1028F000696E69743A256868750A00504154393127
:102900003235206E6F7420726573706F6E64696EFD
:10291000672028256429210A00446F6E65207072A3
:10292000696E74696E672066696C65005072696EC5
:102930007465722073746F707065642064756520AF
:10294000746F206572726F72732E204669782074DE
:102950006865206572726F7220616E6420757365A0
:10296000204D39393920746F207265737461727427
:102970002E202854656D70657261747572652069CA
:10298000732072657365742E2053657420697420FA
:1029900061667465722072657374617274696E67C2
:1029A00029004E6F204C696E65204E756D62657210
:1029B000207769746820636865636B73756D2C207C
:1029C0004C617374204C696E653A20004E6F204351
:1029D0006865636B73756D2077697468206C696EC8
:1029E00065206E756D6265722C204C617374204C8D
:1029F000696E653A2000636865636B73756D206D61
:102A000069736D617463682C204C617374204C6928
:102A10006E653A20004C696E65204E756D62657278
:102A2000206973206E6F74204C617374204C696E42
:102A300065204E756D6265722B312C204C6173746C
:102A4000204C696E653A20006673656E736F725F25
:102A50006175746F6C6F61645F636865636B5F73EE
:102A600074617274202D206175746F6C6F616420C5
:102A7000454E41424C45440A006673656E736F7261
:102A80005F6175746F6C6F61645F636865636B5FD2
:102A900073746F70202D206175746F6C6F6164208A
:102AA00044495341424C45440A0053544F50504509
:102AB000442E2000566F6C74616765730054656D19
:102AC0007065726174757265730042656C74207311
:102AD00074617475730053656E736F7220696E66EE
:102AE0006F00457874727564657220696E666F0058
:102AF00058595A2063616C2E2064657461696C7347
:102B000000756E6B6E6F776E004D4D553220636FA2
:102B10006E6E656374656400446174653A00686F45
:102B200077746F2E707275736133642E636F6D00EE
:102B3000666F72756D2E707275736133642E636F7C
:102B40006D00707275736133642E636F6D00746F06
:102B500020756E6C6F61642066696C616D656E7462
:102B600000746F206C6F61642066696C616D656EC6
:102B70007400507265737320746865206B6E6F62A9
:102B8000003E43616E63656C0050726568656174F8
:102B9000696E6720746F20756E6C6F61640050728F
:102BA0006568656174696E6720746F206C6F61641D
:102BB000005072656865617420746865206E6F7A74
:102BC0007A6C6521004552524F523A0046696C6159
:102BD0006D656E7420657874727564696E67202601
:102BE000207769746820636F727265637420636F05
:102BF0006C6F723F004175746F6C6F6164696E67D2
:102C00002066696C616D656E742069732061637400
:102C10006976652C206A75737420707265737320F1
:102C2000746865206B6E6F6220616E6420696E73DC
:102C30006572742066696C616D656E742E2E2E004F
:102C4000546F74616C207072696E742074696D6564
:102C500000546F74616C2066696C616D656E740000
:102C60005072696E742074696D650046696C616D9F
:102C7000656E742075736564005269676874004CF2
:102C800065667400592064697374616E63652066BB
:102C9000726F6D206D696E00536576657265207385
:102CA0006B657700536C6967687420736B65770098
:102CB0004D6561737572656420736B6577005B3079
:102CC0003B305D20706F696E74206F66667365744B
:102CD0000041646A757374696E67205A00526573A7
:102CE000657400526561722073696465205B756D5F
:102CF0005D0046726F6E7420736964655B756D5D0F
:102D000000526967687420736964655B756D5D0066
:102D10004C6566742073696465205B756D5D005356
:102D200065742074656D70657261747572653A00C2
:102D3000466C617368416972204950204164647235
:102D40003A004D4D5532202020202020204E2F418A
:102D50000025642E25642E25642D25640020465709
:102D60003A00466562203132203230313900453335
:102D700044763666756C6C0045494E53795F313048
:102D80006100315F37356D6D5F4D4B33002D2D2D5B
:102D90002D2D2D2D2D2D2D2D2D00207265706F20A8
:102DA000556E6B6E6F776E0020332E352E322D31BF
:102DB000393939004669726D776172653A00256468
:102DC0002E25642E25642E2564004D373032004DAB
:102DD00037303100464C4558202D20203234300009
:102DE00050502020202D20203235340048495053A7
:102DF000202D20203232300041425320202D20202F
:102E00003235350050455420202D202032333000FB
:102E1000504C4120202D2020323135004D373032AA
:102E2000004D373031004578747275646572006DFD
:102E30006D000059005800580059005A00256325BC
:102E40002E3132533A2573252B30362E3366001B34
:102E50005B324A2553203A1B5B313B394825382EDB
:102E60003266206D0A2553203A0A25376C646420A7
:102E70003A253268686468203A25303268686420F0
:102E80006D001B5B324A25533A1B5B313B364825AC
:102E9000382E32666D200A2553203A1B5B333B38AF
:102EA000482532646820253032646D202530326434
:102EB000730025362E32666D6D004E2F41001B5B70
:102EC000303B304825533A0A25530A25533A0A2500
:102ED000533A001B5B303B3135484E2F41001B5BA2
:102EE000303B31354825342E326601001B5B303BC8
:102EF000304825533A0A25530A25533A20202535D0
:102F00002E3266010A25533A202025352E326601DD
:102F10000024F4D43050C38E20C2A24017828B709C
:102F200011127A910D816CD90AA861E108C758661F
:102F300007615143061E4B5D05C145A7041A4111A7
:102F400004093D9803713931034036DB0265339142
:102F500002D4305402802E1D02632CEE01752AC566
:102F600001B028A001102781018F2564012B244B7B
:102F700001E0223401AC211F018D200D01801FFCD6
:102F800000841EED00971DDF00B81CD200E61BC6B2
:102F900000201BBC00641AB200B219A8000A19A0D4
:102FA000006A189900D117910040178B00B516845C
:102FB0000031167E00B31579003A157300C7146FFF
:102FC0000058146A00EE1366008813630025135E30
:102FD00000C7125B006C12570015125400C111514A
:102FE0000070114F0021114B00D61049008D104781
:102FF000004610440002104200C00F4000800F3E07
:1030000000420F3C00060F3B00CB0E3800930E37FA
:10301000005C0E3500270E3400F30D3200C10D3177
:1030200000900D3000600D2E00320D2D00050D2C8E
:1030300000D90C2B00AE0C2900850C29005C0C2754
:1030400000350C27000E0C2600E80B2400C40B24CE
:1030500000A00B23007D0B23005A0B2100390B210C
:1030600000180B2000F80A1F00D90A1E00BB0A1E18
:10307000009D0A1D00800A1D00630A1C00470A1BF0
:10308000002C0A1B00110A1A00F7091A00DD0919A1
:1030900000C4091900AB091900920917007B09182F
:1030A00000630917004C091600360916002009169E
:1030B000000A091500F5081500E0081400CC0814F2
:1030C00000B8081400A4081400900813007D08122A
:1030D000006B08130058081200460812003408114B
:1030E00000230811001208110001081100F0071058
:1030F00000E0071000D0071000C0071000B0070F55
:1031000000A107100091070E0083070F0074070F3E
:103110000065070E0057070E0049070E003B070D1C
:10312000002E070E0020070D0013070D0006070DE7
:1031300000F9060C00ED060D00E0060C00D4060CAC
:1031400000C8060C00BC060C00B0060C00A4060B60
:103150000099060C008D060B0082060B0077060B0B
:10316000006C060B0061060A0057060B004C060AAD
:103170000042060A0038060A002E060A0024060A43
:10318000001A060A001006090007060A00FD0509D4
:1031900000F4050900EB050900E2050900D905095D
:1031A00000D0050900C7050900BE050900B50508DE
:1031B00000AD050800A50509009C05080094050858
:1031C000008C050800840508007C050800740508CB
:1031D000006C050700650508005D05070056050839
:1031E000004E0507004705070040050800380507A1
:1031F00000310507002A050700230507001C050606
:1032000000160507000F0507000805060002050760
:1032100000FB040600F5040700EE040600E80406BF
:1032200000E2040700DB040600D5040600CF040614
:1032300000C9040600C3040600BD040600B7040666
:1032400000B1040500AC040600A6040600A00405B5
:10325000009B04060095040500900406008A0405FE
:103260000085040500800406007A04050075040545
:1032700000700405006B0405006604050061040588
:10328000005C04050057040500520405004D0405C8
:103290000048040500430405003E0404003A040508
:1032A0000035040500300404002C04050027040444
:1032B00000230405001E0404001A0404001604057B
:1032C00000110404000D04040009040500040404B2
:1032D0000000040400FC030400F8030400F40304E9
:1032E00000F0030400EC030400E8030400E403041A
:1032F00000E0030400DC030400D8030400D403044A
:1033000000D0030400CC030400C8030300C503037A
:103310000024F404D9201BC40C5C0E9804C4095F7B
:103320000265077101F405F900FB04B30048048746
:1033300000C10369005803550003034500BE023A6B
:10334000008402310053022A0029022500040220D1
:1033500000E4011C00C8011900AF01170098011416
:103360000084011300710110006101100051010E71
:103370000043010D0036010B002B010B0020010B57
:1033800000150109000C01090003010800FB0008F9
:1033900000F3000800EB000700E4000600DE000672
:1033A00000D8000600D2000600CC000500C70005CA
:1033B00000C2000500BD000400B9000400B500040F
:1033C00000B1000400AD000400A9000400A5000342
:1033D00000A20003009F0004009B0003009800036C
:1033E000009500020093000300900003008D00028E
:1033F000008B0003008800020086000200840003A6
:1034000000810002007F0002007D0002007B0002BC
:1034100000790002007700010076000200740002CB
:103420000072000100710002006F0002006D0001D7
:10343000006C0002006A00010069000200670001E0
:1034400000660001006500010064000200620001E6
:103450000061000100600001005F0002005D0001EA
:10346000005C0001005B0001005A000100590001EE
:1034700000580001005700010056000100550001EE
:1034800000540001005300000053000100520001ED
:103490000051000100500001004F0001004E0000EB
:1034A000004E0001004D0001004C0001004B0000E7
:1034B000004B0001004A00010049000100480000E3
:1034C00000480001004700010046000000460001DE
:1034D00000450000004500010044000100430000D9
:1034E00000430001004200000042000100410000D2
:1034F0000041000100400001003F0000003F0001CA
:10350000003E0000003E0001003D0000003D0001C3
:10351000003C0000003C0000003C0001003B0000BB
:10352000003B0001003A0000003A000100390000B1
:1035300000390001003800000038000000380001A8
:1035400000370000003700010036000000360000A0
:103550000036000100350000003500000035000194
:10356000003400000034000000340001003300008B
:103570000033000000330001003200000032000080
:103580000032000100310000003100000031000174
:10359000003000000030000000300001002F00006B
:1035A000002F0000002F0000002F0001002E00005F
:1035B000002E0000002E0001002D0000002D000054
:1035C000002D0000002D0001002C0000002C000048
:1035D000002C0000002C0001002B0000002B00003C
:1035E000002B0000002B0001002A0000002A000030
:1035F000002A0000002A0001002900000029000024
:103600000029000000290000002900010028000016
:103610000028000000280000002800000028000109
:1036200000270000002700000027000000270000FE
:1036300000270001002600000026000000260000F0
:1036400000260000002600010025000000250000E3
:1036500000250000002500000025000000250001D5
:1036600000240000002400000024000000240000CA
:1036700000240001002300000023000000230000BC
:1036800000230000002300000023000000230001AD
:1036900000220000002200000022000000220000A2
:1036A0000022000000220001002100000021000093
:1036B0000021000000210000002100000021000086
:1036C0000021000100200000002000000020000078
:1036D000002000000020000000200000002000006A
:1036E00000200001001F0000001F0000001F00005C
:1036F000001F0000001F0000001F0000001F00014D
:10370000001E0000001E0000001E0000001E000041
:1037100000473830004D3435004D3435205A0047CD
:1037200037360057697A6172642073746174653A40
:103730002025640044697361626C65206661726D66
:10374000206D6F6465004661726D206E756D6265F7
:1037500072004D3834004D34340047323820570061
:103760004739390044697361626C65206661726D26
:10377000206D6F64653F0043616C696272617465BE
:1037800000506C65617365206C6F616420504C4122
:103790002066696C616D656E742066697273742E43
:1037A00000497320504C412066696C616D656E74F0
:1037B000206C6F616465643F0043616E63656C00FB
:1037C00046696C616D656E740053656C6563742049
:1037D000504C412066696C616D656E743A0052759B
:1037E0006E6E696E672057697A6172642077696CC2
:1037F0006C2064656C6574652063757272656E74A7
:103800002063616C6962726174696F6E20726573A6
:10381000756C747320616E642073746172742066B9
:10382000726F6D2074686520626567696E6E696E7F
:10383000672E20436F6E74696E75653F0050726528
:1038400068656174696E67206E6F7A7A6C652E2088
:10385000506C6561736520776169742E00456A65F7
:10386000637400556E6C6F61640055736520756EEE
:103870006C6F616420746F2072656D6F7665206671
:10388000696C616D656E74203120696620697420F1
:1038900070726F747275646573206F757473696488
:1038A00065206F66207468652072656172204D4DD9
:1038B0005520747562652E2055736520656A6563B1
:1038C000742069662069742069732068696464657E
:1038D0006E20696E20747562652E004C6F6164699C
:1038E0006E672066696C616D656E7400506C656111
:1038F000736520696E7365727420504C412066694F
:103900006C616D656E7420746F20746865206578D5
:103910007472756465722C207468656E20707265AF
:103920007373206B6E6F6220746F206C6F61642004
:1039300069742E00506C6561736520696E736572E1
:103940007420504C412066696C616D656E74207402
:103950006F2074686520666972737420747562657F
:10396000206F66204D4D552C207468656E20707256
:1039700065737320746865206B6E6F6220746F20AE
:103980006C6F61642069742E00596F752063616EDD
:1039900020616C7761797320726573756D65207431
:1039A00068652057697A6172642066726F6D204382
:1039B000616C6962726174696F6E202D3E20576977
:1039C0007A6172642E00506C65617365206368656E
:1039D000636B206F75722068616E64626F6F6B201D
:1039E000616E6420666978207468652070726F6209
:1039F0006C656D2E205468656E20726573756D65FB
:103A0000207468652057697A617264206279207237
:103A100065626F6F74696E67207468652070726983
:103A20006E7465722E00416C6C20697320646F6E39
:103A3000652E204861707079207072696E74696EAD
:103A4000672100506C6561736520636C65616E2051
:103A50006865617462656420616E64207468656E77
:103A600020707265737320746865206B6E6F622EB0
:103A700000446F20796F752077616E7420746F2019
:103A8000726570656174206C617374207374657005
:103A900020746F20726561646A7573742064697341
:103AA00074616E6365206265747765656E206E6F04
:103AB0007A7A6C6520616E64206865617462656401
:103AC0003F00492077696C6C2073746172742074B4
:103AD0006F207072696E74206C696E6520616E640F
:103AE00020796F752077696C6C20677261647561ED
:103AF0006C6C79206C6F77657220746865206E6FCE
:103B00007A7A6C6520627920726F746174696E676D
:103B100020746865206B6E6F622C20756E74696C02
:103B200020796F75207265616368206F7074696DAC
:103B3000616C206865696768742E20436865636BF3
:103B40002074686520706963747572657320696E8E
:103B5000206F75722068616E64626F6F6B20696E92
:103B600020636861707465722043616C6962726180
:103B700074696F6E2E004E6F7720492077696C6CE8
:103B80002063616C69627261746520646973746139
:103B90006E6365206265747765656E207469702058
:103BA0006F6620746865206E6F7A7A6C6520616E2E
:103BB0006420686561746265642073757266616310
:103BC000652E00497320697420504C412066696C51
:103BD000616D656E743F0053656C656374206E6F34
:103BE0007A7A6C6520707265686561742074656DA1
:103BF0007065726174757265207768696368206D9D
:103C000061746368657320796F7572206D61746586
:103C10007269616C2E004E6F7720492077696C6C59
:103C20002070726568656174206E6F7A7A6C6520A9
:103C3000666F7220504C412E0049732066696C619A
:103C40006D656E74206C6F616465643F004973201C
:103C500066696C616D656E742031206C6F6164659E
:103C6000643F004E6F7720492077696C6C2070723A
:103C70006568656174206E6F7A7A6C6520666F7214
:103C800020504C412E00492077696C6C2072756E73
:103C9000207A2063616C6962726174696F6E206E54
:103CA0006F772E004E6F772072656D6F766520748A
:103CB00068652074657374207072696E7420667212
:103CC0006F6D20737465656C2073686565742E0074
:103CD000506C656173652072656D6F7665207368E1
:103CE000697070696E672068656C706572732066B4
:103CF000697273742E00492077696C6C2072756E3E
:103D00002078797A2063616C6962726174696F6E80
:103D1000206E6F772E2049742077696C6C20746157
:103D20006B6520617070726F782E203132206D6962
:103D30006E732E0046697273742C20492077696C6B
:103D40006C2072756E207468652073656C6674658E
:103D5000737420746F20636865636B206D6F737478
:103D600020636F6D6D6F6E20617373656D626C792A
:103D70002070726F626C656D732E0048692C20494B
:103D800020616D20796F7572204F726967696E616D
:103D90006C205072757361206933207072696E7483
:103DA00065722E20576F756C6420796F75206C6971
:103DB0006B65206D6520746F206775696465207977
:103DC0006F75207468726F756768207468652073FA
:103DD000657475702070726F636573733F00452D55
:103DE000636F7272656374005A2D636F72726563DC
:103DF0007400592D636F727265637400582D636F80
:103E000072726563740053706F6F6C4A6F696E20D5
:103E100020205B4E2F415D0053706F6F6C4A6F69BD
:103E20006E2020205B6F66665D0053706F6F6C4A7A
:103E30006F696E202020205B6F6E5D00536F756E82
:103E4000642020202020205B6C6F75645D00536F20
:103E5000756E642020202020205B6D7574655D00E8
:103E6000536F756E64202020205B73696C656E74DF
:103E70005D00536F756E642020202020205B6F6EE4
:103E800063655D00536F756E642020202020205BE9
:103E90006C6F75645D00536F72743A20202020208F
:103EA000205B6E6F6E655D00536F72743A20205B0D
:103EB000616C7068616265745D00536F72743A2062
:103EC00020202020205B74696D655D0053442063D1
:103ED00061726420205B6E6F726D616C5D00534493
:103EE0002063617264205B666C73684169725D0077
:103EF00052506920706F727420202020205B6F6EFA
:103F00005D0052506920706F7274202020205B6F1A
:103F100066665D0054656D702E2063616C2E2020F6
:103F2000205B6F6E5D0054656D702E2063616C2E9A
:103F300020205B6F66665D004C696E2E20636F7299
:103F400072656374696F6E0046616E7320636865A5
:103F5000636B20205B6F66665D0046616E73206355
:103F60006865636B2020205B6F6E5D00462E2061CC
:103F700075746F6C6F6164205B6F66665D00462EC2
:103F8000206175746F6C6F616420205B6F6E5D00E3
:103F9000462E206175746F6C6F6164205B4E2F41FB
:103FA0005D0046696C2E2073656E736F72205B4EE8
:103FB0002F415D0044697361626C652073746570A4
:103FC00070657273004D6F76652061786973005477
:103FD000656D70657261747572650054656D702EE3
:103FE0002063616C6962726174696F6E00526573FF
:103FF00065742058595A2063616C6962722E0050B2
:1040000049442063616C6962726174696F6E004239
:104010006564206C6576656C20636F72726563748D
:10402000004D65736820426564204C6576656C6957
:104030006E670043616C696272617465205A004367
:10404000616C6962726174652058595A0053656CDD
:1040500066746573742020202020202020200046D4
:1040600069727374206C617965722063616C2E00D3
:1040700057697A617264004C6F61642066696C6193
:104080006D656E742035004C6F61642066696C61EB
:104090006D656E742034004C6F61642066696C61DC
:1040A0006D656E742033004C6F61642066696C61CD
:1040B0006D656E742032004C6F61642066696C61BE
:1040C0006D656E742031004C6F616420616C6C0012
:1040D0004C6F61642066696C616D656E742035009B
:1040E0004C6F61642066696C616D656E742034008C
:1040F0004C6F61642066696C616D656E742033007D
:104100004C6F61642066696C616D656E742032006D
:104110004C6F61642066696C616D656E742031005E
:10412000456A6563742066696C616D656E742035DF
:1041300000456A6563742066696C616D656E742004
:104140003400456A6563742066696C616D656E74E0
:10415000203300456A6563742066696C616D656E25
:1041600074203200456A6563742066696C616D6510
:104170006E74203100506C656173652070756C6CD5
:10418000206F75742066696C616D656E7420696D51
:104190006D6564696174656C7900556E6C6F6164FE
:1041A000696E672066696C616D656E740057697A27
:1041B00061726420656E642073746174653A2025B1
:1041C000640A0043686F6F736520636F6C6F723AA7
:1041D000004D3730322043004661726D206E756DA0
:1041E000626572004D363030004D3234004D32334E
:1041F00020257300052E2E00526573756D696E675C
:10420000207072696E7400537570706F727400461E
:1042100061696C207374617473204D4D5500466163
:10422000696C20737461747300537461746973747E
:1042300069637320200043616C6962726174696F05
:104240006E004175746F4C6F61642066696C616DBE
:10425000656E7400456A6563742066696C616D659E
:104260006E7400556E6C6F61642066696C616D657B
:104270006E74004C6F616420746F206E6F7A7A6C7C
:1042800065004C6F61642066696C616D656E7400D9
:104290004E6F2053442063617264005072696E74E3
:1042A0002066726F6D20534400526573756D6520F2
:1042B0007072696E74005061757365207072696EFA
:1042C0007400507265686561740054756E65004CC9
:1042D0006976652061646A757374205A0046696E58
:1042E000697368696E67206D6F76656D656E74734E
:1042F00000536F756E642020202020205B6C6F754A
:10430000645D00536F756E642020202020205B6D5B
:104310007574655D00536F756E64202020205B739B
:10432000696C656E745D00536F756E64202020208B
:1043300020205B6F6E63655D00536F756E64202097
:10434000202020205B6C6F75645D00437261736890
:10435000206465742E20205B4E2F415D0043726106
:104360007368206465742E2020205B6F6E5D0043AF
:1043700072617368206465742E20205B6F66665DD1
:10438000004D6F6465202020205B537465616C7460
:10439000685D004D6F646520202020205B4E6F72A9
:1043A0006D616C5D0046696C2E2073656E736F7273
:1043B00020205B6F6E5D0046696C2E2073656E7306
:1043C0006F72205B6F66665D004368616E67652093
:1043D00066696C616D656E7400466C6F7700537032
:1043E0006565640046616E207370656564004265B2
:1043F00064004E6F7A7A6C650053657474696E67F9
:1044000073005072696E742061626F72746564002B
:10441000596573004E6F0053746F70207072696E2F
:10442000740046696C6520696E636F6D706C6574AD
:10443000652E20436F6E74696E756520616E7977A5
:1044400061793F00496E666F2073637265656E0027
:104450004D61696E0000002110422063308440A548
:1044600050C660E770088129914AA16BB18CC1AD3B
:10447000D1CEE1EFF13112100273325222B55294D3
:1044800042F772D662399318837BB35AA3BDD39C8B
:10449000C3FFF3DEE36224433420040114E664C75F
:1044A00074A44485546AA54BB528850995EEE5CFDB
:1044B000F5ACC58DD55336722611163006D776F673
:1044C000669556B4465BB77AA719973887DFF7FE2B
:1044D000E79DD7BCC7C448E5588668A778400861FF
:1044E0001802282338CCC9EDD98EE9AFF94889697B
:1044F000990AA92BB9F55AD44AB77A966A711A5013
:104500000A333A122AFDDBDCCBBFFB9EEB799B58CA
:104510008B3BBB1AABA66C877CE44CC55C222C039E
:104520003C600C411CAEED8FFDECCDCDDD2AAD0B1A
:10453000BD688D499D977EB66ED55EF44E133E32B2
:104540002E511E700E9FFFBEEFDDDFFCCF1BBF3A6A
:10455000AF599F788F8891A981CAB1EBA10CD12D59
:10456000C14EF16FE18010A100C230E3200450255C
:104570004046706760B9839893FBA3DAB33DC31CD0
:10458000D37FE35EF3B1029012F322D232354214AC
:104590005277625672EAB5CBA5A89589856EF54F1C
:1045A000E52CD50DC5E234C324A0148104667447FC
:1045B0006424540544DBA7FAB79987B8975FE77E70
:1045C000F71DC73CD7D326F2369106B0165766764C
:1045D00076154634564CD96DC90EF92FE9C899E9BC
:1045E000898AB9ABA94458654806782768C018E19C
:1045F000088238A3287DCB5CDB3FEB1EFBF98BD810
:104600009BBBAB9ABB754A545A376A167AF10AD0EB
:104610001AB32A923A2EFD0FED6CDD4DCDAABD8B5B
:10462000ADE89DC98D267C076C645C454CA23C833B
:104630002CE01CC10C1FEF3EFF5DCF7CDF9BAFBAAF
:10464000BFD98FF89F176E367E554E745E932EB28B
:104650003ED10EF01E7C3C3E5E2B3D3F2F5B5D3B12
:104660002C2A225C0022206661696C65643A204233
:1046700075666665722066756C6C21002200656E39
:10468000717565696E6720220020003E003E0020A3
:10469000003E003E0054656D706572617475726510
:1046A0002063616C6962726174696F6E2066616912
:1046B0006C65642E20436F6E74696E756520776932
:1046C0007468207072657373696E67207468652002
:1046D0006B6E6F622E0054656D70657261747572D9
:1046E000652063616C6962726174696F6E20646FCA
:1046F0006E652E20436F6E74696E756520776974E0
:1047000068207072657373696E6720746865206BCA
:104710006E6F622E0054656D70657261747572659E
:104720002063616C6962726174696F6E2066616991
:104730006C65640054656D70657261747572652096
:1047400063616C6962726174696F6E20697320665F
:10475000696E697368656420616E64206163746961
:1047600076652E2054656D702E2063616C696272CF
:104770006174696F6E2063616E2062652064697385
:1047800061626C656420696E206D656E752053658D
:104790007474696E67732D3E54656D702E2063616D
:1047A0006C2E004E2F410020203000202031004987
:1047B000523A0046494E44413A0050494E44413A2B
:1047C0000053656E736F7220737461746500457871
:1047D000747275646572004D6F7665205A004D6F76
:1047E00076652059004D6F76652058001B5B324A74
:1047F000437261736820646574656374696F6E20C9
:1048000063616E1B5B313B30486265207475726E6C
:104810006564206F6E206F6E6C7920696E1B5B3251
:104820003B30484E6F726D616C206D6F6465001B8C
:104830005B324A5741524E494E473A1B5B313B303F
:1048400048437261736820646574656374696F6E50
:104850001B5B323B304864697361626C656420693C
:104860006E1B5B333B3048537465616C7468206D1C
:104870006F6465004175746F6C6F6164696E672069
:1048800066696C616D656E7420617661696C6162E8
:104890006C65206F6E6C79207768656E2066696C38
:1048A000616D656E742073656E736F72206973201D
:1048B0007475726E6564206F6E2E2E2E00455252F6
:1048C0004F523A2046696C616D656E742073656E57
:1048D000736F72206973206E6F7420726573706FCE
:1048E0006E64696E672C20706C6561736520636807
:1048F00065636B20636F6E6E656374696F6E2E0007
:1049000043757272656E74005573656420647572C8
:10491000696E67207072696E74005049442063614B
:104920006C2E2066696E6973686564005049442086
:1049300063616C2E202020202020202020202000B9
:10494000506C656173652077616974004D31313752
:10495000204669727374206C617965722063616CA2
:104960002E005072696E7420706175736564004921
:104970006E76616C6964205049442063616C2E201E
:10498000726573756C74732E204E6F742073746F20
:1049900072656420746F20454550524F4D2E004D76
:1049A000353030004731205A3135204631353030EE
:1049B00000473931004731205835302059313930DE
:1049C00020453020463730303000473930004D37F1
:1049D0003032004D3730322043004D3730322055D1
:1049E000004D373032004D37303220430047312000
:1049F0005A313520463135303000473931004731A2
:104A00002058353020593139302045302046373054
:104A10003030004D383300473930004D3834004DC8
:104A2000313034205330004D3834004D373032208F
:104A30004300473120583130205931383020463436
:104A4000303030004731205A313020463133303059
:104A50002E303030004D313430205330004D313065
:104A60003420533000473120452D302E303735303B
:104A7000302046323130302E3030303030004D3141
:104A800030370047312058353020593535204533EF
:104A90002E363237373300473120583230302059E4
:104AA00035352045302E34393338360047312058DB
:104AB000323030205937352045332E3632373733B0
:104AC00000473120583530205937352045302E34B5
:104AD00039333836004731205835302059393520A0
:104AE00045332E3632373733004731205832303095
:104AF000205939352045302E343933383600473186
:104B0000205832303020593131352045332E36325D
:104B1000373733004731205835302059313135206F
:104B200045302E343933383600473120583530205F
:104B3000593133352045332E36323737330047313C
:104B4000205832303020593133352045302E36361A
:104B50003137340047312058323030205931353523
:104B60002045322E36323737330047312058313026
:104B700030205931353520453200473120583735FE
:104B800020593135352045322E3500473120463108
:104B9000303830004731205A302E313530204637FA
:104BA0003230302E303030004731205835302059E7
:104BB000313535004731204634303030004D323009
:104BC00034205331303030004731205A35204637B9
:104BD0003230302E30303000473120452D312E35E7
:104BE000303030302046323130302E3030303030BE
:104BF000004D3833004739300047323100473932F1
:104C00002045302E3000473120583130302E3020B2
:104C10004531322E352046313030302E300047318C
:104C2000205836302E302045392E30204631303055
:104C3000302E300047312058352E302045342E306C
:104C40002046313030302E30004731205A302E325D
:104C5000302046313030302E300047312058353545
:104C60002E30204532352046313430302E3000474A
:104C70003120592D322E302046313030302E300048
:104C8000473120583234302E30204532352E3020F6
:104C90002046323230302E30004739322045302E17
:104CA00030004731205A302E332046313030302EFC
:104CB00030004731205835352E302045382E3020F1
:104CC00046323030302E300047312058352E3020DB
:104CD0004533322E302046313830302E30004731C7
:104CE000205835352E30204533322E302046313095
:104CF00037332E30004731205A302E3420463130A1
:104D000030302E3000473120592D332E302046319F
:104D10003030302E30004D383300473932204530A6
:104D20002E3000473238004D313039205332313582
:104D3000004D31393020533630004D31343020535E
:104D40003630004D3130342053323135004D313062
:104D50003700000E1315110E000000041209120492
:104D60000000001C1F11111F00000006191803137A
:104D70000C00040E1F041C000000040A0A0A0A1199
:104D8000110E001F1511151F0000000103161C084D
:104D900000000000110A04110A040C12120C000099
:104DA00000002563252D3138532563002563252E0A
:104DB0003135533A2573253364002563252E31326E
:104DC000533A25732500457872656D6520737061CF
:104DD0006E206F6620746865205A2076616C756558
:104DE00073210000004041000000400000E4420048
:104DF00000004000005743000000400000574300FF
:104E000000C4420000E4420000C4420000404100EF
:104E100000C44200004041000042430000E4420060
:104E20000042430000574300004243205B6F666628
:104E30005D00426564206C6576656C696E6720660E
:104E400061696C65642E2053656E736F72206469AE
:104E5000646E7420747269676765722E204465629F
:104E6000726973206F6E206E6F7A7A6C653F20577F
:104E7000616974696E6720666F722072657365740C
:104E80002E0043616E6E6F7420656E7465722073C0
:104E900075626469723A2000534420636172642031
:104EA0006F6B006F70656E526F6F74206661696C16
:104EB000656400766F6C756D652E696E6974206629
:104EC00061696C656400534420696E697420666191
:104ED000696C0057726974696E6720746F20666927
:104EE0006C653A200046696C652073656C65637477
:104EF0006564002053697A653A200046696C652034
:104F00006F70656E65643A20001F1F1F1F1F1F1FF3
:104F10001F2E002E004E6F77206672657368206624
:104F2000696C653A20004E6F7720646F696E672068
:104F300066696C653A20002220706F730022207031
:104F40006172656E743A2200535542524F5554496E
:104F50004E452043414C4C207461726765743A227F
:104F600000747279696E6720746F2063616C6C20C5
:104F70007375622D67636F64652066696C65732065
:104F80007769746820746F6F206D616E79206C652D
:104F900076656C732E204D4158206C6576656C20CB
:104FA00069733A00536F7274696E672066696C6545
:104FB0007300536F6D652066696C65732077696C4B
:104FC0006C206E6F7420626520736F727465642E3E
:104FD000204D61782E204E6F2E206F662066696C02
:104FE000657320696E203120666F6C64657220667F
:104FF0006F7220736F7274696E672069732031302D
:10500000302E0046696C616D656E742073656E7339
:105010006F7200537761707065640046726F6E74D2
:105020002F6C6566742066616E7300417869730049
:1050300041786973206C656E677468004C6F6F739C
:10504000652070756C6C657900456E6473746F7063
:10505000206E6F742068697400456E6473746F709D
:10506000004D6F746F7200456E6473746F707300DF
:10507000576972696E67206572726F72004265646B
:10508000202F20486561746572004E6F7420636F35
:105090006E6E6563746564004865617465722F5453
:1050A0006865726D6973746F7200506C65617365C9
:1050B00020636865636B203A0053656C66746573A2
:1050C00074206572726F7220210046696C616D6593
:1050D0006E742073656E736F723A005072696E74ED
:1050E0002066616E3A004578747275646572206658
:1050F000616E3A0043616C6962726174696E672027
:10510000686F6D650053656C6674657374206661C5
:10511000696C6564202000416C6C20636F7272655D
:10512000637420202020202000436865636B696E33
:10513000672073656E736F72732000436865636BDD
:10514000696E6720686F74656E642020004368652F
:10515000636B696E67206265642020202020004315
:105160006865636B696E67205A20617869732020D7
:1051700000436865636B696E6720592061786973C5
:10518000202000436865636B696E67205820617852
:105190006973202000436865636B696E6720656EE4
:1051A0006473746F7073004572726F72202D207378
:1051B0007461746963206D656D6F727920686173C5
:1051C000206265656E206F766572777269747465AA
:1051D0006E00436172642072656D6F766564002DA8
:1051E0002D2D2D2D2D2D2D2D2D2D2D2D2D2D2D2DEF
:1051F0002D2D2D000000000000110A0450525553BF
:105200004133444657002079303D25640A00207818
:10521000303D25640A004F4B0A004552524F522040
:1052200061643D25640A002020207A303D25640A0F
:1052300000207A303D25640A002079303D25640A3B
:10524000002078303D25640A0078797A63616C5FCC
:1052500066696E645F706F696E745F63656E7465B6
:1052600072320A0000002100240027002A002D00CD
:105270003000330001010000040107010A010000B1
:105280002200250028002B002E00310034000201EE
:105290000000050108010B0100002000230026008A
:1052A00029002C002F00320000010000030106013C
:1052B000090105050505070508080808020202029C
:1052C0000A0A0808040404040101010101010101A2
:1052D0000303030303030303040707070C0C0C0C6D
:1052E0000C0C0C0C02020202060606060606060656
:1052F0000B0B0B0B0B0B0B0B07070A0A0A0A0A0A0C
:1053000005050504040408080102102020080810FF
:105310002040102040800201020108040201010225
:1053200004081020408080402010080402018004FE
:105330000201804020100804020108040201010259
:10534000040810204080010204081020408010084A
:105350000408801020400440801020400480000099
:105360000A0B02090C0D0E080703040100000000DF
:10537000000000000000000000000000000000002D
:1053800000000000000000000000121110000000EA
:10539000000000000000000000000000000000000D
:1053A00000000000000000000000000000000000FD
:1053B00000000000773235783230636C5F63666DD1
:1053C0000A00773235783230636C5F656E746572CF
:1053D0000A0020746F6F206C6F6E6720657874729E
:1053E0007573696F6E2070726576656E74656400A2
:1053F00020636F6C6420657874727573696F6E20BA
:1054000070726576656E74656400526573656E646E
:105410000025533A20256C640A25530A002079643C
:105420005F6D696E3D25752079645F6D61783D25FE
:10543000752079645F6176673D25752073685F61CB
:1054400076673D25750A002073745F73756D3D2581
:10545000752079645F73756D3D25752065725F7386
:10546000756D3D25752065725F6D61783D256868B5
:10547000750A00004B494C4C45442E20005072697F
:105480006E7465722068616C7465642E206B696C43
:105490006C28292063616C6C656421004B494C4C7D
:1054A0003A2025640A004D31303420496E76616C13
:1054B000696420657874727564657220004D3130BE
:1054C0003520496E76616C69642065787472756404
:1054D000657220004D31303920496E76616C696407
:1054E00020657874727564657220004D3231382001
:1054F000496E76616C696420657874727564657252
:1055000020004D32323120496E76616C696420652D
:105510007874727564657220006673656E736F725D
:105520005F6F715F6D656173737572655F73746FC3
:10553000702C20256868752073616D706C65730A26
:10554000006673656E736F725F6F715F6D65617317
:10555000737572655F73746172740A004D36303012
:10556000004653454E534F525F5245434F564552A6
:10557000006673656E736F725F7570646174652029
:105580002D204D3630300A006673656E736F725F82
:105590006572725F636E74203D20300A00473120CF
:1055A0004533204632303000473120452D332046E8
:1055B000323030004D3730310020573A0020453A24
:1055C00000543A005A206C6976652061646A7573EC
:1055D00074206F7574206F662072616E67652E206F
:1055E00053657474696E6720746F20302E20436C8D
:1055F00069636B20746F20636F6E74696E75652EBE
:10560000005A206C6976652061646A757374206F36
:105610007574206F662072616E67652E2053657405
:1056200074696E6720746F20300048656174696E1C
:10563000672064697361626C6564206279207361BC
:10564000666574792074696D65722E001000C90258
:1056500010012C014001220170011801B0010E015E
:10566000F00104015002FA00B002F0003003E6003D
:10567000D003DC009004D2007005C800A006BE0074
:105680000008B400B009AA00D00BA000600E96007C
:1056900060118C000015820020197800C01D6E007A
:1056A000A0226400B0275A00902C50000031460020
:1056B000E0343C0010383200903A2800603C1E0074
:1056C000A03D1400803E0A00203F000070012C0124
:1056D00090012701B0012201C0011D01F001180154
:1056E0001002130130020E01600209019002040150
:1056F000C002FF000003FA004003F5008003F00041
:10570000D003EB002004E6007004E100E004DC00BC
:105710004005D700C005D2004006CD00D006C80025
:105720008007C3003008BE00F008B900C009B4000B
:10573000B00AAF00B00BAA00D00CA500000EA0006C
:10574000500F9B00C01096005012910000148C0066
:10575000C0158700B0178200B0197D00D01B7800FB
:10576000001E730040206E0090226900F024640047
:1057700040275F0090295A00E02B5500102E500062
:1057800020304B0010324600E033410090353C00A1
:105790001037370070383200A0392D00B03A280099
:1057A000A03B2300603C1E00103D1900903D1400FA
:1057B000103E0F00703E0A00C03E0500003F000092
:1057C00090137D00B0157800F0177300601A6E001A
:1057D000F01C6900A01F640050225F0020255A00C1
:1057E000E0275500902A5000202D4B00A02F4600A6
:1057F000F031410010343C00F0353700A037320062
:1058000020392D00603A2800703B2300603C1E00C8
:10581000203D1900C03D1400403E0F00A03E0A008C
:10582000F03E0500403F0000703FFBFF903FF6FF59
:10583000B03FF1FFC03FECFFD03FE7FFE03FE2FFAA
:10584000F03FDDFFF03FD8FF20484F54454E442045
:10585000544845524D414C2052554E4157415900F4
:10586000204845415442454420544845524D414CFE
:105870002052554E4157415900544845524D414CD4
:105880002052554E41574159004245442054484505
:10589000524D414C2052554E4157415900205448D9
:1058A00045524D414C2052554E41574159202820D8
:1058B0005052454845415420484F54454E442900D4
:1058C00020544845524D414C2052554E4157415964
:1058D00020282050524548454154204845415442D3
:1058E0004544290050524548454154204552524FA5
:1058F00052004245442050524548454154204552AB
:10590000524F52004572723A204D494E54454D5007
:10591000204245440054656D70657261747572650E
:1059200020686561746564206265642073776974BA
:1059300063686564206F66662E204D494E54454D60
:105940005020747269676765726564202100457232
:10595000723A204D494E54454D50003A20457874D6
:105960007275646572207377697463686564206F0B
:1059700066662E204D494E54454D5020747269671D
:105980006765726564202100504154393132355FBA
:105990005245535F593D256868750A005041543996
:1059A0003132355F5245535F583D256868750A00AE
:1059B0005553415254322072782046756C6C212127
:1059C000210A0053657474696E67732053746F7293
:1059D00065640053746F7265642073657474696ED6
:1059E00067732072657472696576656400486172D8
:1059F00064636F6465642044656661756C742053EC
:105A0000657474696E6773204C6F616465640056D9
:105A10003200000000C8420000C8420000C8430035
:105A2000008C430000484300004843000040410010
:105A300000F042E8030000E8030000C8000000880E
:105A400013000000409C4400409C44000000000003
:105A5000000000204E00000000204100002041CD49
:105A6000CCCC3E0000204000000000000000000000
:105A7000000000CDCCCC3E3D0A8141FF08433EB042
:105A800099AB438F42FC42E65A343F4C62B045002A
:105A90000000000040400000344200000000000010
:105AA000000000000041000000E03F0000C842008C
:105AB00000C842000040410000F042C0030000C0A6
:105AC000030000C800000088130000454550524FF5
:105AD0004D204572726F720057616974696E67205C
:105AE000666F72206E6F7A7A6C6520616E642062D8
:105AF000656420636F6F6C696E670053656C662028
:105B000074657374204F4B0053656C662074657325
:105B1000742073746172742020004578747220665A
:105B2000616E2073706565643A202564200A005018
:105B300072696E742066616E2073706565643A20C8
:105B40002564200A005465737420323A0A004578AF
:105B500074722066616E2073706565643A202564F6
:105B6000200A005072696E742066616E2073706541
:105B700065643A202564200A005465737420313A24
:105B80000A006C63645F73656C66636865636B5F72
:105B9000617869732025642C2025640A004D38340F
:105BA000004731205A3135204631303030004732FD
:105BB0003820570025632041584953205347313D31
:105BC00025640A0041786973206C656E67746820EB
:105BD000646966666572656E63653A252E33660A8A
:105BE000004D656173757265642061786973206C1E
:105BF000656E6774683A252E33660A00436F6E74CB
:105C0000696E7565207769746820616E6F74686568
:105C10007220626F7764656E3F002500202020208F
:105C20002020002020202020200045524153494EB2
:105C30004720616C6C206461746100466163746F1D
:105C400072792052455345540000007F4300805430
:105C5000430000524300000000000080C09A9919E0
:105C60003E00000000000080C09A99193E0000A08C
:105C7000400000A04000000040253364207374659C
:105C8000703D253264206D73636E743D2534640A63
:105C90000000007F43008058439AD95143FFFFFF23
:105CA00046696C616D656E74206F7574206F662037
:105CB00072616E6765202564200A0067636F646502
:105CC0005F4D37303120626567696E0A00332E35CB
:105CD0002E32007263006265746100616C706861ED
:105CE000006465760078797A63616C5F73706972BD
:105CF000616C322063783D25642063793D25642002
:105D00007A303D256420647A3D256420726164699F
:105D100075733D25642061643D25640A00746D63DC
:105D2000323133305F676F746F5F73746570202535
:105D300064202564202564202564200A002E006F3D
:105D400070656E206661696C65642C2046696C65BF
:105D50003A20004D3234004D3233202573006175F6
:105D6000746F25692E670022206661696C65643A4C
:105D7000204275666665722066756C6C2100456E02
:105D8000717565696E6720746F207468652066722E
:105D90006F6E743A2022004572726F723A002200D0
:105DA000456E717565696E6720746F207468652033
:105DB00066726F6E743A2022006563686F3A004520
:105DC00072723A205052494E542046414E2045525C
:105DD000524F52005072696E742066616E2073706B
:105DE000656564206973206C6F77657220746865DF
:105DF0006E206578706563746564004572723A2040
:105E0000455854522E2046414E204552524F520082
:105E100045787472756465722066616E2073706572
:105E20006564206973206C6F776572207468656E95
:105E3000206578706563746564002F2F206163743A
:105E4000696F6E3A7061757365004572723A204DE4
:105E5000415854454D50003A204578747275646538
:105E600072207377697463686564206F66662E209C
:105E70004D415854454D502074726967676572658D
:105E8000642021004572723A204D415854454D50CE
:105E9000204245440054656D706572617475726589
:105EA0002068656174656420626564207377697435
:105EB00063686564206F66662E204D415854454DD9
:105EC00050207472696767657265642021004669B5
:105ED0006C2E2058643A2533642059643A25336483
:105EE0000A496E743A202533642020536875743A49
:105EF000202533640046696C616D656E742073659E
:105F00006E736F720A69732064697361626C656491
:105F10002E001B5B303B304825533A20253464204B
:105F200052504D0A25533A20202534642052504DBA
:105F30000A005072696E742046414E004E6F7A7AA4
:105F40006C652046414E00546F74616C004C617367
:105F500074207072696E74004D4D55206C6F6164D1
:105F6000206661696C73004D4D55206661696C73E4
:105F7000004C617374207072696E74206661696C84
:105F800075726573004D4D5520706F776572206690
:105F900061696C73004D4D55206C6F6164206661C2
:105FA000696C73004D4D55206661696C7300546FC8
:105FB00074616C206661696C75726573004372610F
:105FC00073680046696C616D2E2072756E6F757412
:105FD0007300506F776572206661696C75726573C6
:105FE00000546F74616C206661696C757265730032
:105FF00043726173680046696C616D2E2072756E24
:106000006F75747300506F776572206661696C7587
:10601000726573004C617374207072696E742066CF
:1060200061696C7572657300546F74616C004C61CA
:106030007374207072696E7400416D6269656E746C
:1060400000426564004E6F7A7A6C650042656C743C
:106050002073746174757300436F6F6C646F776E37
:10606000001B5B303B304825531B5B313B314825DF
:10607000532020252D33641B5B323B3148255320B0
:1060800020252D33641B5B333B3148001B5B303BC9
:10609000304825531B5B313B314825532020252DAB
:1060A00033641B5B323B314825532020252D33645C
:1060B0001B5B333B3148255320252D3364001B5B8C
:1060C000303B304825531B5B313B31482553202062
:1060D000252D33641B5B323B314825532020252D71
:1060E00033641B5B333B3148255320205820252D3A
:1060F000336420205920252D3364001B5B303B3056
:106100004825531B5B313B314825532020252D3337
:10611000641B5B323B314825532020252D33641B03
:106120005B333B3148255320205820252D336420F4
:10613000205920252D3364001B5B323B3148255309
:106140003A2020256425631B5B333B314850494E80
:1061500044413A2020202025642563001B5B303B0E
:10616000314825533A202020256425631B5B313BB1
:10617000314825533A202020202020256425630023
:106180001B5B313B31485057523A202020202020C1
:1061900025642E25303164561B5B323B3148424525
:1061A000443A20202020202025642E2530316456BA
:1061B000001B5B303B314825531B5B313B32485859
:1061C0002025641B5B323B32485920256400464C35
:1061D0004558202D20203234302F353000505020AB
:1061E00020202D20203235342F31303000484950C6
:1061F00053202D20203232302F3130300041425395
:1062000020202D20203235352F313030005045549C
:1062100020202D20203233302F383500504C4120A3
:10622000202D20203231352F36300041425320209E
:1062300020202D20203235352F313030006E6F7AFE
:106240007A6C65202D20203235302F300066617247
:106250006D2020202D20203235302F363000256350
:10626000252E3132533A2573252B30362E316600D8
:10627000202020202020202020202020202020201E
:1062800020202020003E003E0020003E003E002056
:10629000004E6F74207370696E6E696E6700537084
:1062A000696E6E696E67004C65667420686F746510
:1062B0006E642066616E3F0046726F6E742070726D
:1062C000696E742066616E3F0046616E207465736E
:1062D000740078014A0111241FBECFEFD1E2DEBF66
:1062E000CDBF00E00CBF16E0A0E0B2E0EAEFFEE7B1
:1062F00003E00BBF02C007900D92A03BB107D9F796
:1063000029E1A0EBB6E001C01D92A13DB207E1F783
:1063100011E3CAE6D1E300E006C021970109802F0E
:10632000FE010F9484BEC936D10780E00807A9F7A3
:106330000F946D940D946CBF0C9400002F923F92BB
:106340004F925F926F927F928F929F92AF92BF9285
:10635000CF92DF92EF92FF920F931F93CF93DF9331
:10636000CDB7DEB7C757D1090FB6F894DEBF0FBE61
:10637000CDBF8091841390918513892B11F40C94D7
:10638000FB7182E090E090932602809325028AE3DD
:1063900093E00F943D608823B1F08091600D90915F
:1063A000610D6AE270E005960F94EBBE009711F064
:1063B000DC011C928091600D9091610D05960F9407
:1063C0009C270C94146DC0907315D09074158601A1
:1063D00007571C4E46E050E061E670E1C8010F949B
:1063E0001AB2892B09F0EFC08FE393E00F943D6060
:1063F000882309F49BC088E50F94B7AC182F89E572
:106400000F94B7AC811112600F9403898091B1068B
:1064100001E0080F0093B106811105C08AE596E1FD
:106420000E94CDEB0EC048EC5FEA60E070E08AE5C8
:1064300096E10E9488EB882331F010925A16109250
:10644000B10601E007C0033049F710925A161092C6
:10645000B10600E081E00F944E160F94441682E0DE
:106460000F94BE0E10FF15C086E69FE00F9417B97B
:1064700061E0680F86E69FE00F9429B985E09FE010
:106480000F9424B9BC016F5F7F4F85E09FE00F94AC
:1064900043B911FF15C088E69FE00F9417B961E07A
:1064A000680F88E69FE00F9429B983E09FE00F947E
:1064B00024B9BC016F5F7F4F83E09FE00F9443B925
:1064C00081E00F944E1682E00F94BE0E8AE392E1B3
:1064D0000F94232640E061E081E00F94076F0F9452
:1064E0000389002321F061E08CE69DE01BC0E09170
:1064F000070DF0E0EE0FFF1FEB58FA4E11821082ED
:1065000040E060E08CE192E10E9408FC182F81E0FD
:106510000F944E1661E0112319F08EE59DE002C044
:1065200081E59DE00E9415EA0C94146D8EE493E0E1
:106530000F943D60882379F080917F0E882331F09D
:1065400060E070E080E89FE30E94DE8781E0809356
:106550000F020C94146D8CE593E00F943D6088233A
:1065600011F40C94146D10927F0E81E080930F0251
:106570008091110D811104C00E9472E70C94146D7A
:10658000813011F00C94146DE0E4FDE084918F01F2
:10659000882339F00F94A14F0F5F1F4FF8018491AA
:1065A000F7CF8AE00F94A14FE2E4F7E184918F01E5
:1065B000882311F40C94A56B0F94A14F0F5F1F4F0C
:1065C000F8018491F5CF44E050E06CE570E1C8013A
:1065D0000F941AB2892B09F00EC1860103571C4E85
:1065E00049E050E062E570E1C8010F941AB2892BCE
:1065F000D9F4F601EA56FC4E1081153431F01855E5
:10660000143010F00C94146D01C013E04AE050E017
:1066100060E070E0C60189569C4E0F94D1AF812F87
:106620000F94AC730C94146D49E050E068E470E191
:10663000C8010F941AB2892B61F5F601EA56FC4E97
:106640001081153431F01855143010F00C94146D7D
:1066500001C013E04AE050E060E070E0C6018956F6
:106660009C4E0F94D1AFE12FF0E0E75EF84F40E091
:1066700051E0008002C0569547950A94E2F7842FB6
:10668000880F880F81506823812F0F945A750C94BE
:10669000146D49E050E06EE370E1C8010F941AB246
:1066A000892B11F00C94146DF601EA56FC4E808192
:1066B000853449F008EA902E980EF3E0F91510F4AD
:1066C0000C94146D02C013E0912EE92CF12C5701AB
:1066D000AA0CBB1CF501E05DFD4F1081012F0F706E
:1066E000712E7294BFE07B22272D2770722E111F0E
:1066F0001127111F61816770660F162BF501EF5C82
:10670000FD4F8081882E869486948694382D337030
:10671000832E1A821982C60189569C4EDC012C9167
:106720002223E1F14AE050E0BE016F5F7F4F0F94FA
:10673000D1AF062F0F7089819A81009779F1FC0102
:106740002081222359F14AE050E0BE016F5F7F4F64
:106750000F94D1AF6770762E89819A810097F1F0FE
:10676000DC012C912223D1F04AE050E0BE016F5FA2
:106770007F4F0F94D1AF162F1F7089819A81009798
:1067800069F0FC012081222349F04AE050E0BE017B
:106790006F5F7F4F0F94D1AF6370862EF501E05D80
:1067A000FD4F972D97709295907F612F6795662783
:1067B0006795902B962B9083612F66951181107EA3
:1067C000882D8370880F880F880F162B182B118344
:1067D000C701845E9D4FD701A05EBD4FB701675EC4
:1067E000784FFC0120814C91DB016C91892D0E9436
:1067F000B6AD0C94146D89E693E00F943D60882348
:1068000021F00E9454B50C94146D89E793E00F9425
:106810003D60882309F4B5C18FE793E00F943D6094
:10682000882391F08091070F882311F40C94146D44
:106830000F94D653609370167093711680937216EE
:10684000909373160C94146D84E893E00F943D605C
:10685000882349F08091D60E8F938091D50E8F9327
:1068600082E297E03DC088E893E00F943D60882382
:1068700029F14091291050912A102CE3249FC00146
:10688000259F900D11249F938F9340912710509135
:106890002810249FC001259F900D11249F938F9352
:1068A0008BE097E09F938F930F9447B30F900F90D7
:1068B0000F900F900F900F900C94146D8CE893E054
:1068C0000F943D608823C9F08091070F882391F0D1
:1068D000809133078F93809132078F9388E097E000
:1068E0009F938F930F9447B30F900F900F900F903B
:1068F0000C94146D86EF96E0F0C08FE893E00F944F
:106900003D60882321F0109231070C94146D83E9C7
:1069100093E00F943D60882349F060E085EA9FE0B2
:106920000F9429B961E08AE390E1FCCD88E993E016
:106930000F943D60882321F00E9452A10C94146DA5
:106940008FE993E00F943D60882319F18091070F40
:106950008823C9F08AEA95E5DC018093FC1F9093B7
:10696000FD1FA093FE1FB093FF1F88E08093FB1FC5
:1069700098E10FB6F894A895909360000FBE8093AD
:106980006000F894FFCF85EA93E00F94A3500C9435
:10699000146D87EB93E00F943D60882339F180916B
:1069A000600D9091610D41E061E003960F94C61770
:1069B0008091A4189091A518A091A618B091A7183D
:1069C0008093511990935219A0935319B09354196D
:1069D0008CE998E10E94C4F18C010F94A14F0A3018
:1069E000110531F70F94786F0C94146D8AEB93E0D6
:1069F0000F943D60882381F00F94106781E08093AD
:106A000044078091600D9091610D41E060E0049633
:106A10000F94C6170C94146D8EEB93E00F943D60A9
:106A2000882309F45EC08091070F882309F453C0BE
:106A3000109277156091CB197091CC198BE390E08F
:106A40000F94C2B26091CB197091CC1983E590E09C
:106A50000F94C2B219821B821A82CE0101960E9443
:106A60007CEB00E010E0FF24F3948091250E9091E0
:106A7000260E2091270E3091280E821B930B8F77C4
:106A80009927892B81F00F94FD4EF0927715609134
:106A9000CB197091CC1990E00F94C2B20F5F1F4FC9
:106AA00010927715E2CF64E670E0CE0101960E9465
:106AB00053EB811103C003311105BCF281E08093D7
:106AC00077156091CB197091CC198AE090E00F9402
:106AD000C2B20C94146D8BEF94E00F946FB30C94CE
:106AE000146D81EC93E00F943D60882361F005EC18
:106AF00013E0F80181918F01882311F40C94A56BA8
:106B00000F94A14FF6CF80ED93E00F943D60882362
:106B100061F004ED13E0D8018D918D01882311F40B
:106B20000C94A56B0F94A14FF6CF83EF93E00F94D5
:106B30003D6081110C94146D88EF93E00F943D60DB
:106B4000882341F060E070E088EF9FE00E9491C5EB
:106B50000C94146D8BEF93E00F943D60882321F02B
:106B60000F94D6530C94146D80E094E00F943D6024
:106B7000882311F40C94146D80E00F9433620C940C
:106B8000146D8EE50F94B7AC8AAF81110C94146D1F
:106B900087E40F94B7ACF82E882311F40C94A34328
:106BA0000F94AFAC0F9402BB6C34710509F404C2AE
:106BB0007CF56430710509F4FCC054F46230710551
:106BC00009F4E2C00CF0E9C077FF6DC00C94974364
:106BD0006C31710509F43FC15CF46A30710509F448
:106BE00035C16B30710511F00C94974380E02FC1D3
:106BF0006E31710509F471C16B34710511F00C949B
:106C0000974308E210E0F8ECEF2EF6E0FF2EB5C156
:106C10006835710511F40C94146DECF4613571054F
:106C200011F40C945E4254F46F34710509F431C7C9
:106C30006035710509F459C70C94974366357105A1
:106C400011F40C9407436735710511F00C949743C8
:106C500081E00C9408436C35710511F40C941043D9
:106C60007CF46A35710511F40C940C436B35710595
:106C700011F00C94974381E080937A0F0C94146D7B
:106C80006236710511F40C9470436336710511F08E
:106C90000C9497431092070F60E084EC9FE00F94F0
:106CA00029B90C9492438091B30F81110C94146D07
:106CB0000F944CAB60916C0E70916D0E80916E0EC6
:106CC00090916F0E0F9440B46B017C01409058106E
:106CD0005090591060905A1070905B108090140F73
:106CE0009090150FA090160FB090170FA50194016A
:106CF000C301B2010F94A2B920E030E048EC52E4A5
:106D00000F94A9AD9B01AC01C701B6010F94EEBB76
:106D10001816D4F4A3019201C501B4010F94A2B9CD
:106D200020E030E048EC52E40F94A9ADA7019601B1
:106D30000F94A3B90F9408BB60936C0E70936D0E03
:106D400080936E0E90936F0E80911211882311F430
:106D50000C94126D88E50F94B7AC81110C94126DF0
:106D600089E50F94B7AC81110C94126D8AE50F94EC
:106D7000B7AC81110C94126D85E40F94B7AC8111FE
:106D80000C94E96C0C94126D8091B30F81110C94EA
:106D9000146D0F9409AC81E008C08091B30F81118C
:106DA0000C94146D0F9409AC80E00F941CA50C9406
:106DB000146D80E50F94B7AC882339F00F94AFAC15
:106DC0000F9408BB6B017C0103C0C12CD12C760150
:106DD00083E50F94B7AC882361F00F94AFAC20E04B
:106DE00030E04AE754E40F94A9AD0F9408BB6B015F
:106DF0007C01C114D104E104F10421F08DEE96E090
:106E00000F9423260F9403890F94D653C60ED71ED2
:106E1000E81EF91E0F94D65360937F0F7093800F76
:106E20008093810F9093820F0F94D6536C157D053C
:106E30008E059F0510F00C94146D0F94378280E03E
:106E40000F94614080E00F94BE0EEECF81E00F946E
:106E5000EBA20C94146D88E50F94B7AC8EAF0F9431
:106E6000A5AC1B012C0189E50F94B7AC682E0F94DB
:106E7000A5AC26966CAF7DAF8EAF9FAF26978AE507
:106E80000F94B7ACD82E0F94A5AC4B015C0187E5ED
:106E90000F94B7AC782E83E40F94B7AC7F928F93A6
:106EA000CD2C2696ECACFDAC0EAD1FAD2697262D55
:106EB000B201A1018EAD0F94276C0F900F90BEAD63
:106EC000B1110C94146D61100C94146D71100C942C
:106ED000146DD1100C94146D08C60F94038981E0D1
:106EE0000F94535E8C0180E090E0A8E4B4E48093BA
:106EF0005B0290935C02A0935D02B0935E0260E03F
:106F000070E080E291EC0F947E16809157108F9381
:106F1000809156108F93809155108F9380915410CB
:106F20008F93809153108F93809152108F93809103
:106F300051108F93809150108F9380914F108F93A9
:106F400080914E108F9380914D108F9380914C10B3
:106F50008F938EEE93E49F938F9381ED96E09F93B2
:106F60008F930F9447B3C8010F94325E0FB6F89415
:106F7000DEBF0FBECDBF0C94146DB801012E000C06
:106F8000880B990B0F9442B40E9437949F938F9370
:106F90007F936F931F930F93FF92EF920F9447B3DA
:106FA0000F5F1F4F0FB6F894DEBF0FBECDBF0F3679
:106FB000110519F70C94146D0F948D658A3F30F00C
:106FC00088E093E10E94ACFC0C94146D8091080D54
:106FD000882341F08091090D882321F080910A0DCA
:106FE000811106C081E08093831383E390E197C50C
:106FF00081EC92E10E94ACFC40E060E08EE09BE11D
:107000000E9408FC882309F493C080E090E0A0EA85
:10701000B0E48093541090935510A0935610B09301
:1070200057102091501030915110409152105091B2
:10703000531060914C1070914D1080914E109091B2
:107040004F10F7E06F2EFDE07F2E7F926F92812C24
:10705000912CA8E4AA2EA2E4BA2EB8E5CB2EB0E17A
:10706000DB2EE12CF12C00EA10E40F94EF2C80923F
:10707000541090925510A0925610B092571080E084
:1070800090E0A4E3B3E48093501090935110A09348
:107090005210B093531060914C1070914D1080912C
:1070A0004E1090914F107F926F928501740120E0F5
:1070B00030E044E353E40F94EF2C0F94038986EE01
:1070C0009AE10E94ACFCEAE4FEE1259135914591FC
:1070D000549120935010309351104093521050937C
:1070E0005310E6E4FEE1659175918591949160936A
:1070F0004C1070934D1080934E1090934F10E09071
:107100005410F090551000915610109157107F9226
:107110006F920F94EF2C0F94038941E060E080E0C0
:107120000F94076F0F900F900F900F900F900F908C
:1071300020E030E04CE052E46091881970918919A8
:1071400080918A1990918B190F94EEBB18160CF050
:10715000A4C08091070F8111A0C080E090E0A8EC4E
:10716000B2E48093541090935510A0935610B093AE
:107170005710209150103091511040915210509161
:10718000531060914C1070914D1080914E10909161
:107190004F10E7E0FDE0FF93EF93812C912C18E472
:1071A000A12E12E4B12E08E5C02E00E1D02EE12C74
:1071B000F12C08EC12E40F94EF2C80E090E0ACE0AE
:1071C000B2E48F8F98A3A9A3BAA30F946B1119826D
:1071D0001A821B821C82CE0101960F94257B10928D
:1071E0000C0D10920B0D19821A821B821C821D82BB
:1071F000CE0101960E94CDEB0F900F902F8D38A1FC
:1072000049A15AA1609188197091891980918A19B0
:1072100090918B190F94EEBB181694F58CEF91E1B9
:107220000E94FBFB64E080E00F94971182E00E94D3
:10723000FFB088E899E10E948AB60F94341083E089
:1072400094E00F943410CE014F960E948AB60F94AA
:10725000341085E094E00F94341088EE93E00F949E
:10726000C1440E94E19340E053E567E070E0CE0145
:1072700001960E9488EB882309F4C0CF10E001C07A
:1072800011E064EF71E581E00F944C1181E00F94FF
:107290004E16111102C080E0F8C381E00F944E1623
:1072A00081E090E09093260280932502E5E1F0E1F1
:1072B00084918F01882339F00F94A14F0F5F1F4FE6
:1072C000F8018491F7CF8AE00F94A14F1A821982B6
:1072D000C0908819D0908919E0908A19F0908B1984
:1072E00020E030E040EA50E4C701B6010F9491BAC3
:1072F0000F9402BB25E0269FA001279F500D11246B
:10730000BA01550F880B990B0F9442B43B01382EEC
:10731000292E20E030E04CE052E40F943CB487FF8B
:1073200006C0612C712CACE03A2EB2E42B2EC101C8
:10733000262D372D492F522DC701B6010F94EEBBD4
:10734000181674F420E030E040EA50E4F101662DB4
:10735000772D8F2F922D0F94A3B93B01382E292E14
:107360002F923F927F926F928FEA96E09F938F9336
:107370000F9447B320E030E040EF51E4F101662D77
:10738000772D8F2F922D0F94A2B920E030E04CE89A
:1073900052E40F94A3B90F9402BB70930C0D609349
:1073A0000B0D84E090E09093650E8093640E81E075
:1073B00090E09093F50E8093F40E86EE97E20F9492
:1073C000232680E090E0A0EAB0E4809354109093EC
:1073D0005510A0935610B093571020915010309133
:1073E0005110409152105091531060914C10709177
:1073F0004D1080914E1090914F10B7E04B2EBDE094
:107400005B2E5F924F92812C912C18E4A12E12E4F6
:10741000B12E08E5C02E00E1D02EE12CF12C00EABF
:1074200010E40F94EF2C80E090E0A0EAB1E48093A8
:107430004C1090934D10A0934E10B0934F1080E0DD
:1074400090E0A0E7B2E48093501090935110A09385
:107450005210B0935310E0905410F09055100091DA
:107460005610109157105F924F929C01AD0160E051
:1074700070E080EA91E40F94EF2C8AE999E9A9E1A0
:10748000BEE38093541090935510A0935610B09380
:10749000571020915010309151104091521050913E
:1074A000531060914C1070914D1080914E1090913E
:1074B0004F105F924F921AE9E12E19E9F12E09E17E
:1074C0001EE30F94EF2C0F9403890FB6F894DEBFE0
:1074D0000FBECDBF209188193091891940918A192A
:1074E00050918B19F101662D772D8F2F922D0F94CE
:1074F000EEBB18163CF488EE93E00F94C1440E9452
:10750000E193E8CF60E086EA9FE00F9429B980E03C
:1075100090E0A0EAB0E48093541090935510A093AB
:107520005610B09357102091501030915110409147
:1075300052105091531060914C1070914D108091E9
:107540004E1090914F1007E0402E0DE0502E5F92AC
:107550004F92812C912CE8E4AE2EE2E4BE2EF8E5A9
:10756000CF2EF0E1DF2EE12CF12C00EA10E40F9495
:10757000EF2CE6E4FEE1659175918591949160931D
:107580004C1070934D1080934E1090934F10EAE47E
:10759000FEE12591359145915491209350103093FF
:1075A00051104093521050935310E0905410F090AB
:1075B000551000915610109157105F924F920F94F2
:1075C000EF2C0F94038960E070E080E89FEB0F944C
:1075D0007E160F900F900F900F90882309F45BCECA
:1075E0003091541027963FAF2797409155102B9616
:1075F0004FAF2B97509156102F965FAF2F976091FA
:10760000571063966FAF63976F935F934F933F935A
:1076100082EA96E09F938F930F9447B30F900F9059
:107620000F900F900F900F908EEA9FE09FAF8EAF5C
:1076300044244A94542C13E2C12ED12CE12CF12C79
:107640008201B6010D2C000C880B990B0F9442B4EB
:107650004B015C0197012F5F3F4F3BAF2AAFDF9299
:10766000CF923F932F9346E656E05F934F930F944C
:1076700047B30F900F900F900F900F900F908FEFD8
:107680004816580611F40C94E771BE016F5F7F4FE6
:107690008EAD9FAD0E9491C5A5019401F101662DAB
:1076A000772D8F2F922D0F943CB41816A4F495E0EB
:1076B000E916F10471F095E0C90ED11CAFEF4A1A3A
:1076C0005A0AEEADFFAD3296FFAFEEAFEAACFBACBF
:1076D000B7CF05E010E0C8018752984FDC01AA0F30
:1076E000BB1FBFAFAEAF3801B3E06B0E711C25E01E
:1076F000209FC001219F900D11241BAE1AAEFC01EA
:10770000BD966696FFAFEEAF6697A7E04A2EADE056
:107710005A2EC301029705970CF0B6C166966EAD5E
:107720007FAD66978AAC9BAC680D791D072E000C67
:10773000880B990B0F9442B426966CAF7DAF8EAF39
:107740009FAF26977F926F92F9E5AF2EF6E0BF2E9E
:10775000BF92AF920F9447B37092F50E6092F40E01
:1077600020E030E040EF51E426966CAD7DAD8EAD6B
:107770009FAD26970F94A2B920E030E040E251E49B
:107780000F94A9AD20E030E040EA50E40F9491BAA4
:1077900020E030E048E452E40F94A3B90F9402BB18
:1077A00070930C0D60930B0D80E090E0A0EAB0E4C4
:1077B0008093541090935510A0935610B093571087
:1077C000209150103091511040915210509153100F
:1077D00060914C1070914D1080914E1090914F100F
:1077E0005F924F92812C912CA8E4AA2EA2E4BA2E8B
:1077F000B8E5CB2EB0E1DB2EE12CF12C00EA10E451
:107800000F94EF2C80E090E0A0EAB1E480934C105C
:1078100090934D10A0934E10B0934F10812C912C4B
:10782000F0E7AF2EF2E4BF2E8092501090925110EC
:10783000A0925210B0925310E0905410F090551056
:1078400000915610109157105F924F92812C912CFD
:1078500028E4A22E22E4B22E20E030E040E752E4F9
:10786000BC01CD010F94EF2C2AE939E949E15EE32F
:107870002093541030935510409356105093571046
:10788000209150103091511040915210509153104E
:1078900060914C1070914D1080914E1090914F104E
:1078A0005F924F921AE9E12E19E9F12E09E11EE3E8
:1078B0000F94EF2C0F9403890FB6F894DEBF0FBE20
:1078C000CDBF209188193091891940918A19509122
:1078D0008B1926966CAD7DAD8EAD9FAD26970F941E
:1078E000EEBB18163CF488EE93E00F94C1440E945E
:1078F000E193E7CF80E090E0A0EAB0E480935410F9
:1079000090935510A0935610B0935710209150109B
:1079100030915110409152105091531060914C1081
:1079200070914D1080914E1090914F105F924F9238
:10793000812C912CB8E4AB2EB2E4BB2E18E5C12EFD
:1079400010E1D12EE12CF12C00EA10E40F94EF2C81
:10795000E6E4FEE1659175918591949160934C10F8
:1079600070934D1080934E1090934F10EAE4FEE117
:107970002591359145915491209350103093511099
:107980004093521050935310E0905410F0905510C3
:1079900000915610109157105F924F920F94EF2C58
:1079A0000F94038960E070E080E89FEB0F947E16EF
:1079B000AAADBBAD1596BBAFAAAFBFEF6B1A7B0AE2
:1079C0000F900F900F900F90811103C00F9494A20D
:1079D0005BC027967FAD27972B966FAD2B972F9681
:1079E0009FAD2F9763968FAD6397272F362F492F23
:1079F000582F6091541070915510809156109091AD
:107A000057100F94A2B9162F072FF82EE92E2091A8
:107A10009C1030919D1040919E1050919F10D80164
:107A2000F7016B2F7A2F8F2F9E2F0F94A9AD0F94F4
:107A300002BB7A836983EF92FF920F931F93809129
:107A40008B198F9380918A198F93809189198F93C5
:107A5000809188198F93EDE2F6E0FF93EF930F94F6
:107A600047B3BE016F5F7F4F8EAD9FAD0E9491C542
:107A70002EAD3FAD2E5F3F4F3FAF2EAF0FB6F89408
:107A8000DEBF0FBECDBF45CE81E00F9494A20C9413
:107A9000146D0FEF10E0A5E2CA2EA6E0DA2E1093C7
:107AA000C1190093C019F4E6EF2EF12C84E690E0A2
:107AB0000F94C14451E0E51AF108C1F780912A10F2
:107AC0008F93809129108F931F930F93DF92CF9202
:107AD0000F9447B3055011090F900F900F900F901E
:107AE0000F900F90E1F60C94146D81E080937D0E61
:107AF0002091080D8091400F9091410F222341F079
:107B00002091090D222321F050900A0D51100FC031
:107B1000029749F081E0809383138EE090E10F9407
:107B2000317B0C94146D10927D0E0C94146D0297A1
:107B3000D1F38091640E9091650E28969FAF8EAF21
:107B40002897A091F40EB091F50E2C96BFAFAEAF72
:107B50002C9781E090E09093650E8093640E83E112
:107B600090E09093F50E8093F40E81E00F94BE0E9A
:107B70000F9459760E9414A580E090E0A0EAB0E44A
:107B80008093541090935510A0935610B0935710B3
:107B9000209150103091511040915210509153103B
:107BA00060914C1070914D1080914E1090914F103B
:107BB000E7E06E2EEDE07E2E7F926F92F5E58F2E40
:107BC000982CA82CF1E4BF2EA8E5CA2EA0E1DA2E4D
:107BD000E12CF12C00EA10E40F94EF2CE3EEFDE42D
:107BE000659175918591949160934C1070934D10AF
:107BF00080934E1090934F10E7EEFDE42591359160
:107C0000459154912093501030935110409352104D
:107C100050935310E0905410F0905510009156106E
:107C2000109157107F926F92812C912CE8ECAE2E20
:107C3000E2E4BE2E0F94EF2C0F9403890F900F9067
:107C40000F900F9005EC1FE0C8010F9424B9019626
:107C500039F00E5F1F4F053DEFE01E07A9F75AAE42
:107C600080E00F94535E60969FAF8EAF609783EE77
:107C7000482E8DE4582E612C712CC30163E070E016
:107C80000F9455BE24967FAF6EAF24971C0160FF02
:107C900006C002E0802E912C881A990A14019AAC31
:107CA0009920A1F16114710489F124968EAD9FADE4
:107CB0002497880F991F2496AEACBFAC24978A0DE9
:107CC0009B1D820D931D880F991F8D53904F0F940C
:107CD00024B9BC01990F880B990B0F9442B42AE088
:107CE00037ED43E25CE30F94A9AD20918315309109
:107CF000841540918515509186150F94A3B922964D
:107D00006CAF7DAF8EAF9FAF229706C022961CAEA0
:107D10001DAE1EAE1FAE229720E030E040EA50E4D8
:107D20002093541030935510409356105093571091
:107D30002091501030915110409152105091531099
:107D400060914C1070914D1080914E1090914F1099
:107D5000A7E0BDE0BF93AF93812C912CA0EAAA2E9F
:107D6000A1E4BA2EB8E5CB2EB0E1DB2EE12CF12C4C
:107D700000EA10E40F94EF2C0F940389F20185912F
:107D80009591A591B49180934C1090934D10A09330
:107D90004E10B0934F10F201349685919591A591B4
:107DA000B4918093501090935110A0935210B093BF
:107DB000531060E570E18CE490E10F94FF60E09077
:107DC0005410F090551000915610109157102091BA
:107DD00050103091511040915210509153106091B9
:107DE0004C1070914D1080914E1090914F10F7E013
:107DF0008F2EFDE09F2E9F928F92812C912CA6E1D9
:107E0000AA2EA3E4BA2E0F94EF2C0F9403890F909F
:107E10000F900F900F90BAACBB2081F061147104E9
:107E200069F020E030E040E85FE322966CAD7DAD84
:107E30008EAD9FAD22970F94A2B904C060E070E0B0
:107E400080E291EC0F947E16882309F48BC0C090D9
:107E50005410D0905510E0905610F0905710A70194
:107E6000960160E070E080EA90E40F94A2B92DECF6
:107E70003CEC4CEC5DE30F943CB487FD73C02AAD41
:107E80002223A1F0A701960122966CAD7DAD8EADA7
:107E90009FAD22970F94A2B99F7720E030E040E891
:107EA0005FE30F94EEBB18160CF45CC0C090881909
:107EB000D0908919E0908A19F0908B198091180759
:107EC0008823A9F00F942462882389F0C701B601A2
:107ED0000E94379420919C1030919D1040919E10EB
:107EE00050919F100F9491BA9B01AC0103C020E008
:107EF00030E0A901A7E024968EAD9FAD2497A89FFE
:107F00008001A99F100D1124020D131D000F111FD8
:107F1000000F111F0E571A4E60915410709155109A
:107F200080915610909157100F94A2B9F801618377
:107F30007283838394838091F40E9091F50E019760
:107F40009093F50E8093F40EFFEF6F1A7F0A81E095
:107F50000F94BE0E28E0420E511C39E063167104E6
:107F600009F08BCE80E090E0A0EAB0E4809354105A
:107F700090935510A0935610B09357102091501025
:107F800030915110409152105091531060914C100B
:107F900070914D1080914E1090914F10E7E0FDE0F0
:107FA000FF93EF93812C912C10EAA12E11E4B12EB6
:107FB00008E5C02E00E1D02EE12CF12C00EA10E4FF
:107FC0000F94EF2C0F9403890F900F9049E06416E3
:107FD000710409F4A3C085E090E00E948ED5B7E05B
:107FE0006B2EBDE07B2E170128018FE892E10E94E5
:107FF000FBFB8EE190E00F942FA20F948C5E5091CA
:108000001A0F5AAF10921A0F1092190F20E030E099
:1080100040E85FE3609154107091551080915610C4
:10802000909157100F94A2B97B018C01609354106A
:1080300070935510809356109093571020915010C4
:1080400030915110409152105091531060914C104A
:1080500070914D1080914E1090914F107F926F92C1
:10806000812C912CE0EAAE2EE1E4BE2EF8E5CF2E75
:10807000F0E1DF2E0F94EF2C0F94038961E0609301
:108080001A0F1092190F84E00E948FAF20925410A3
:108090003092551040925610509257102091501027
:1080A00030915110409152105091531060914C10EA
:1080B00070914D1080914E1090914F107F926F9261
:1080C000E12CF12C00EA10E40F94EF2C0F940389BB
:1080D0000E94F8AE8AAD80931A0F1092190F82E0B9
:1080E0000F94F0880F900F900F900F90A8019701B8
:1080F0000F94EEBB18160CF478CF1092650E109208
:10810000640E81E00F944E1641E061E081E00F942F
:10811000076F81E0809383130C94146D60968EAD8D
:108120009FAD60970F94325E0E94C1A46091050DCF
:108130007091060D072E000C880B990B0F9442B41A
:10814000905820919C1030919D1040919E1050911C
:108150009F100F9491BA0E94D2A480EC9FE00F94DC
:1081600017B9082FDE011196BBAFAAAF10E08090BF
:10817000890290908A02A0908B02B0908C02229685
:108180008CAE9DAEAEAEBFAE229766ED262E65E1FB
:10819000362E22968CAC9DACAEACBFAC22978982B9
:1081A0009A82AB82BC82AAADBBAD8D91BBAFAAAFA8
:1081B0000F94B7AC882329F00F94A5AC4B015C0158
:1081C0001BC0013009F02EC1123028F4112341F0F8
:1081D0008EEB9FE00AC0123031F08CEB9FE005C0BF
:1081E0008FEB9FE002C08DEB9FE00F9417B9882EB4
:1081F000880F9908AA08BB0881149104A104B1044E
:1082000009F410C1D501C401B7FE07C0882799271A
:10821000DC0188199909AA09BB0985369105A105D0
:10822000B1050CF432C0E7E9FDE584917F018823B4
:1082300041F00F94A14FFFEFEF1AFF0AF70184916D
:10824000F6CFEAEEFFE084917F01882341F00F949E
:10825000A14FFFEFEF1AFF0AF7018491F6CFC50196
:10826000B4010F949165E1EEFFE084917F018823D2
:1082700041F00F94A14FFFEFEF1AFF0AF70184912D
:10828000F6CF8AE00F94A14FCDC0C501B4010F9481
:1082900042B42FE632E143E85AE30F94A9AD6B01F3
:1082A0007C0120E030E040E05FE3123009F463C07D
:1082B000133009F48CC0113071F10F94A9AD2B016A
:1082C0003C0152E8A52E55E1B52EA3019201D5013E
:1082D00015966D917D918D919C9118970F94A3B9EE
:1082E000F5016583768387839087A7019601618175
:1082F0007281838194810F94A3B9D50111966D93F6
:108300007D938D939C931497BCE1AB0EB11C2A1402
:108310003B04D9F687C00F94A9AD2B013C0142E87C
:10832000A42E45E1B42EA3019201F5016581768169
:10833000878190850F94A3B9D50115966D937D9390
:108340008D939C931897A701960119966D917D9135
:108350008D919C911C970F94A3B9F5016187728749
:1083600083879487FCE1AF0EB11C26EDA21625E1B0
:10837000B206C9F657C00F94A9AD2B013C0133E8F2
:10838000A32E35E1B32EA3019201D5015C966D9128
:108390007D918D919C915F970F94A3B9F501648FA6
:1083A000758F868F978FA701960160817181828179
:1083B00093810F94A3B9D5016D937D938D939D9374
:1083C0005D01BFE8AB16B5E1BB06E9F62BC00F9423
:1083D000A9AD2B013C012FE9A22E25E1B22EA3016C
:1083E0009201F50160817181828193810F94A3B91B
:1083F000D5016D937D938D939D935D01A7019601AA
:1084000058966D917D918D919C915B970F94A3B936
:10841000F501608F718F828F938FFBEAAF16F5E1C4
:10842000BF06E9F61F5F143009F0B3CE0F947176E2
:1084300081E0809382150F94EC09E091070D24E010
:10844000E29FF0011124E55EF04F20E030E04FE2C2
:1084500053E460817181828193810F94EEBB181681
:1084600084F480911807882361F00F942462882394
:1084700041F080910B0D90910C0DC29714F00C946B
:108480006A6D81E090E090932602809325028EE150
:1084900094E10F94232628964EAD5FAD2897509314
:1084A000650E4093640E2C968EAD9FAD2C979093E5
:1084B000F50E8093F40E10927D0E34C180918215DA
:1084C000882309F495C0E7EDFFE084918F018823AC
:1084D00039F00F94A14F0F5F1F4FF8018491F7CF30
:1084E00067E070E080E090E00F949165E5EDFFE0DB
:1084F00084918F01882339F00F94A14F0F5F1F4F94
:10850000F8018491F7CF67E070E080E090E00F948D
:108510009165E2ECFFE084918F01882339F00F949C
:10852000A14F0F5F1F4FF8018491F7CF65E070E016
:1085300080E090E00F949165E0EBFFE084918F0183
:10854000882339F00F94A14F0F5F1F4FF8018491DA
:10855000F7CF8AE00F94A14F00E010E08DEA682E7B
:108560008FE0782E9BEAA92E9FE0B92EE12CF12C0A
:108570004801F8EA8F0E911CF3018491BDEACB2EDD
:10858000BFE0DB2E882341F00F94A14FFFEFCF1AFD
:10859000DF0AF6018491F6CFF401EE0DFF1DEE57D0
:1085A000FA4E618172818381948145E00F94265057
:1085B000F4E0EF0EF11C2CE1E216F104E9F6F5010E
:1085C0008491ABEAEA2EAFE0FA2E882341F00F94B3
:1085D000A14FFFEFEF1AFF0AF7018491F6CF0C517C
:1085E00011090C33FFEF1F0709F0C0CF0C94146D75
:1085F000EDE8FFE084918F01882311F40C94A56BC2
:108600000F94A14F0F5F1F4FF8018491F5CF86EEB5
:108610000F942E620C94146D10927A0F0C94146DBA
:1086200085E40F94B7AC811102C00F94038977E001
:10863000672E73E0772EECE4AE2EE0E1BE2EF8EE6E
:108640008F2EF0E19F2ED12CD3018D913D010F94FF
:10865000B7AC8823C9F1B3E0DB120CC00F94AFAC08
:10866000F501608371838283938388E590E10E94A2
:1086700040D62AC00F94AFAC9B01AC01D4016D91E0
:108680007D918D919C910F94A3B9F50160837183C5
:1086900082839383E0905410F0905510009156100F
:1086A000109157102091501030915110409152105C
:1086B0005091531060914C1070914D1080914E105C
:1086C00090914F100F94FB71D394F4E0AF0EB11C56
:1086D00024E0820E911C34E0D312B6CF0C94146DBA
:1086E00081E08093070F0F94D653609370167093B8
:1086F000711680937216909373166091070F84EC35
:108700009FE00F9429B962E377E081EC9FE00E943B
:1087100091C51092660E60E08FEF9FE00F9429B92B
:108720000C94146D82E00F94BE0E0C94146D809125
:1087300073159091741587579C4E9F938F9388E77C
:108740009FE00C9470348DE40F94B7AC882311F43F
:108750000C94616AE091600DF091610D3196819108
:108760008032E9F38930D9F380538A3060F0809108
:1087700073159091741587579C4E9F938F9383E642
:108780009FE00C9470340F94AFAC0F9402BBAB011C
:10879000BC01CA015093340D4093330D4937510544
:1087A00011F40C9486520CF0DEC04F32510509F4DE
:1087B00092C70CF061C04931510509F461C33CF521
:1087C0004431510509F4C3C294F44131510509F40F
:1087D000B4C234F44230510508F4FCC10C944A6A26
:1087E0004231510511F40C947B4F0C944A6A463186
:1087F000510509F4F0C20CF4EAC24731510509F4FD
:10880000F0C24831510509F404C30C944A6A4E3150
:10881000510509F46BC48CF44B31510509F44BC379
:108820000CF43BC34C31510509F434C44D315105AE
:1088300011F40C945C6A0C944A6A4A32510509F4AA
:108840001CC654F44F31510509F4BCC540325105E2
:1088500009F41DC50C944A6A4C32510509F42CC721
:108860004D32510511F00C944A6A8AE50F94B7AC69
:108870000E9415720C945C6A4936510511F40C94EF
:10888000454CA4F54435510511F40C947B4FDCF4B0
:108890004135510511F40C945D4F34F449345105C0
:1088A00009F461C70C944A6A4235510511F40C94DD
:1088B000774F4335510511F00C944A6A81E080935B
:1088C000380D0C945C6A4635510511F40C94DD4F5B
:1088D00014F40C94C24F4C35510511F40C94FC4F18
:1088E0004836510509F49CC70C944A6A4037510533
:1088F00009F4B5C7A4F44B36510511F40C94574F45
:1089000014F40C94274F4D36510511F40C94644D1A
:108910004E36510511F40C9480500C944A6A43373A
:10892000510511F40C94D05084F44137510511F4E1
:108930000C9493504237510511F00C944A6AE1ECC3
:10894000FCE084918F010C94A9514737510511F433
:108950000C948B524837510511F00C944A6A1092CE
:1089600024020C945C6A8E3541E0940711F40C9457
:1089700090690CF081C0803D910511F40C94FC5578
:10898000DCF58B3C910511F40C9459540CF58E3B9D
:10899000910511F40C94FE4D34F48C38910509F4D2
:1089A00063C70C944A6A883C910511F40C94A8534F
:1089B000893C910511F00C944A6A47E0C42E43E0CB
:1089C000D42E50E9E52E50E1F52E10E00C9414540D
:1089D0008D3C910511F40C94F75414F40C94B2549A
:1089E0008E3C910511F40C94A6558F3C910511F421
:1089F0000C94C5550C944A6A803F910511F40C946F
:108A00005C6ACCF48C3D910511F40C9479563CF4DD
:108A1000813D910511F40C9424560C944A6A8D3DC5
:108A2000910511F40C94A456823E910511F40C9416
:108A3000C5560C944A6A8E3261E0960711F40C9484
:108A4000B2586CF48C32B1E09B0711F40C942857A7
:108A50008D32914011F40C945E570C944A6A8F3217
:108A6000F1E09F0711F40C94C7588033914011F442
:108A70000C941A580C944A6A8A3532E0930711F420
:108A80000C941D650CF049C0853F51E0950711F429
:108A90000C94DE5CECF48039A1E09A0711F40C949C
:108AA000965C3CF48F35914011F40C945C6A0C9404
:108AB0004A6A8339F1E09F0711F40C949A5C843F71
:108AC000914011F00C944A6A0F9494520C945C6A91
:108AD0008D3F31E0930711F40C949E5F6CF4863F58
:108AE00051E0950711F40C94E25C873F914011F43A
:108AF0000C94E65C0C944A6A8835A2E09A0711F45B
:108B00000C9479608935924011F00C944A6A0E9465
:108B1000ECEA0F949E8D0C945C6A8D35E3E09E0721
:108B200011F40C94F165DCF48E3B22E0920711F411
:108B30000C94396A3CF48D3B924011F40C942D6AEC
:108B40000C944A6A833553E0950711F40C94BA5F8C
:108B50008C35934011F40C9420650C944A6A8C383F
:108B6000A3E09A0711F40C945C6A94F48438E3E06F
:108B70009E0711F40C940D688B38934011F00C94FF
:108B80004A6A17E0A12E13E0B12E00E00C94706940
:108B9000803A23E0920709F4E6C3873E934011F040
:108BA0000C944A6A1092B30F1092340F8091830F85
:108BB0009091840FA091850FB091860F8093620DE4
:108BC0009093630DA093640DB093650D0F94E344EF
:108BD0000C945C6AE091600DF091610D8F010E5F65
:108BE0001F4F80E50F94B7AC882371F00F94AFACA2
:108BF0000F9408BB6B017C01AA24A394672B682BFC
:108C0000692B31F4A12C04C0A12CC12CD12C7601EC
:108C100083E50F94B7AC882391F00F94AFAC20E0BC
:108C200030E04AE754E40F94A9AD0F9408BB6B0100
:108C30007C01BB24B394672B682B692B09F4B12CFE
:108C40006AE270E0C8010F94EBBE009711F0DC01FE
:108C50001C92F801CF0121912032E1F3A11007C04D
:108C6000B11005C0222319F00F949C2704C08EE791
:108C700092E10F94232681E080936B0E10926A0E8E
:108C80000F9403890F94D65360937F0F7093800FD6
:108C90008093810F9093820FC114D104E104F104F9
:108CA00019F10F94D653C60ED71EE81EF91E84E0A4
:108CB00090E090932602809325020F94D6536C1572
:108CC0007D058E059F0510F00C94AC6D0F948F0FF1
:108CD00081110C94AC6D0F94378281E00F94614048
:108CE00080E00F94BE0EE9CF84E090E090932602DE
:108CF000809325020F948F0F811109C00F94378242
:108D000081E00F94614080E00F94BE0EF3CF82E0CB
:108D100090E0909326028093250280917616882316
:108D200031F088EF91E40F9423260C945C6A8EE175
:108D300094E10F9423260C945C6A85E792E10F94EA
:108D4000232617981698159814980C945C6AE5E1F8
:108D5000F6E084918F01882339F00F94A14F0F5FC3
:108D60001F4FF8018491F7CF8AE00F94A14F109222
:108D70005719109256198AEC96E10E9433EF8BE155
:108D8000EAECF6E1DE01119601900D928A95E1F789
:108D900040E050E0BE016F5F7F4F86E094E00F94AB
:108DA000F87FCE0101960F945160E7E0F6E08491E0
:108DB0008F01882339F00F94A14F0F5F1F4FF801E7
:108DC0008491F7CF8AE00F94A14F0C945C6A0F94C2
:108DD000991C0C945C6A10927616109277160C947B
:108DE0005C6A8091600D9091610D6AE270E004967A
:108DF0000F94EBBE009711F0DC011C928091600D86
:108E00009091610D41E061E004960F94C6170C94B7
:108E10005C6A8091781681111EC060E086E69FE052
:108E20000F9429B960E088E69FE00F9429B960E0CB
:108E300085E69FE00F9429B960E084E69FE00F94F7
:108E400029B960E082ED9EE00F9429B960E08FECD3
:108E50009EE00F9429B980917716882329F081E04C
:108E600080937616109278160F94D6536093740EF2
:108E70007093750E8093760E9093770E0C945C6AC7
:108E800080917616882311F40C945C6A1092761601
:108E900081E0809378160C945C6A80917716882321
:108EA00011F40C945C6A83E50F94B7AC81110C94B7
:108EB000B86D0C945C6A80917616882309F4B8C06A
:108EC00002E916E1F80181918F01882319F00F94CE
:108ED000A14FF8CFEEE3FDE084918F01882339F0B4
:108EE0000F94A14F0F5F1F4FF8018491F7CFE9EE68
:108EF000F4E084918F01882339F00F94A14F0F5F24
:108F00001F4FF8018491F7CF609151197091521958
:108F100080915319909154194AE00F94B54FECE3A6
:108F2000FDE084918F01882339F00F94A14F0F5FEA
:108F30001F4FF8018491F7CF6091491970914A1938
:108F400080914B1990914C194AE00F94B54F8AE0EB
:108F50000F94A14F0F94D65350E6C52E5AEED52E3E
:108F6000E12CF12CA70196010F9467B949015A0130
:108F70006091740E7091750E8091760E9091770EBF
:108F8000A70196010F9467B98401021B130BC80156
:108F90006CE370E00F9441BECB019927EAE0F0E06A
:108FA000BF010F9455BE282FCB01BF010F9455BEB2
:108FB000805D8093B819205D2093B9191092BA1979
:108FC00068EBE62E69E1F62E6701D6018D916D0101
:108FD000882319F00F94A14FF8CF8AE30F94A14F83
:108FE000C8016CE370E00F9441BE6AE070E00F943A
:108FF00055BE605D6093B819805D8093B919109279
:10900000BA19F70181917F01882319F00F94A14FBC
:10901000F8CFEAE3FDE084918F01882311F40C94EA
:109020005C6A0F94A14F0F5F1F4FF8018491F5CF39
:1090300080917816882371F0EAE2FDE084918F0137
:10904000882309F4BFCE0F94A14F0F5F1F4FF80183
:109050008491F6CF80917F0E882371F0EEE1FDE0E0
:1090600084918F01882309F4ADCE0F94A14F0F5F37
:109070001F4FF8018491F6CFEEE0FDE084918F015F
:10908000882309F49FCE0F94A14F0F5F1F4FF80163
:109090008491F6CF8091600D9091610D6AE270E04D
:1090A00004960F94EBBE8C01892BA9F08091731567
:1090B000909174156EE470E087579C4E0F94EBBE50
:1090C00060E270E00F94EBBE01969093610D809387
:1090D000600DD8011C928091600D9091610D41E06E
:1090E00060E004960F94C6170C945C6A8091771622
:1090F000882311F40C945C6A0F94786F8091600D52
:109100009091610D6AE270E004960F94EBBE8C01C1
:10911000892BA9F080917315909174156EE470E01D
:1091200087579C4E0F94EBBE60E270E00F94EBBE4D
:1091300001969093610D8093600DF8011082C090AC
:10914000600DD090610D86010C5F1F4F80917716E6
:10915000882311F40C945C6A8CE998E10E9459F21E
:10916000109276161F8E1AA28AEC96E19093E6165C
:109170008093E5160115110591F0D60114968C9196
:109180008F3239F4BE01615E7F4FC8010F946C715C
:1091900006C087EE96E19093E6168093E5166091FF
:1091A000E5167091E61619821C8222E0A801CE0114
:1091B00001960E9420F48823A1F0CE0101960F941D
:1091C000667F882371F061E0CE0101960E94DAF19A
:1091D000009739F025EEFC0120831C820E945EEC92
:1091E000F82ECE0101960F945160FF2021F1E0E0AE
:1091F000FDE084917F01882341F00F94A14FFFEFA0
:10920000EF1AFF0AF7018491F6CFD8018D918D01F5
:10921000882319F00F94A14FF8CF8AE00F94A14F43
:109220001092511910925219109253191092541908
:109230000F94891A26C0E8EEFCE084917F01882310
:1092400041F00F94A14FBFEFEB1AFB0AF701849195
:10925000F6CFD8018D918D01882319F00F94A14F7D
:10926000F8CFE6EEFCE084918F01882339F00F946B
:10927000A14F0F5F1F4FF8018491F7CF8AE00F9441
:10928000A14FCE014F960F9451600C945C6A80916F
:10929000761681110F9403890091600D1091610D74
:1092A0000C5F1F4F6AE270E0C8010F94EBBE7C01B7
:1092B00061E270E0C8010F94EBBE009719F08C01D9
:1092C0000F5F1F4FE114F10411F0D7011C9280E5EC
:1092D0000F94B7ACF82E8091600D9091610D081736
:1092E000190708F4F12C80917716882311F40C9457
:1092F0005C6A41E04F2561E0C8010F94C61783E521
:109300000F94B7AC8823B9F08091600D9091610DF6
:109310008017910780F40F94A5ACAB01BC0140937A
:1093200051195093521960935319709354198CE941
:1093300098E10E949DEE80917716882329F081E0C4
:109340008093761610927816F1100C945C6A0F9444
:10935000D6536093740E7093750E8093760E90932F
:10936000770E0C945C6A8091600D9091610D6AE2B9
:1093700070E005960F94EBBE8C01892BA9F08091CB
:109380007315909174156EE470E087579C4E0F949E
:10939000EBBE60E270E00F94EBBE01969093610D1E
:1093A0008093600DF80110828091600D9091610DA5
:1093B00021E02093751641E060E005960F94C617F2
:1093C0000C945C6A0F94D6530091740E1091750E34
:1093D0002091760E3091770E6B017C01C01AD10A74
:1093E000E20AF30AC701B60128EE33E040E050E09C
:1093F0000F9467B9CA01B9012CE330E040E050E0B6
:109400000F9467B97F936F93C701B60120E63AEED8
:1094100040E050E00F9467B93F932F9384E59FE0BD
:109420009F938F938E010F5F1F4F1F930F930F9486
:10943000A0B3E9EBFDE584910FB6F894DEBF0FBE53
:10944000CDBF7F01882341F00F94A14F3FEFE31A76
:10945000F30AF7018491F6CF7801D7018D917D0150
:10946000882319F00F94A14FF8CF8AE00F94A14FF1
:10947000C8010F949C270C945C6A83E50F94B7ACE9
:10948000882311F40C945C6A0F94AFAC0F9402BB68
:109490004B015C017B0180E50F94B7AC882339F068
:1094A000BFEF8B16910409F010F40C94C96D0DE018
:1094B00010E0EDE8F2E0819191918017910711F4AD
:1094C0000C945C6A22E0E53CF207A9F7063011052E
:1094D00029F49092C1198092C01904C017FF02C0EC
:1094E0000C945C6AD02E61E0802F0F94D621682DF9
:1094F000802F0F94A82161E0802F0F94D621E114D2
:10950000F10431F460E0802F0F94A8210C945C6A80
:109510003FEFE316F10431F461E0802F0F94A821AE
:109520000C945C6AF801FF27E25AFC4AE4918E2F02
:1095300090E0FC013197E231F10508F0ADC08827D9
:10954000EE58FF4F8F4F0D9484BE84B5806884BD64
:1095500087BC0C945C6A84B5806284BD88BC0C9422
:109560005C6A80918000806880938000909289007E
:10957000809288000C945C6A809180008062809365
:10958000800090928B0080928A000C945C6A80919B
:10959000800088608093800090928D0080928C0083
:1095A0000C945C6A8091B00080688093B0008092D7
:1095B000B3000C945C6A8091B00080628093B0002C
:1095C0008092B4000C945C6A8091900080688093D3
:1095D000900090929900809298000C945C6A80911F
:1095E000900080628093900090929B0080929A00FD
:1095F0000C945C6A809190008860809390009092B7
:109600009D0080929C000C945C6A8091A000806810
:109610008093A0008091A0008F7B8093A000909207
:10962000A9008092A8000C945C6A8091A0008062DE
:109630008093A0009092AB008092AA000C945C6A88
:109640008091A00088608093A0009092AD008092ED
:10965000AC000C945C6A80912001806880932001AA
:1096600090922901809228010C945C6A80912001DB
:1096700080628093200190922B0180922A010C94A9
:109680005C6A8091200188608093200190922D0176
:1096900080922C010C945C6A40E8E416F10434F4E6
:1096A00060E08D2D0F94A8210C945C6A61E08D2DF3
:1096B0000F94A8210C945C6A8FEF0F942E6260E0E7
:1096C00070E088EF9FE00F9443B90F94440C0F941F
:1096D000260C0C945C6A84E090E0909326028093C0
:1096E00025020F9444160E9436B20F94378281E00F
:1096F0000F94614060E080E00F94971187ED9CE04B
:109700000F94BE1061E080E00F9497111E9903C082
:1097100081ED9CE002C084ED9CE00F94BE1062E0FD
:1097200080E00F9497111D9903C08BEC9CE002C060
:109730008EEC9CE00F94BE1063E080E00F949711D4
:109740001C9903C085EC9CE002C088EC9CE00F945F
:10975000BE100F948F0F882341F20F9444160F947C
:10976000A08C0C945C6A80E50F94B7AC882331F030
:109770000F94AFAC0F9408BB6093390282E50F944D
:10978000B7AC882341F00F94AFAC0F9408BB709333
:109790003F0260933E0281E50F94B7AC882331F01D
:1097A0000F94AFAC0F9408BB6093380283E50F941D
:1097B000B7AC882341F00F94AFAC0F9408BB709303
:1097C0003D0260933C0280913F028F9380913E0264
:1097D0008F93809139021F928F9383EC95E09F9332
:1097E0008F930AEC15E01F930F930F9447B380916A
:1097F0003D028F9380913C028F93809138021F929B
:109800008F938CEB95E09F938F931F930F930F94FF
:1098100047B30FB6F894DEBF0FBECDBF0C945C6AA1
:10982000BE016F5F7F4F88E690E00F94D2AA81114E
:109830000C945C6A83E50F94B7AC882311F40C9404
:109840005C6A19810F94AFAC11110C945C6A0F948F
:1098500002BB70937615609375150C945C6A63E097
:109860008BEB95E00F94024083E50F94B7AC88230F
:1098700011F40C945C6A0F94AFAC0F9402BB70931C
:109880000C0D60930B0D0C945C6ABE016F5F7F4FF3
:1098900089E690E00F94D2AA81110C945C6AEEE400
:1098A000FFE084918F01882339F00F94A14F0F5F5F
:1098B0001F4FF8018491F7CFE98124E0E29FF00186
:1098C0001124E55EF04F608171818281938141E0D6
:1098D0000F942650EBE4FFE084918F01882339F048
:1098E0000F94A14F0F5F1F4FF8018491F7CFE981CB
:1098F000F0E0EE0FFF1FEB58FA4E60817181072EEA
:10990000000C880B990B0F9442B441E00F94265041
:10991000E7E4FFE084918F01882339F00F94A14F91
:109920000F5F1F4FF8018491F7CF6091110770917D
:109930001207809113079091140741E00F9426506D
:10994000E4E4FFE084918F01882339F00F94A14F64
:109950000F5F1F4FF8018491F7CF60910B0D70914D
:109960000C0D072E000C880B990B0F9442B441E0AC
:109970000F942650E1E4FFE084918F01882339F0B1
:109980000F94A14F0F5F1F4FF8018491F7CF60E054
:1099900070E0CB010F949165EFE3FFE084918F01BC
:1099A000882339F00F94A14F0F5F1F4FF801849166
:1099B000F7CF60911B0F70911C0F80911D0F90913C
:1099C0001E0F41E00F942650ECE3FFE084918F01DD
:1099D000882339F00F94A14F0F5F1F4FF801849136
:1099E000F7CF6091751570917615072E000C880BD6
:1099F000990B0F9442B441E00F942650E8E3FFE046
:109A000084918F01882339F00F94A14F0F5F1F4F6E
:109A1000F8018491F7CFE981F0E0EF54F04F6081D5
:109A200070E080E090E00F949165E3E3FFE08491C3
:109A30008F01882339F00F94A14F0F5F1F4FF8015A
:109A40008491F7CF6091B00F70E080E090E00F94C8
:109A50009165EFE2FFE084918F01882339F00F9444
:109A6000A14F0F5F1F4FF8018491F7CF60918819C4
:109A70007091891980918A1990918B1941E00F9406
:109A80002650EBE2FFE084918F01882339F00F9498
:109A9000A14F0F5F1F4FF8018491F7CF6091841998
:109AA00070918519809186199091871941E00F94E2
:109AB00026508AE00F94A14F81E090E09093260217
:109AC000809325020C94FB71BE016F5F7F4F8DE682
:109AD00090E00F94D2AA81110C945C6A8DE398E215
:109AE0000F94232681E090E09093510D8093500DC8
:109AF0008091070F882329F060E081E090E00E94C8
:109B000026F783E50F94B7AC882379F019810F9479
:109B1000AFAC111106C00F9402BB70937615609321
:109B2000751581E08093060212C082E50F94B7ACF0
:109B3000882369F019810F94AFAC111106C00F94FE
:109B400002BB7093761560937515109206020F9400
:109B5000D6534B015C01F9800F2D10E0F801EE0F98
:109B6000FF1FEB58FA4E60817181072E000C880BA5
:109B7000990B0F9442B4F801EE0FFF1FEE0FFF1F79
:109B8000E55EF04F11E020813181428153810F94D5
:109B9000EEBB18160CF010E01093870F81E090E0F8
:109BA000909326028093250210927E0E4F2DC501C0
:109BB000B4010F946F438FE298E20F94232682E062
:109BC00090E090932602809325029093510D80930C
:109BD000500D8091070F882329F060E082E090E02B
:109BE0000E9426F70F94D65360937F0F7093800FD7
:109BF0008093810F9093820F0C945C6A83E298E2C9
:109C00000F94232683E090E09093510D8093500DA4
:109C10008091070F882329F060E081E090E00E94A6
:109C200026F783E50F94B7AC882361F00F94AFACAF
:109C30000F9402BB70930C0D60930B0D81E0809329
:109C400006020FC082E50F94B7AC882351F00F9441
:109C5000AFAC0F9402BB70930C0D60930B0D109280
:109C600006020F94D6534B015C0110927E0E609158
:109C70000B0D70910C0D072E000C880B990B0F9497
:109C800042B411E02091110730911207409113075F
:109C9000509114070F94EEBB18160CF010E01093BF
:109CA000870F81E090E0909326028093250208E2DE
:109CB0001FE084E2E82E8FE0F82E90E2C92E9FE0AC
:109CC000D92E8091870F60910B0D70910C0D882318
:109CD000B9F080917E0E811113C0072E000C880B05
:109CE000990B0F9442B420911107309112074091C3
:109CF0001307509114070F94EEBB1816BCF08BC0DD
:109D0000072E000C880B990B0F9442B42091110779
:109D10003091120740911307509114070F943CB4EF
:109D200087FF79C080910602811175C00F94D653C8
:109D3000DC01CB0188199909AA09BB09893E934026
:109D4000A105B10508F45EC08091070F811156C0CE
:109D5000E091070D24E0E29FF0011124E55EF04F51
:109D60004080518062807380F8018491B8E2AB2E0C
:109D7000BFE0BB2E882341F00F94A14FFFEFAF1A35
:109D8000BF0AF5018491F6CF42E0C301B2010F94FE
:109D90002650F7018491A4E2AA2EAFE0BA2E8823C0
:109DA00041F00F94A14FFFEFAF1ABF0AF501849164
:109DB000F6CF6091070D70E080E090E00F94916520
:109DC000F6018491F0E2AF2EFFE0BF2E882341F030
:109DD0000F94A14FFFEFAF1ABF0AF5018491F6CFA0
:109DE00060911107709112078091130790911407E9
:109DF00041E00F9426508AE00F94A14F0F94D65360
:109E00004B015C010F94378280E00F94614080E049
:109E10000F94BE0E56CF8AE198E20F94232682E07B
:109E200090E0909326028093250284E090E0909346
:109E3000510D8093500D0F94D65360937F0F709304
:109E4000800F8093810F9093820F0C945C6A83E55E
:109E50000F94B7AC882319F10F94AFAC20E030E039
:109E6000A9010F943CB487FD0FC00F94AFAC20E064
:109E700030E04FE753E40F94EEBB181644F00F9414
:109E8000AFAC0F9402BB05C060E070E002C06FEFA2
:109E900070E07093C1196093C0190C945C6A8FEFE5
:109EA00090E09093C1198093C0190C945C6A109251
:109EB000C1191092C0190C945C6A0F945D490F94FB
:109EC0000389149A0F9416891092C1191092C0191F
:109ED00068EE73E080E090E00F949E5387E094E09A
:109EE0000F94232680E00F94BE0E0C945C6A1092AF
:109EF000380D0C945C6A83E50F94B7AC882399F015
:109F00000F94AFAC20E030E04AE754E40F94A9ADE1
:109F10000F9408BB60938102709382028093830246
:109F2000909384021DC088E50F94B7AC81110C9406
:109F3000D06D89E50F94B7AC81110C94D06D8AE592
:109F40000F94B7AC81110C94D06D85E40F94B7AC2D
:109F500081110C94D06D0F940389149A0F94168973
:109F60008FEF9FEF90933F0280933E0290933D02CC
:109F700080933C0280933902809338021092390D0D
:109F80000C945C6A83E50F94B7AC882311F40C94AD
:109F90005C6A0F94AFAC20E030E04AE754E40F94E1
:109FA000A9AD0F9408BB60937B0F70937C0F8093D7
:109FB0007D0F90937E0F0C945C6A83E50F94B7AC91
:109FC000882311F40C945C6A0F94AFAC20E030E06D
:109FD0004AE754E40F94A9AD0F9408BB60937D0247
:109FE00070937E0280937F02909380028FE596E1CA
:109FF0000E94CDEB0C945C6A27E033E03BAF2AAFC4
:10A0000000E910E1E5E9CE2EEDE0DE2EF12CAAAD5F
:10A01000BBAD8D91BBAFAAAF0F94B7AC882309F449
:10A0200063C0B3E0FB1259C00F94AFAC2B013C01ED
:10A0300020E030E040EA51E40F943CB487FF45C093
:10A04000A3019201F80164817581868197810F9443
:10A0500091BA4B015C019B01AC016091E4107091DD
:10A06000E5108091E6109091E7100F94A9AD6093F0
:10A07000E4107093E5108093E6109093E710209021
:10A080004C0230904D02A5019401D1011C966D91B6
:10A090007D918D919C911F970F94A9ADF1016487DB
:10A0A000758786879787D6016D917D918D919C915B
:10A0B0000F9440B4A50194010F94A9AD0F9408BB6F
:10A0C000F6016083718382839383D80114964D9245
:10A0D0005D926D927C92179707C00F94AFACF80118
:10A0E0006483758386839783F3940C5F1F4FF4E03A
:10A0F000CF0ED11C74E0872EF81089CF0C945C6AC7
:10A100008EE40F94B7AC882311F40C945C6A0F941E
:10A11000A5AC6093620D7093630D8093640D909372
:10A12000650D0C945C6A83E50F94B7AC882379F0D5
:10A130008091600D9091610D4AE050E060E070E028
:10A1400001960F94D1AF60932F020C945C6AE9EBF7
:10A15000FDE584918F01882339F00F94A14F0F5FA3
:10A160001F4FF8018491F7CFC0902F02D12CE12C22
:10A17000F12CE9E1FFE084918F01882339F00F94FD
:10A18000A14F0F5F1F4FF8018491F7CF4AE0C7013D
:10A19000B6010F94B54F8AE00F94A14F0C945C6AFE
:10A1A00086E50F94B7AC882379F0EDECFCE584915B
:10A1B0008F01882311F40C94E2460F94A14F0F5F96
:10A1C0001F4FF8018491F5CF85E50F94B7AC382E79
:10A1D0008823D9F1E090600DF090610DFFEFEF1A48
:10A1E000FF0AF092610DE092600D270167014601C0
:10A1F000D6018D916D0190ED980F9A30C0F38E329B
:10A2000011F00C945C6A5D013501F50181915F01EB
:10A2100090ED980F9A30C0F38E3211F00C945C6A76
:10A22000CF018C01DC012C90019620ED220D2A300B
:10A23000C0F3822D0F94F92581110C94EF6DBDE2CE
:10A240002B120C945C6A0C94EF6DEBEFFEE08491A2
:10A250008F01882339F00F94A14F0F5F1F4FF80132
:10A260008491F7CFEDECFCE584918F01882339F0E0
:10A270000F94A14F0F5F1F4FF8018491F7CFE1EAD0
:10A28000FEE084918F01882339F00F94A14F0F5F76
:10A290001F4FF8018491F7CFEDE9FEE084918F0123
:10A2A000882339F00F94A14F0F5F1F4FF80184915D
:10A2B000F7CFEEE8FEE084918F01882339F00F9408
:10A2C000A14F0F5F1F4FF8018491F7CFE1E8FEE047
:10A2D00084918F01882339F00F94A14F0F5F1F4F96
:10A2E000F8018491F7CFE0E7FEE084918F018823A5
:10A2F00039F00F94A14F0F5F1F4FF8018491F7CFF2
:10A30000EEE6FEE084918F01882339F00F94A14F8F
:10A310000F5F1F4FF8018491F7CFE7E6FEE08491CD
:10A320008F01882339F00F94A14F0F5F1F4FF80161
:10A330008491F7CFE2E4FEE084918F01882311F449
:10A340000C94E2460F94A14F0F5F1F4FF8018491C8
:10A35000F5CF882339F00F94A14F0F5F1F4FF801FD
:10A360008491F7CF60914C1070914D1080914E10F8
:10A3700090914F1042E00F942650EDEBFCE0849159
:10A380008F01882339F00F94A14F0F5F1F4FF80101
:10A390008491F7CF609150107091511080915210BC
:10A3A0009091531042E00F942650E9EBFCE0849129
:10A3B0008F01882339F00F94A14F0F5F1F4FF801D1
:10A3C0008491F7CF60915410709155108091561080
:10A3D0009091571042E00F942650E5EBFCE08491F9
:10A3E0008F01882339F00F94A14F0F5F1F4FF801A1
:10A3F0008491F7CF609158107091591080915A1044
:10A4000090915B1042E00F942650EEEDF4E08491C1
:10A410008F01882339F00F94A14F0F5F1F4FF80170
:10A420008491F7CF80E00F94E2880F9442B420919A
:10A4300094103091951040919610509197100F9470
:10A4400091BA42E00F942650E1EBFCE084918F0139
:10A45000882339F00F94A14F0F5F1F4FF8018491AB
:10A46000F7CF81E00F94E2880F9442B420919810C6
:10A470003091991040919A1050919B100F9491BA7D
:10A4800042E00F942650EDEAFCE084918F0188238E
:10A4900039F00F94A14F0F5F1F4FF8018491F7CF50
:10A4A00082E00F94E2880F9442B420919C10309186
:10A4B0009D1040919E1050919F100F9491BA42E0D0
:10A4C0000F942650E9EAFCE084918F01882339F04B
:10A4D0000F94A14F0F5F1F4FF8018491F7CF83E0D6
:10A4E0000F94E2880F9442B42091A0103091A110F3
:10A4F0004091A2105091A3100F9491BA42E00F9492
:10A5000026508AE00F94A14F0C945C6A81E08093FE
:10A5100024020C945C6AE2EAF5E084918F018823BE
:10A5200039F00F94A14F0F5F1F4FF8018491F7CFBF
:10A530008AE00F94A14FEAE9F5E084918F01882326
:10A5400039F00F94A14F0F5F1F4FF8018491F7CF9F
:10A550001E9B0DC0E0E9F5E084918F018823A1F0F6
:10A560000F94A14F0F5F1F4FF8018491F7CFEBE8D5
:10A57000F5E084918F01882339F00F94A14F0F5F8C
:10A580001F4FF8018491F7CF8AE00F94A14FE3E8C1
:10A59000F5E084918F01882339F00F94A14F0F5F6C
:10A5A0001F4FF8018491F7CF8091060182FF0DC003
:10A5B000E0E9F5E084918F018823A1F00F94A14F89
:10A5C0000F5F1F4FF8018491F7CFEBE8F5E084911E
:10A5D0008F01882339F00F94A14F0F5F1F4FF801AF
:10A5E0008491F7CF8AE00F94A14FEBE7F5E08491D7
:10A5F0008F01882339F00F94A14F0F5F1F4FF8018F
:10A600008491F7CF1D9B0DC0E0E9F5E084918F01A7
:10A610008823A1F00F94A14F0F5F1F4FF801849181
:10A62000F7CFEBE8F5E084918F01882339F00F94A0
:10A63000A14F0F5F1F4FF8018491F7CF8AE00F946D
:10A64000A14FE3E7F5E084918F01882339F00F945F
:10A65000A14F0F5F1F4FF8018491F7CF8091060142
:10A6600087FF0DC0E0E9F5E084918F018823A1F018
:10A670000F94A14F0F5F1F4FF8018491F7CFEBE8C4
:10A68000F5E084918F01882339F00F94A14F0F5F7B
:10A690001F4FF8018491F7CF8AE00F94A14FEBE6AA
:10A6A000F5E084918F01882339F00F94A14F0F5F5B
:10A6B0001F4FF8018491F7CF1C9B0DC0E0E9F5E036
:10A6C00084918F018823A1F00F94A14F0F5F1F4F3A
:10A6D000F8018491F7CFEBE8F5E084918F018823AE
:10A6E00039F00F94A14F0F5F1F4FF8018491F7CFFE
:10A6F0008AE00F94A14FE3E6F5E084918F0188236F
:10A7000039F00F94A14F0F5F1F4FF8018491F7CFDD
:10A7100001990FC0E0E9F5E084918F01882311F4DD
:10A720000C94E2460F94A14F0F5F1F4FF8018491E4
:10A73000F5CFEBE8F5E084918F01882311F40C94B8
:10A74000E2460F94A14F0F5F1F4FF8018491F5CFA0
:10A750001091070D84E50F94B7AC882301F10F9495
:10A76000AFAC0F9408BB162F6623C9F0E9EBFDE5EB
:10A7700084918F01882339F00F94A14F0F5F1F4FF1
:10A78000F8018491F7CF0CE415E0D8018D918D018B
:10A79000882311F40C945C6A0F94A14FF6CF84E4E3
:10A7A0000F94B7AC882311F40C945C6A0F94AFAC8F
:10A7B00020E030E0A9010F943CB4811103C0109255
:10A7C00027112EC00F94AFACB4E01B9FF0011124F1
:10A7D000E85DFE4E6083718382839383C09028116D
:10A7E000D0902911E0902A11F0902B1120E030E058
:10A7F000A901C701B6010F943CB4811106C0C12C58
:10A80000D12C60EEE62E6FE3F62EC0922811D09286
:10A810002911E0922A11F0922B1181E080932711E7
:10A820000F94D03E0C945C6AF60181916F010F94F5
:10A83000B7AC882399F10F94AFAC0F9408BB1230DA
:10A84000ACF4653CF9E07F0781059105A0F4562F33
:10A85000472F382F292F613CA3E07A078105910506
:10A8600090F050EC43E030E020E00DC0562F472F31
:10A87000382F292F08C050EC43E030E020E064EC92
:10A8800079E080E090E0F70164A375A386A397A325
:10A89000E455FF4F50834183328323831F5FF4E0ED
:10A8A000EF0EF11C143009F0BFCF0E94E2D50C94DA
:10A8B0005C6A27E0A22E23E0B22E30E9C32E30E1FD
:10A8C000D32E912CD5018D915D010F94B7AC8823C7
:10A8D00009F43EC00F94AFAC7B018C01B1E0B91517
:10A8E00014F120E030E048E453E40F94EEBB181676
:10A8F0003CF4512C612C88E4782E93E4892E04C01A
:10A900005E2C6F2C702E812E20E030E048EC52E45B
:10A91000B701C8010F94EEBB18164CF4E12CF12CD2
:10A9200008EC12E404C0562E6F2C782E812E852D53
:10A93000962DA72DB82DF601848B958BA68BB78B02
:10A94000C701D801E456FF4F80839183A283B3836C
:10A950009394F4E0CF0ED11C14E0812E9810B2CF66
:10A960000C945C6A83E50F94B7AC8823E9F00F94EC
:10A97000AFAC6093C4107093C5108093C6109093D1
:10A98000C71084E50F94B7AC882311F40C945C6A6B
:10A990000F94AFAC6093C8107093C9108093CA1025
:10A9A0009093CB100C945C6A80E50F94B7AC88232D
:10A9B00051F00F94AFAC6093C4107093C5108093A6
:10A9C000C6109093C71082E50F94B7AC882351F05E
:10A9D0000F94AFAC6093C8107093C9108093CA10E5
:10A9E0009093CB1084E50F94B7AC0C945C6A83E52C
:10A9F0000F94B7AC882351F00F94AFAC6093CC1098
:10AA00007093CD108093CE109093CF1084E50F9467
:10AA1000B7AC882351F00F94AFAC6093D010709313
:10AA2000D1108093D2109093D31082E40F94B7ACDE
:10AA3000882361F00F94AFAC0F9408BB6093D410DF
:10AA40007093D5108093D6109093D71088E50F940B
:10AA5000B7AC882391F00F94AFAC6093DC10709387
:10AA6000DD108093DE109093DF106093D810709308
:10AA7000D9108093DA109093DB1089E50F94B7AC6E
:10AA8000882351F00F94AFAC6093DC107093DD100D
:10AA90008093DE109093DF108AE50F94B7AC882383
:10AAA00051F00F94AFAC6093E0107093E11080937D
:10AAB000E2109093E31085E40F94B7AC882351F033
:10AAC0000F94AFAC6093E4107093E5108093E610A0
:10AAD0009093E71020E030E040E251E46091D8101C
:10AAE0007091D9108091DA109091DB100F94EEBB29
:10AAF000181664F480E090E0A0E2B1E48093D810EE
:10AB00009093D910A093DA10B093DB1020E030E0DE
:10AB100040E251E46091DC107091DD108091DE1014
:10AB20009091DF100F94EEBB181614F00C945C6A31
:10AB300080E090E0A0E2B1E48093DC109093DD101F
:10AB4000A093DE10B093DF100C945C6AA7E0EA2EAD
:10AB5000A3E0FA2E08EE10E1B4EFCB2EB0E1DB2E2D
:10AB6000D7018D917D010F94B7AC882339F00F94F4
:10AB7000AFACF80160837183828393830C5F1F4FB6
:10AB8000C016D10669F70C945C6A83E50F94B7ACE4
:10AB9000882351F00F94AFAC60931311709314118C
:10ABA000809315119093161186E40F94B7AC882307
:10ABB00081F00F94AFAC20E030E040E752E40F9416
:10ABC00091BA609317117093181180931911909393
:10ABD0001A118AE50F94B7AC882311F40C945C6ABF
:10ABE0000F94AFAC60931B1170931C1180931D11D7
:10ABF00090931E110C945C6A83E50F94B7AC882384
:10AC000051F00F94AFAC60931F117093201180939B
:10AC100021119093221186E40F94B7AC882311F48C
:10AC20000C945C6A0F94AFAC20E030E040E752E453
:10AC30000F9491BA6093231170932411809325117E
:10AC4000909326110C945C6A83E50F94B7AC88232B
:10AC500011F40C945C6A0F94AFAC0F9402BB6115B5
:10AC6000710551F06130710569F481E08093121132
:10AC70001092180F0C945C6A109212111092180F17
:10AC80000C945C6AE9EBFDE584918F01882339F02F
:10AC90000F94A14F0F5F1F4FF8018491F7CFE9E3A5
:10ACA000F5E084918F01882339F00F94A14F0F5F55
:10ACB0001F4FF8018491F7CF00917315109174150F
:10ACC00007571C4ED8018D918D01882319F00F94E0
:10ACD000A14FF8CFEDE3FEE084918F01882311F4BA
:10ACE0000C94E2460F94A14F0F5F1F4FF80184911F
:10ACF000F5CF82E40F94B7AC882341F080915502E0
:10AD000090915602909305028093040283E50F947C
:10AD1000B7AC882341F00F94AFAC0F9402BB709393
:10AD200056026093550282E50F94B7AC882311F464
:10AD30000C945C6A809104029091050290935602F3
:10AD4000809355020C945C6A83E50F94B7AC88231A
:10AD500009F466CD0F94AFAC0F9402BB6B017C017C
:10AD600084E50F94B7AC882359F0BE016F5F7F4F25
:10AD70008DED90E00F94D2AA81110C945C6A50CDB5
:10AD8000D0926002C0925F024BCD80E50F94B7ACC9
:10AD9000882311F40C945C6A0F94AFAC0F9402BB3F
:10ADA000F62E862F972F6C0183E50F94B7AC88237E
:10ADB00031F00F94AFAC0F9402BB8B0102C00FEFC8
:10ADC0001FEFC8010196039710F00C945C6AEDE840
:10ADD000F2E085EC92E021913191C216D30611F494
:10ADE0000C945C6A8E179F07B1F7D7FE02C00C94D3
:10ADF0005C6A0F940389EF2C60E08F2D0F94D621AD
:10AE00000F3FFFEF1F0731F00130110571F401E032
:10AE100010E00DC08F2D0F94802131E020E0892BB0
:10AE200009F030E0032F122F02C000E010E08E2D59
:10AE30000F9480218017910711F40C945C6A0F9491
:10AE4000378280E00F94614080E00F94BE0EEFCF18
:10AE500083E50F94B7AC882331F00F94AFAC0F9417
:10AE600002BB8B0102C00EE610E080E50F94B7AC88
:10AE7000882329F00F94AFAC0F9402BB02C068EE98
:10AE800073E0072E000C880B990B1016110694F432
:10AE900020910A0730910B072230310528F42091C8
:10AEA00002012460209302010F949E530F94EE7AC6
:10AEB0000C945C6A0F949E530C945C6A80E50F942A
:10AEC000B7AC882351F00F94AFAC6093F810709337
:10AED000F9108093FA109093FB1089E40F94B7ACAB
:10AEE000882381F00F94AFAC2CEA35EC47E25EE3A7
:10AEF0000F94A9AD6093FC107093FD108093FE1029
:10AF00009093FF1084E40F94B7AC882381F00F94E2
:10AF1000AFAC2CEA35EC47E25EE30F9491BA609354
:10AF2000001170930111809302119093031183E437
:10AF30000F94B7AC882351F00F94AFAC609300022C
:10AF40007093010280930202909303020F94118880
:10AF5000E2E4F7E184918F01882339F00F94A14F47
:10AF60000F5F1F4FF8018491F7CF04E114E0D8017F
:10AF70008D918D01882319F00F94A14FF8CF609126
:10AF8000F8107091F9108091FA109091FB1042E046
:10AF90000F94265008E114E0F80181918F01882375
:10AFA00019F00F94A14FF8CF2CEA35EC47E25EE39D
:10AFB0006091FC107091FD108091FE109091FF1037
:10AFC0000F9491BA42E00F9426500CE114E0D8019E
:10AFD0008D918D01882319F00F94A14FF8CF2CEAA1
:10AFE00035EC47E25EE360910011709101118091B0
:10AFF0000211909103110F94A9AD42E00F942650D5
:10B0000000E214E0F80181918F01882319F00F9478
:10B01000A14FF8CF6091000270910102809102026D
:10B020009091030242E00F9426508AE00F94A14FC2
:10B030000C945C6A80E50F94B7AC882351F00F94B0
:10B04000AFAC609304117093051180930611909337
:10B05000071189E40F94B7AC882381F00F94AFAC4B
:10B060002CEA35EC47E25EE30F94A9AD609308113A
:10B070007093091180930A1190930B1184E40F943B
:10B08000B7AC882381F00F94AFAC2CEA35EC47E2E3
:10B090005EE30F9491BA60930C1170930D1180933D
:10B0A0000E1190930F110F941188E2E4F7E184914F
:10B0B0008F01882339F00F94A14F0F5F1F4FF801C4
:10B0C0008491F7CF04E114E0D8018D918D0188239C
:10B0D00019F00F94A14FF8CF6091041170910511F0
:10B0E000809106119091071142E00F94265008E1DB
:10B0F00014E0F80181918F01882319F00F94A14F7A
:10B10000F8CF2CEA35EC47E25EE3609108117091CC
:10B11000091180910A1190910B110F9491BA42E09C
:10B120000F9426500CE114E0D8018D918D018823F5
:10B1300019F00F94A14FF8CF2CEA35EC47E25EE30B
:10B1400060910C1170910D1180910E1190910F1161
:10B150000F94A9AD42E00F9426508AE00F94A14FBE
:10B160000C945C6A83E50F94B7AC882319F00F94B4
:10B17000AFAC03C060E070E0CB01609361027093FC
:10B18000620280936302909364020C945C6A85E48B
:10B190000F94B7AC882359F00F94AFAC0F9402BB57
:10B1A00024967FAF6EAF249777FF05C013C0249617
:10B1B0001FAE1EAE249763961FAE639765961FAEB3
:10B1C000659726E167962FAF679733E468963FAFA0
:10B1D00068970EC063961FAE639765961FAE65971E
:10B1E0004CE867964FAF679752E468965FAF6897F1
:10B1F00083E50F94B7AC882371F00F94AFAC6396DE
:10B200006FAF639765967FAF659767968FAF6797C8
:10B2100068969FAF689783E40F94B7AC882349F092
:10B220000F94AFAC0F9402BBA6967FAF6EAFA697FC
:10B2300006C085E090E0A6969FAF8EAFA697A69633
:10B240008EAC9FACA69790924D0D80924C0D1092B3
:10B25000F30E10924F0D10924E0D0F94D65362962E
:10B260006CAF7DAF8EAF9FAF62972496AEACBFAC94
:10B270002497B7FC05C02AE0A7962FAFA79704C074
:10B280003DE2A7963FAFA7970F94D653E3966CAFD6
:10B290007DAF8EAF9FAFE39724968EAC9FAC249783
:10B2A00018141904B4F404E214E0D8018D918D014E
:10B2B000882319F00F94A14FF8CF8AE00F94A14F83
:10B2C00081E08093F30E10924F0D10924E0D0C946E
:10B2D0005C6A0EE414E0F80181918F01882319F073
:10B2E0000F94A14FF8CF8AE00F94A14F0F945D49BE
:10B2F00024968EAC9FAC24978FE7892809F454C01C
:10B300008093B00F8EEF0F942C5462968CAC9DAC52
:10B31000AEACBFAC62976C968CAE9DAEAEAEBFAE1F
:10B320006C97AF968CAE9DAEAEAEBFAEAF972B9680
:10B330001FAE2B976D961FAE6D9720E46E962FAFC4
:10B340006E973CE16F963FAF6F9746E4A0964FAF84
:10B35000A097A1961FAEA197A2961FAEA297A39603
:10B360001FAEA397A4961FAEA497EFE78E2E912C45
:10B37000A12CB12C2A968CAE9DAEAEAEBFAE2A9754
:10B38000FFE74F2E512C612C712CAB961CAE1DAEDD
:10B390001EAE1FAEAB9721E0E8962FAFE8971AAE2E
:10B3A0001EAE212C312C06C08093B10FAECF80E0B1
:10B3B0000F94BE0EA8958091B20F882309F47AC12C
:10B3C0000F94E24D24968EAC9FAC2497892859F4B3
:10B3D00090901B0F9AAEA0901C0FAEAE20901D0F48
:10B3E00030901E0F0AC0B0901107BAAE80901207BD
:10B3F0008EAE20901307309014072AAD3EADA10108
:10B40000A1966FADA197A2967FADA297A3968FAD9F
:10B41000A397A4969FADA4970F94EEBB181674F053
:10B420009AACA1969FAEA197AEACA296AFAEA297F2
:10B43000A3962FAEA397A4963FAEA4976D962FAD7B
:10B440006D976E963FAD6E976F964FAD6F97A096C6
:10B450005FADA0976AAD7EADC1010F94EEBB18162B
:10B4600074F0BAAC6D96BFAE6D978EAC6E968FAE23
:10B470006E976F962FAE6F97A0963FAEA0970F94E2
:10B48000D653DC01CB01E3968CAC9DACAEACBFAC2B
:10B49000E39788199909AA09BB09853C9940A10538
:10B4A000B10550F00F941A820F94D653E3966CAF07
:10B4B0007DAF8EAF9FAFE397E8968FACE89788207B
:10B4C00009F477C02AAD3EADA10163966FAD6397D5
:10B4D00065967FAD659767968FAD679768969FADC8
:10B4E00068970F943CB487FFE5C00F94D653DC01F6
:10B4F000CB0162968CAC9DACAEACBFAC62978819A8
:10B500009909AA09BB0989389341A105B10508F435
:10B51000D1C0D301C2012A968CAC9DACAEACBFACFD
:10B520002A9788199909AA09BB092496AEACBFAC21
:10B530002497B595A79597958795AB2831F080937B
:10B54000B00F880F0F942C5402C08093B10F0F944A
:10B55000D6536C966CAF7DAF8EAF9FAF6C974B019F
:10B560005C0162962CAD3DAD4EAD5FAD6297821A27
:10B57000930AA40AB50AAB968CAE9DAEAEAEBFAE32
:10B58000AB9763968FAC6397A1968FAEA1976596A4
:10B590009FAC6597A2969FAEA2976796AFAC679750
:10B5A000A396AFAEA3976896BFAC6897A496BFAEBC
:10B5B000A4972AAD3EADA10163966FAD63976596E2
:10B5C0007FAD659767968FAD679768969FAD6897D3
:10B5D0000F94EEBB181614F00C94DC700F94D65335
:10B5E000DC01CB016C968CAC9DACAEACBFAC6C9767
:10B5F00088199909AA09BB0989389341A105B105A0
:10B6000010F40C94DC700F94D65362966CAF7DAF3F
:10B610008EAF9FAF6297DC01CB0188199909AA0907
:10B62000BB0920914E0D30914F0D1216130614F4E4
:10B630000C94076F2A968CAD9DADAEADBFAD2A9729
:10B64000840D951DA61DB71D24968EAC9FAC249726
:10B65000B595A79597958795892811F40C94D8707E
:10B660008093B00F880F0F942C5480914E0D9091C1
:10B670004F0D019690934F0D80934E0D63969FACA6
:10B6800063976D969FAE6D976596AFAC65976E9616
:10B69000AFAE6E976796BFAC67976F96BFAE6F976A
:10B6A00068968FAC6897A0968FAEA09721E0E89639
:10B6B0002FAFE89720E030E040EA51E463966FADA9
:10B6C000639765967FAD659767968FAD6797689628
:10B6D0009FAD68970F94A3B92AAD3EADA1010F9419
:10B6E0003CB487FF0EC0E8E3FCE084918F0188231F
:10B6F00009F4E3CD0F94A14F0F5F1F4FF801849120
:10B70000F6CF0F94D653DC01CB01AF968CAC9DAC39
:10B71000AEACBFACAF9788199909AA09BB09813DA6
:10B720009740A105B10508F4B4C024968EAC9FAC37
:10B730002497892881F0E090B00FF12CE5E3FCE03C
:10B7400084918F018823B9F00F94A14F0F5F1F4F91
:10B75000F8018491F7CFE090B10FF12CE2E3FCE027
:10B7600084918F01882339F00F94A14F0F5F1F4FF1
:10B77000F8018491F7CF42E06AAD7EADC1010F942C
:10B780002650EEE2FCE084918F01882339F00F947B
:10B79000A14F0F5F1F4FF8018491F7CFB701FF0C46
:10B7A000880B990B0F9491658AE00F94A14F2B960B
:10B7B0008FAC2B97882009F452C0A7969FACA7970F
:10B7C000891418F4282D2F5F59C02B968FAC2B9716
:10B7D000A7969FACA797891054C0282D2F5F2B9652
:10B7E0002FAF2B97E4962FADE497E5963FADE59705
:10B7F000E6964FADE697E7965FADE7976AAD7EAD0B
:10B80000C1010F94A2B96B017C0120E030E0A901D5
:10B810000F94EEBB18165CF420E030E040EA50E4F0
:10B82000C701B6010F943CB487FF2BC00AC020E0CB
:10B8300030E040EA50ECC701B6010F94EEBB181699
:10B8400004F524966FAD2497661F6627661F80E077
:10B850000F94CD4981E08093F30E0C945C6A8AAC1E
:10B86000E4968FAEE4979EACE5969FAEE597E6969C
:10B870002FAEE697E7963FAEE79721E02B962FAFE6
:10B880002B970F94D653AF966CAF7DAF8EAF9FAF13
:10B89000AF970F94D6536B017C010F94D6536C96DF
:10B8A0000CAD1DAD2EAD3FAD6C9762968CAC9DACD2
:10B8B000AEACBFAC6297080D191D2A1D3B1DC01A06
:10B8C000D10AE20AF30ADC01CB018C0D9D1DAE1DED
:10B8D000BF1D81389F44A241B10570F0E1E1FCE059
:10B8E00084918F01882309F4E8CC0F94A14F0F5F56
:10B8F0001F4FF8018491F6CF80914E0D90914F0D1E
:10B90000A6968EAC9FACA697881699060CF04FCDE4
:10B91000E5EBFBE084918F01882309F4CECC0F94F2
:10B92000A14F0F5F1F4FF8018491F6CF0F94038949
:10B930000C945C6A80912D10882311F40C945C6A3D
:10B9400085E40F94B7AC882331F00F94AFAC0F941B
:10B9500008BB162F01C01FEF86E40F94B7AC8823F5
:10B9600031F00F94AFAC0F9408BB062F01C00FEF5E
:10B970001F920F931F921F9384EA9BE09F938F93D4
:10B980000F9447B31F920F931F921F938CE99BE074
:10B990009F938F930E947EA10FB6F894DEBF0FBED7
:10B9A000CDBF1AE00E9469A1181614F40C945C6AC9
:10B9B000115011F00C94E1700C945C6A0F941C51BE
:10B9C0000C945C6A0F94E6500C945C6A8091F310BE
:10B9D0008F938091F2108F938091F1108F938091CB
:10B9E000F0108F938091EF108F938091EE108F93D2
:10B9F0008091ED108F938091EC108F938091EB10DC
:10BA00008F938091EA108F938091E9108F938091AA
:10BA1000E8108F9309EB1DE51F930F931F930F936E
:10BA20008091E7108F938091E6108F938091E510BD
:10BA30008F938091E4108F938091E3108F93809186
:10BA4000E2108F938091E1108F938091E0108F939B
:10BA50008091DF108F938091DE108F938091DD10A5
:10BA60008F938091DC108F938091DB108F93809166
:10BA7000DA108F938091D9108F938091D8108F9383
:10BA80008091D7108F938091D6108F938091D5108D
:10BA90008F938091D4108F938091D3108F93809146
:10BAA000D2108F938091D1108F938091D0108F936B
:10BAB0008091CF108F938091CE108F938091CD1075
:10BAC0008F938091CC108F931F930F931F930F939D
:10BAD0008091CB108F938091CA108F938091C91061
:10BAE0008F938091C8108F938091C7108F9380910E
:10BAF000C6108F938091C5108F938091C4108F933F
:10BB00001F930F931F930F9380914B118F938091ED
:10BB10004A118F93809149118F93809148118F938F
:10BB2000809147118F93809146118F938091451199
:10BB30008F93809144118F93809143118F938091C3
:10BB400042118F93809141118F93809140118F9377
:10BB500080913F118F9380913E118F9380913D1181
:10BB60008F9380913C118F931F930F931F930F938B
:10BB70008091C3108F938091C2108F938091C110D8
:10BB80008F938091C0108F938091BF108F9380917D
:10BB9000BE108F938091BD108F938091BC108F93B6
:10BBA0008091BB108F938091BA108F938091B910C0
:10BBB0008F938091B8108F938091B7108F9380915D
:10BBC000B6108F938091B5108F938091B4108F939E
:10BBD0001F930F931F930F9380913B118F9380912D
:10BBE0003A118F93809139118F93809138118F93EF
:10BBF000809137118F93809136118F9380913511F9
:10BC00008F93809134118F93809133118F93809112
:10BC100032118F93809131118F93809130118F93D6
:10BC200080912F118F9380912E118F9380912D11E0
:10BC30008F9380912C118F931F930F931F930F93CA
:10BC40008091B3108F938091B2108F938091B11037
:10BC50008F938091B0108F938091AF108F938091CC
:10BC6000AE108F938091AD108F938091AC108F9315
:10BC70008091AB108F938091AA108F938091A9101F
:10BC80008F938091A8108F938091A7108F938091AC
:10BC9000A6108F938091A5108F938091A4108F93FD
:10BCA0001F930F931F930F938091A3108F938091F5
:10BCB000A2108F938091A1108F938091A0108F93E9
:10BCC00080919F108F9380919E108F9380919D10F3
:10BCD0008F9380919C108F9380919B108F93809174
:10BCE0009A108F93809199108F93809198108F93D1
:10BCF000809197108F93809196108F9380919510DB
:10BD00008F93809194108F931F930F931F930F9392
:10BD10008CEE98E09F938F930F9447B30FB6F894EF
:10BD2000DEBF0FBECDBF2CEA35EC47E25EE360918B
:10BD300000117091011180910211909103110F94E3
:10BD4000A9AD9F938F937F936F932CEA35EC47E2D5
:10BD50005EE36091FC107091FD108091FE10909157
:10BD6000FF100F9491BA9F938F937F936F9380915D
:10BD7000FB108F938091FA108F938091F9108F931D
:10BD80008091F8108F931F930F931F930F938FEB56
:10BD900098E09F938F930F9447B32CEA35EC47E2DA
:10BDA0005EE360910C1170910D1180910E119091D4
:10BDB0000F110F94A9AD9F938F937F936F932CEAEC
:10BDC00035EC47E25EE360910811709109118091B2
:10BDD0000A1190910B110F9491BA9F938F937F93B7
:10BDE0006F93809107118F93809106118F938091AB
:10BDF00005118F93809104118F931F930F931F93BD
:10BE00000F938AE898E09F938F930F9447B30FB6F0
:10BE1000F894DEBF0FBECDBF809112111F928F9399
:10BE20001F930F931F930F9320E030E040E752E4FD
:10BE30006091231170912411809125119091261108
:10BE40000F94A9AD9F938F937F936F93809122114D
:10BE50008F93809121118F93809120118F938091E6
:10BE60001F118F931F930F931F930F9380911E1198
:10BE70008F9380911D118F9380911C118F938091CE
:10BE80001B118F9320E030E040E752E460911711DE
:10BE9000709118118091191190911A110F94A9ADF8
:10BEA0009F938F937F936F93809116118F938091BF
:10BEB00015118F93809114118F93809113118F938B
:10BEC0001F930F931F930F9389E897E09F938F938E
:10BED0000F9447B30FB6F894DEBF0FBECDBF80916D
:10BEE00027118823E9F080912B118F9380912A11DB
:10BEF0008F93809129118F93809128118F931F9395
:10BF00000F931F930F9383E697E09F938F930F9464
:10BF100047B30FB6F894DEBF0FBECDBF0C945C6A7A
:10BF20001F930F9384E497E09F938F930F9447B3ED
:10BF30000F900F900F900F900C945C6AE9EBFDE569
:10BF400084918F01882339F00F94A14F0F5F1F4F09
:10BF5000F8018491F7CFEDE2FEE084918F01882310
:10BF600011F40C945C6A0F94A14F0F5F1F4FF801FE
:10BF70008491F5CF8AE50F94B7AC882309F489C082
:10BF80000F94AFAC6B017C0120E030E040E751EC56
:10BF90000F94EEBB87FD38C020E030E040EA50EC63
:10BFA000C701B6010F943CB4181674F1F7FAF09477
:10BFB000F7F8F094C092F410D092F510E092F610D9
:10BFC000F092F710E9EBFDE584918F01882339F0B9
:10BFD0000F94A14F0F5F1F4FF8018491F7CFE0E35B
:10BFE000F5E084918F01882339F00F94A14F0F5F02
:10BFF0001F4FF8018491F7CF8AE00F94A14F8AE098
:10C000000F94A14F0C945C6AE9EBFDE584918F01DC
:10C01000882339F00F94A14F0F5F1F4FF8018491CF
:10C02000F7CFE0E3F5E084918F01882339F00F9496
:10C03000A14F0F5F1F4FF8018491F7CFEBE6F5E0BA
:10C0400084918F01882339F00F94A14F0F5F1F4F08
:10C05000F8018491F7CF61EF7FEF8FEF9FEF0F949F
:10C060009165E3E6F5E084918F01882339F00F9420
:10C07000A14F0F5F1F4FF8018491F7CF6BEF7FEF58
:10C080008FEF9FEF0F9491658AE00F94A14F0C946E
:10C090005C6AE9EBFDE584918F01882339F00F9408
:10C0A000A14F0F5F1F4FF8018491F7CFE0E3F5E058
:10C0B00084918F01882339F00F94A14F0F5F1F4F98
:10C0C000F8018491F7CF8AE00F94A14F8091F4108A
:10C0D0009091F510A091F610B091F710BC01CD0130
:10C0E000905842E00F9426508AE00F94A14F0C9490
:10C0F0005C6A0F94038985E40F94B7AC882329F018
:10C100000F94AFAC6B017C0105C0C12CD12CE12C8C
:10C1100000ECF02E8CE40F94B7AC81110F94AFAC0F
:10C120008AE50F94B7AC882329F00F94AFAC2B01AC
:10C130003C011CC020E030E048EC51E46091541018
:10C140007091551080915610909157100F943CB4F7
:10C1500087FF07C0412C512C18ED612E11E4712E80
:10C1600005C0412C512C612CB0E47B2E88E50F9446
:10C17000B7AC882339F00F94AFAC6AAF7BAF8CAF0C
:10C180009DAF0AC0812C912CA3E5AA2EA3E4BA2E60
:10C190008AAE9BAEACAEBDAE89E50F94B7AC88233A
:10C1A00049F00F94AFAC22966CAF7DAF8EAF9FAFCE
:10C1B000229706C022961CAE1DAE1EAE1FAE229761
:10C1C00080912D10882311F40C94E77081E694E09F
:10C1D0000F943D60882311F40C94E770332433945A
:10C1E0000F9403898091070F882329F060E086E18E
:10C1F00090E00E9426F7909055022F969FAE2F97C1
:10C2000020905602E091070DF0E0EE0FFF1FEB5873
:10C21000FA4EA080B1806496BFAEAEAE6497209116
:10C22000C0193091C11966963FAF2EAF66978091C5
:10C230004C1090914D10A0914E10B0914F10269639
:10C240008CAF9DAFAEAFBFAF269789839A83AB8388
:10C25000BC838090501090905110A0905210B090DC
:10C2600053102A968CAE9DAEAEAEBFAE2A978D828D
:10C270009E82AF82B8862091541030915510409123
:10C280005610509157102E962CAF3DAF4EAF5FAF6A
:10C290002E9729873A874B875C87209158103091D9
:10C2A000591040915A1050915B102D873E874F874F
:10C2B000588BC701B6010F94A3B9609358107093BF
:10C2C000591080935A1090935B1047E05DE05F93A4
:10C2D0004F93812C912C98EEA92E92E4B92E28E54B
:10C2E000C22E20E1D22E2E96ECACFDAC0EAD1FADD1
:10C2F0002E972A962CAD3DAD4EAD5FAD2A97269672
:10C300006CAD7DAD8EAD9FAD26970F94EF2C0F9445
:10C31000038920915410309155104091561050913E
:10C320005710C301B2010F94A3B97B018C01609334
:10C33000541070935510809356109093571020917D
:10C340005010309151104091521050915310609103
:10C350004C1070914D1080914E1090914F10A7E0AD
:10C36000BDE0BF93AF93812C912CE0E7AE2EE1E4CA
:10C37000BE2E0F94EF2C0F9403898AAC9BACACAC0F
:10C38000BDAC80924C1090924D10A0924E10B09285
:10C390004F1022962CAD3DAD4EAD5FAD2297209350
:10C3A0005010309351104093521050935310E0901E
:10C3B0005410F0905510009156101091571047E00E
:10C3C0005DE05F934F93812C912CF8E4AF2EF2E463
:10C3D000BF2E22962CAD3DAD4EAD5FAD22976AAD1E
:10C3E0007BAD8CAD9DAD0F94EF2C0F9403890F9016
:10C3F0000F900F900F900F900F9080912D10811142
:10C4000024C084E090E090932602809325020F944C
:10C41000D6534B015C0183E990E10E94FBFBCC24E5
:10C42000C394D12CE12CF12CD1100C942B710F94CE
:10C430008F0F882311F40C942B719FB7F89480917F
:10C4400002018B7F809302019FBF1092B006809102
:10C450002D10882319F00E9410A102C00E940FDB4A
:10C460000F94038980912D1081115DC084E090E0CC
:10C47000909326028093250241E060E08CEA91E1EE
:10C480000E9408FC8093B006811148C00F944416A6
:10C4900062E080E00F94971180E499E40F94BE105D
:10C4A00020E030E048EC52E460914C1070914D1067
:10C4B00080914E1090914F100F94A2B960934C1040
:10C4C00070934D1080934E1090934F10E090541045
:10C4D000F090551000915610109157102091501067
:10C4E000309151104091521050915310E7E0FDE00F
:10C4F000FF93EF93812C912CB8E4AB2EB2E4BB2ECA
:10C50000E8E5CE2EE0E1DE2E0F94EF2C0F940389A8
:10C510008CE791E10E94ACFC0F900F9080912D1060
:10C52000882309F478C0311072C080917F0E88236F
:10C5300029F060E080913B020E94D99F84E090E066
:10C5400090932602809325028CEB90E10E94FBFBE6
:10C55000FF24F39400E010E00F948F0F811139C095
:10C560000F94378281E00F946140043F41E014074B
:10C5700011F400E010E080910101846080930101DA
:10C5800001151105A1F480910A0790910B070097FE
:10C5900021F00197B9F4FF20A9F09FB7F89480919A
:10C5A00002018460809302019FBFF12C0BC0043113
:10C5B000110541F49FB7F894809102018B7F80931D
:10C5C00002019FBF0F5F1F4F84E090E00F94C144B2
:10C5D000C3CF9FB7F894809102018B7F80930201B3
:10C5E0009FBF80917F0E882391F00F94441662E0E4
:10C5F00080E00F94971180E499E40F94BE1080E6D8
:10C600000E94AC9E40E060E080E00E94FB9A832D97
:10C610000F94A0A159C00F94441661E080E00F94DC
:10C62000971185E191E10F94BE108091070281116D
:10C6300007C062E00F94971182E091E10F94BE1061
:10C6400084E090E090932602809325020E94C9B373
:10C650000F948F0F81111AC00F94378281E00F94CD
:10C6600061400E9410B4882399F380910A07909149
:10C670000B07029728F480910201846080930201E5
:10C6800082E390E00F94C1440F94EE7A0E946EB260
:10C6900082E090E090932602809325020F9441A1BE
:10C6A00080910A0790910B07029728F4809102016C
:10C6B00084608093020182E390E00F94C1440F9460
:10C6C000EE7A80E00F944E163110F3C01092B0064F
:10C6D000F4E0CF2ED12CA2E0AA2EB12C8091B0068E
:10C6E000813009F4E6C01092B006D0922602C092C2
:10C6F00025020F94441660E080E00F9497118BE4BC
:10C7000091E10F94BE1061E081E00F94971180E1F8
:10C7100094E40F94BE1062E081E00F94971187E3D8
:10C7200091E10F94BE1063E081E00F94971185E2D0
:10C7300091E10F94BE1061E080E00F94971186E6BE
:10C7400094E00F943410E090C2190E2C000CFF08F6
:10C750000E9436B201E010E08091B006811168C0FD
:10C760000F94378281E00F9461408091C219082EA6
:10C77000000C990B9701281B390B37FF03C031952B
:10C7800021953109253031050CF444C08E159F05E3
:10C7900014F401501109E816F90634F40F5F1F4F25
:10C7A0000430110564F009C00430110534F401159A
:10C7B000110529F401E010E002C003E010E061E09F
:10C7C00080E00F9497118FE396E00F94341062E0AD
:10C7D00080E00F9497118FE396E00F94341063E09C
:10C7E00080E00F9497118FE396E00F943410602F40
:10C7F00080E00F94971186E694E00F943410E09057
:10C80000C2190E2C000CFF0864E670E080E090E096
:10C810000F949E530F948F0F882309F49DCF00939C
:10C82000B00664EF71E080E090E00F949E5394CFE7
:10C830000F9444160F94A08CB0922602A092250269
:10C840008091B0068230F9F0833041F50F9403896E
:10C850000E940B8A0F94441660E080E00F949711B9
:10C860008EE591E10F94BE1062E080E00F94971185
:10C8700080E499E40F94BE1087E99DE10F940BA228
:10C880000F9403892BCF80912D10882321F080E015
:10C890000F94A0A123CF0F9441A120CF0F94441651
:10C8A00062E080E00F9497118CE691E10F94BE1046
:10C8B00015CF81E00F944E1666968EAD9FAD6697AC
:10C8C0009093C1198093C01931103FC020E030E02F
:10C8D00040EA50E4609158107091591080915A10BC
:10C8E00090915B100F94A3B96093581070935910F6
:10C8F00080935A1090935B10E0905410F090551074
:10C9000000915610109157102091501030915110F5
:10C91000409152105091531060914C1070914D10F5
:10C9200080914E1090914F10E7E0FDE0FF93EF9360
:10C93000812C912CA12CB0E4BB2EE8E5CE2EE0E1B9
:10C94000DE2E0F94EF2C0F900F90E0905410F0908B
:10C95000551000915610109157102D813E814F8136
:10C96000588569817A818B819C81B7E06B2EBDE00F
:10C970007B2E7F926F92812C912CE8E4AE2EE2E424
:10C98000BE2EF8E5CF2EF0E1DF2E0F94EF2C0F94A2
:10C990000389E984FA840B851C852D813E814F81B2
:10C9A000588569817A818B819C817F926F92812CDD
:10C9B000912CA0E7AA2EA1E4BA2E0F94EF2C0F948D
:10C9C0000389CE010D960E9440D680E1FE0131968A
:10C9D000ACE4B0E101900D928A95E1F780E1ECE4DE
:10C9E000F0E1A8E0BFE001900D928A95E1F72F9663
:10C9F0009FAD2F9790935502209256022F929F93AE
:10CA00008BE397E09F938F938E01015E1F4F1F93DF
:10CA10000F930F94A0B360E0C8010E9415EA8EE165
:10CA200094E10F9423261092650E1092640E0FB6B7
:10CA3000F894DEBF0FBECDBF3FC50E942CE73CC5BA
:10CA400083E50F94B7AC882309F436C50F94AFACD7
:10CA50000F9402BB6B017C012B0180E499E40F94DD
:10CA60002326EAE0FEE084918F01882339F00F94B9
:10CA7000A14F0F5F1F4FF8018491F7CF0D2C000CD1
:10CA8000EE08FF08C701B6010F9491658AE00F9484
:10CA9000A14F0F94D6534B015C0110927E0E609112
:10CAA0000B0D70910C0D072E000C880B990B0F9439
:10CAB00042B420E030E0A9010F943CB4811111C0D0
:10CAC0006091751570917615072E000C880B990BE7
:10CAD0000F9442B411E020E030E0A9010F943CB47F
:10CAE000811110E0052C000C66087708A5E02A2EBD
:10CAF000AEE03A2E111115C080917E0E81116CC0EE
:10CB0000C301B2010F9442B4209188193091891960
:10CB100040918A1950918B190F94EEBB18168CF026
:10CB20005BC0C301B2010F9442B4209188193091C7
:10CB3000891940918A1950918B190F943CB487FF41
:10CB40004BC00F94D653DC01CB0188199909AA096F
:10CB5000BB09893E9340A105B10508F434C0E7E064
:10CB6000FEE084915F01882341F00F94A14FFFEF15
:10CB7000AF1ABF0AF5018491F6CF609188197091C0
:10CB8000891980918A1990918B1941E00F94265050
:10CB9000F1018491F5E0AF2EFEE0BF2E882341F035
:10CBA0000F94A14FFFEFAF1ABF0AF5018491F6CFA2
:10CBB000C701B6010F9491658AE00F94A14F0F94BD
:10CBC000D6534B015C010F94378280E00F94614093
:10CBD00080E00F94BE0E8ECF82E497E10F9423265F
:10CBE0006BC48FE30F94B7AC882309F4BCC00F94D7
:10CBF00024621A821982882381F008E614E0D801A1
:10CC00008D918D01882319F00F94A14FF8CF8AE000
:10CC10000F94A14F0CE714E00AC003E914E0F801F7
:10CC200081918F01882399F30F94A14FF8CFD801F8
:10CC30008D918D01882319F00F94A14FF8CF8AE0D0
:10CC40000F94A14F88248A94982C540173E2472EA4
:10CC5000512C612C712CE0EB2E2EEFE03E2E1AAE03
:10CC600069817A81072E000C880B990B0F9442B4CE
:10CC700020919C1030919D1040919E1050919F10DA
:10CC80000F9491BA6B017C012AAD21110DC0E1E036
:10CC9000FEE084918F01882359F00F94A14F0F5F1C
:10CCA0001F4FF8018491F7CFC501B4010F9491652E
:10CCB000EEEFFDE084918F01882339F00F94A14FAE
:10CCC0000F5F1F4FF8018491F7CFC301B2010F949A
:10CCD0009165EBEFFDE084918F01882339F00F948B
:10CCE000A14F0F5F1F4FF8018491F7CF69817A81BF
:10CCF000072E000C880B990B0F949165E8EFFDE06F
:10CD000084918F01882339F00F94A14F0F5F1F4F3B
:10CD1000F8018491F7CF20E030E04AE754E4C701FE
:10CD2000B6010F94A9AD42E00F9426508AE00F940B
:10CD3000A14FFAADFF5FFAAFF63009F4BDC3BE01F3
:10CD40006F5F7F4FC1010E9477C5B2E02B0E311C8F
:10CD5000E5E04E0E511C611C711CFFEF8F1A9F0AFB
:10CD6000AF0ABF0A7DCF81E20F94B7AC882309F4E4
:10CD70004AC061E086EA9FE00F9447B988E090E0FE
:10CD80009A838983BE016F5F7F4F80EB9FE00E9493
:10CD900091C588E190E09A838983BE016F5F7F4FE0
:10CDA00082EB9FE00E9491C580E390E09A838983A3
:10CDB000BE016F5F7F4F84EB9FE00E9491C580E5CD
:10CDC00090E09A838983BE016F5F7F4F86EB9FE07F
:10CDD0000E9491C588E790E09A838983BE016F5FC6
:10CDE0007F4F88EB9FE00E9491C507EA14E0D801CD
:10CDF0008D918D01882319F00F94A14FF8CF8AE00F
:10CE00000F94A14F59C38AE50F94B7AC882319F149
:10CE100061E086EA9FE00F9447B91A82198200EB1D
:10CE20001FE0BE016F5F7F4FC8010E9491C50E5F7A
:10CE30001F4F0A3BBFE01B07A1F708EB14E0F80106
:10CE400081918F01882319F00F94A14FF8CF8AE0C8
:10CE50000F94A14F31C383E50F94B7AC882309F435
:10CE6000CEC00F94AFAC0F9402BB7A83698389E480
:10CE70000F94B7AC882309F41FC30F94AFAC0F9481
:10CE800008BB653008F018C3862F90E08852984F91
:10CE9000BE016F5F7F4F880F991F0E9491C502EC02
:10CEA00014E0D8018D918D01882319F00F94A14FC2
:10CEB000F8CF8AE00F94A14F0CE714E0F8018191BC
:10CEC0008F01882319F00F94A14FF8CF8AE00F94B7
:10CED000A14F2EEA222E2FE0322E44244A94542CC5
:10CEE000320143E2842E912CA12CB12C1AAE1A826D
:10CEF0001982FAADFF2331F0BE016F5F7F4FC10190
:10CF00000E9477C569817A81072E000C880B990BE6
:10CF10000F9442B420919C1030919D1040919E102E
:10CF200050919F100F9491BA6B017C012AAD211191
:10CF30000DC0E4EFFDE084918F01882359F00F9438
:10CF4000A14F0F5F1F4FF8018491F7CFC301B201CA
:10CF50000F949165E1EFFDE084918F01882339F012
:10CF60000F94A14F0F5F1F4FF8018491F7CFC501B8
:10CF7000B4010F949165EEEEFDE084918F0188235A
:10CF800039F00F94A14F0F5F1F4FF8018491F7CF35
:10CF900069817A81072E000C880B990B0F9491659B
:10CFA000EBEEFDE084918F01882339F00F94A14FBF
:10CFB0000F5F1F4FF8018491F7CF20E030E04AE780
:10CFC00054E4C701B6010F94A9AD42E00F94265076
:10CFD0008AE00F94A14FFAADFF5FFAAF25E0820E11
:10CFE000911CA11CB11C3FEF431A530A630A730A38
:10CFF00042E0240E311CF63009F079CF5DC2EAED33
:10D00000FDE084918F01882309F456C20F94A14F4B
:10D010000F5F1F4FF8018491F6CF0F9403898BE4C3
:10D020000F94B7AC882399F00F947CAC6B017C0112
:10D0300020E030E0A9010F94EEBB87FD08C0C0924C
:10D04000690FD0926A0FE0926B0FF0926C0F82E53D
:10D050000F94B7AC882361F00F947CAC6B017C011A
:10D0600020E030E0A9010F943CB487FF89C006C0DE
:10D07000C12CD12C90E8E92E9FEBF92E84E40F947B
:10D08000B7AC882329F00F947CAC4B015C0106C03F
:10D09000812C912C80E8A82E8FEBB82E87E50F9479
:10D0A000B7AC882329F00F947CAC2B013C0106C05F
:10D0B000412C512C00E8602E0FEB702E88E40F9469
:10D0C000B7AC882339F00F947CAC6AAF7BAF8CAFE0
:10D0D0009DAF08C020E030E040E85FEB2AAF3BAFF7
:10D0E0004CAF5DAF20E030E0A901C501B4010F9461
:10D0F000EEBB87FD45C020E030E0A901C301B201CD
:10D100000F94EEBB87FD3CC020E030E0A9016AAD82
:10D110007BAD8CAD9DAD0F94EEBB87FD31C020E0A3
:10D1200030E0A901C501B4010F943CB4882391F10A
:10D1300020E030E040E05FE3C501B4010F94A9AD09
:10D140006B017C012AAD3BAD4CAD5DADC301B201BD
:10D150000F94A9AD4B015C01A7019601C701B6016F
:10D160000F94A9AD2BED3FE049E450E40F94A9AD35
:10D170009B01AC01C501B4010F9491BA6B017C0114
:10D1800020E030E0A901C701B6010F94EEBB87FF94
:10D1900004C00BC0C12CD12C7601C092650FD09277
:10D1A000660FE092670FF092680FE9EBFDE584915E
:10D1B0008F01882339F00F94A14F0F5F1F4FF801A3
:10D1C0008491F7CFE0E3F7E084918F01882339F071
:10D1D0000F94A14F0F5F1F4FF8018491F7CF60911B
:10D1E000690F70916A0F80916B0F90916C0F42E004
:10D1F0000F9426508AE00F94A14FEAE2F7E0849161
:10D200008F01882339F00F94A14F0F5F1F4FF80152
:10D210008491F7CFC090650FD090660FE090670FB4
:10D22000F090680F20E030E0A901C701B6010F942B
:10D230003CB4882349F042E0C701B6010F94265060
:10D240008AE00F94A14F38C1E5E2F7E084918F01A5
:10D25000882311F40C94E2460F94A14F0F5F1F4FE7
:10D26000F8018491F5CF0F94A5AC0F9442B46B01F3
:10D270007C0120E030E0A9010F943CB487FD40C060
:10D2800020E030EA40E854E4C701B6010F94EEBB59
:10D29000181674F120E030E047E054E4C701B6010D
:10D2A0000F94EEBB87FD2FC020E030E04CE752E446
:10D2B000C701B6010F94A9AD20E030EA40E854E47C
:10D2C0000F9491BA0F9408BB162F802F0F94FAA1D8
:10D2D000612F802F0F94E9A10F5F043009F4ECC097
:10D2E000D5018D915D010F94B7AC8823A9F3BBCF15
:10D2F000C12CB0EADB2EB0E8EB2EB4E4FB2ED4CF89
:10D30000C12CD12C760120E030E04CE752E4C7017B
:10D31000B6010F94A9AD20E034EB40E954E4D0CF3E
:10D3200085E40F94B7AC882309F4C6C00F94AFAC62
:10D330000F9408BB4B015C018B016830710569F0EB
:10D340006031710551F06032710539F0603471055A
:10D3500021F06038710509F0AFC00F94038980E0B7
:10D3600091E07C0100901C0702C0F694E7940A94B7
:10D37000E2F7C4010E9493AD80931C0720911F0225
:10D3800040912302682F83E00E94B6AD80908C10FC
:10D3900090908D10A0908E10B0908F10E016F10636
:10D3A00070F5C801B7010F9441BE6B01E12CF12C5F
:10D3B000C701B6010F9440B49B01AC016091A0106D
:10D3C0007091A1108091A2109091A3100F94A9AD1B
:10D3D0006093A0107093A1108093A2109093A3105B
:10D3E000A5019401C701B6010F9458B960938C1040
:10D3F00070938D1080938E1090938F105DC0C70135
:10D40000B8010F9441BE6B01E12CF12CC701B601AC
:10D410000F9440B49B01AC016091A0107091A110D9
:10D420008091A2109091A3100F9491BA6093A010D4
:10D430007093A1108093A2109093A310C501B40122
:10D44000A70196010F9468BE20938C1030938D1025
:10D4500040938E1050938F102FC080912D108823F1
:10D4600029F085E40F94B7AC81119EC70F94AD6588
:10D4700023C083E40F94B7AC90912D10882329F03A
:10D480009923D1F00E9410A117C09111FBCF0E94E7
:10D490000FDB12C0809173159091741587579C4EC5
:10D4A0009F938F9385EC9DE09F938F930F9447B349
:10D4B0000F900F900F900F901092340D1092330D2B
:10D4C000B3C284E50F94B7AC882309F442C120911C
:10D4D000600D3091610DF90131968F01021B130B24
:10D4E0007F0181918032C9F38930B9F3082E000C95
:10D4F000990B0F94A8BEF7018083E091600DF09125
:10D50000610DE00FF11F808190ED980F953008F4C8
:10D5100061C08F3309F447C0883781F08336A9F1A1
:10D52000E5EBFDE084918F01882309F40EC10F948F
:10D53000A14F0F5F1F4FF8018491F6CF80912D10FE
:10D54000882309F471C240E050E060EC77E384E6A0
:10D5500092E10E9429DC80933A0290913B02891368
:10D5600007C080913A0D882319F08BE99DE064C0D3
:10D570000F94038980913A02805F0E94AC9E43E041
:10D5800061E081E00E94FB9A4FC280912D108823B8
:10D5900009F44AC20F9403890E94C29E80913A0204
:10D5A00080933B0261C080912D1040E050E08823C1
:10D5B00051F060EC77E384E692E10E9429DC8093ED
:10D5C0003A0211E01BC06AE472E183E592E10E9435
:10D5D00029DC0EC70F94AFAC0F9408BB862F609365
:10D5E0003A0290912D10992341F09091EE069923E3
:10D5F00021F0909153029111F9C610E00F94038924
:10D6000080913A0221E030E0082E01C0220F0A94F6
:10D61000EAF79091390D292B2093390D90912D1017
:10D62000992329F190913B0289130DC090913A0DF5
:10D63000992349F081E89DE09F938F930F9447B31E
:10D640000F900F90D8C6805F0E94AC9E43E061E0CF
:10D6500081E00E94FB9A0E94C29E80913A028093D0
:10D660003B02112309F4E0C10E943599DDC18823F2
:10D6700009F432C0E9EBFDE584918F01882339F08C
:10D680000F94A14F0F5F1F4FF8018491F7CFEFE781
:10D69000FDE084918F01882339F00F94A14F0F5F33
:10D6A0001F4FF8018491F7CF60913A0270E080E05B
:10D6B00090E00F9491658AE00F94A14FEFE1F5E0BF
:10D6C00084918F01882309F440C00F94A14F0F5F0C
:10D6D0001F4FF8018491F6CF86E40F94B7AC8823EE
:10D6E00099F00F94AFAC6B017C0120E030E0A90110
:10D6F0000F94EEBB181644F4C0925B02D0925C0209
:10D70000E0925D02F0925E02E9EBFDE584918F010B
:10D71000882339F00F94A14F0F5F1F4FF8018491B8
:10D72000F7CFEDE0F5E084918F01882339F00F9475
:10D73000A14F0F5F1F4FF8018491F7CF6091070D44
:10D7400070E080E090E00F9491658AE00F94A14F23
:10D750006BC184E40F94B7AC882309F404C10F941F
:10D76000AFAC0F9402BB6330710509F05DC186EC6C
:10D7700094E09F938F930F9447B381E40F94B7ACD9
:10D780000F900F908823B9F08091600D9091610DFA
:10D79000DC0111962C91283741F440E150E060E023
:10D7A00070E002960F94D1AF04C00F94AFAC0F9409
:10D7B00002BB7B0102C0E12CF12C83E40F94B7ACD7
:10D7C000882339F00F94AFAC0F9402BB262F872F1C
:10D7D00002C020E080E1BFE1FB22A22EB82EE1E0F2
:10D7E000AE16E0E1BE0618F0A12CA0E1BA2EC501EC
:10D7F0008E0D9F1D8130904128F080E090E15C010A
:10D80000AE18BF0888E50F94B7AC882309F470C040
:10D810002091600D3091610D2F5F3F4FAE014F5F42
:10D820005F4F6A01FA0100E010E0D9018C912F5F8F
:10D830003F4F882389F10031110561F18032A9F34E
:10D840008A3051F190ED980F9A3018F48295807FCC
:10D8500007C09FE9980F9630A8F48295807F805783
:10D860009D012E5F3F4F11969C9140ED490F4A302C
:10D8700010F4842B0BC04FE9490F463018F497552C
:10D88000892B04C011950195110906C081930F5F82
:10D890001F4FCBCF00E110E058010115110541F1F8
:10D8A000812C912CD6016D916D01C4018E0D9F1DAF
:10D8B0000F9447B9BFEF8B1A9B0A0815190591F70A
:10D8C000FF92EF921F930F9389E994E09F938F93B8
:10D8D0000F9447B36091CB197091CC198AE090E016
:10D8E0000F94C2B20F900F900F900F900F900F9067
:10D8F0006701E12CF12CA114B10409F495C08D2D20
:10D900000F9443AC8C2D0F9443AC6091CB19709164
:10D91000CC1980E290E00F94C2B210E1EFEFCE1A82
:10D92000DE0AEE0AFE0AC60101970F9417B9082F06
:10D930006091CB197091CC1980E290E00F94C2B243
:10D94000802F0F9443AC1150F1E0AF1AB10811F0E1
:10D950001111E4CF6091CB197091CC198AE090E05D
:10D960000F94C2B2C8CFE9EBFDE584918F01882303
:10D9700039F00F94A14F0F5F1F4FF8018491F7CF3B
:10D98000E9E3F5E084918F01882339F00F94A14FEA
:10D990000F5F1F4FF8018491F7CF0091731510911D
:10D9A000741507571C4ED8018D918D01882319F0ED
:10D9B0000F94A14FF8CFEAE7FDE084918F0188230F
:10D9C00009F4C3CE0F94A14F0F5F1F4FF80184914C
:10D9D000F6CFC090140FD090150FE090160FF09076
:10D9E000170F209158103091591040915A105091B2
:10D9F0005B10C701B6010F94A2B94B015C012DEC7D
:10DA00003CEC4CEC5DEB0F943CB487FD3AC02DEC44
:10DA10003CEC4CEC5DE3C501B4010F94EEBB181671
:10DA20000CF438C00F9476A881E090E09093260221
:10DA3000809325020F94D65360937F0F7093800FCD
:10DA40008093810F9093820FE0917315F09174157C
:10DA5000EA57FC4E8081813019F0863009F0CBC442
:10DA6000E2E4F7E184918F01882339F00F94A14F0C
:10DA70000F5F1F4FF8018491F7CF8AE00F94A14FF9
:10DA8000BAC4E091070DF0E0E85EF04F80818111AB
:10DA900092C409C0E091070DF0E0E85EF04F80818C
:10DAA000882309F4BFCFC0925810D0925910E09249
:10DAB0005A10F0925B1088E590E10E9440D6E09108
:10DAC000070DF0E0E85EF04F908181E089270F9428
:10DAD000EBA291C420E030E040E85FE36091581091
:10DAE0007091591080915A1090915B100F94A3B9C6
:10DAF000609358107093591080935A1090935B1054
:10DB0000E0905410F090551000915610109157105D
:10DB1000209150103091511040915210509153105B
:10DB200060914C1070914D1080914E1090914F105B
:10DB3000E7E0FDE0FF93EF93812C912CE8ECAE2E13
:10DB4000E3E4BE2EF8E5CF2EF0E1DF2E0F94EF2CAC
:10DB50000F900F900C94414282E090E09093260247
:10DB60008093250210926B0E10926A0E0C948D46D3
:10DB70000F94A5ACAB01BC014093511950935219BD
:10DB800060935319709354198CE998E10E949DEEAB
:10DB900093CC0F94AFAC0F9402BB8B010C94594AF9
:10DBA0000F94038988E50F94B7AC882319F0179A6E
:10DBB0001092080D89E50F94B7AC882319F0169AD6
:10DBC0001092090D8AE50F94B7AC85E40F94B7ACB9
:10DBD000882311F40C94B04F149A0C94B04F1A820D
:10DBE00019824AE050E0BE016F5F7F4FC7010F947A
:10DBF000D1AF78A36F8F89819A818816990609F031
:10DC00005BCC4AE050E0BE016F5F7F4FC6010F94CE
:10DC1000D1AF7AA369A389819A816816790609F040
:10DC20004BCC4AE050E0BE016F5F7F4FC5010F94BF
:10DC3000D1AF7CA36BA389819A810817190709F0DA
:10DC40003BCC8FE790E09EA38DA35801EFEFAE1A77
:10DC5000BE0AD8018C918D3211F575016701BFEFB5
:10DC6000CB1ADB0AF70180810F94F925382E811138
:10DC700002C07601F3CFEA18FB08DE2CC701992712
:10DC80008330910569F543E050E061EE7CE5C50124
:10DC90000F941AB2892B09F042C01EA21DA2332094
:10DCA00009F40ACCCE0101960F947579882309F402
:10DCB00003CCFE017F96DE011196AE01495D5F4FF8
:10DCC000219131918D919D918217930708F44CC059
:10DCD0002817390708F4F0CB4E175F0789F7ECCB0C
:10DCE0008530910571F445E050E06BED7CE5C501B0
:10DCF0000F941AB2892B99F481E090E09EA38DA332
:10DD0000CECF049761F444E050E066ED7CE5C501B8
:10DD10000F941AB2892B19F482E090E0EFCF8EEFC6
:10DD20008E0D823008F0C8CBD80111968C911197D6
:10DD30008F7D823509F0C0CB12968C918F7D833414
:10DD400009F0BACBB2E0DB1203C083E090E0D6CF9B
:10DD5000F801838190ED980F9A3008F0ADCB082E32
:10DD6000000C990B8E97CACF8CED91E10E94FBFBC2
:10DD700044EC5CE062E080E00F943916D2011D9122
:10DD80002D01812F0F94F925811108C06FEC76E0E9
:10DD9000812F110F990B0F94C2B2F0CF4CEC51E1CF
:10DDA00063E080E00F94391680910A0790910B0789
:10DDB000029728F48091020184608093020182E33B
:10DDC00090E00F94C1440F94EE7A84EF91E00F94A9
:10DDD000C14480910A0790910B07029728F4809123
:10DDE000020184608093020182E390E00F94C144B9
:10DDF0000F94EE7A80E090E00F942FA281E00F94D0
:10DE00004E160F94441680E00F94BE0E55CBAB9681
:10DE1000CCACDDACEEACFFACAB97C80ED91EEA1EA5
:10DE2000FB1EAB962CAD3DAD4EAD5FADAB97281B49
:10DE3000390B4A0B5B0B2A966CAD7DAD8EAD9FAD59
:10DE40002A970F9458B9A70196010F9468BEDA017A
:10DE5000C901840D951DA61DB71D84319105A1052D
:10DE6000B105E4F02C013D018C3E9105A105B10501
:10DE70002CF06BEE462E512C612C712C40E8441690
:10DE8000510461047104DCF05EEF852E912CA12C0D
:10DE9000B12C84189508A608B7080AC034E1432EAF
:10DEA000512C612C712C44E1842E912CA12CB12C8D
:10DEB0002A968CAE9DAEAEAEBFAE2A9706C02A960D
:10DEC0004CAE5DAE6EAE7FAE2A97E1EAFCE0849187
:10DED0008F01882339F00F94A14F0F5F1F4FF80176
:10DEE0008491F7CFC301B2010F949165ECE9FCE096
:10DEF00084918F01882339F00F94A14F0F5F1F4F3A
:10DF0000F8018491F7CF2A966CAD7DAD8EAD9FADB3
:10DF10002A970F949165E5E9FCE084918F018823AD
:10DF200039F00F94A14F0F5F1F4FF8018491F7CF85
:10DF300042E06D966FAD6D976E967FAD6E976F9662
:10DF40008FAD6F97A0969FADA0970F942650EEE8E7
:10DF5000FCE084918F01882339F00F94A14F0F5F6B
:10DF60001F4FF8018491F7CF42E0A1966FADA197C2
:10DF7000A2967FADA297A3968FADA397A4969FADCF
:10DF8000A4970F9426508AE00F94A14F80914E0DD4
:10DF900090914F0D039714F40C941A5B2A966CAD74
:10DFA0007DAD8EAD9FAD2A970F9442B420E030E056
:10DFB00040E850E40F94A9AD4B015C016D962FAD84
:10DFC0006D976E963FAD6E976F964FAD6F97A0961B
:10DFD0005FADA097A1966FADA197A2967FADA297D6
:10DFE000A3968FADA397A4969FADA4970F94A2B9C3
:10DFF00020ED3FE049E450E40F94A9AD20E030E08B
:10E0000040E05FE30F94A9AD9B01AC01C501B401F1
:10E010000F9491BA4B015C01C701B6010F9442B451
:10E0200020E030E04AE754E40F9491BA6B017C01A0
:10E03000E8E8FCE084918F01882339F00F94A14F28
:10E040000F5F1F4FF8018491F7CF42E0C501B40183
:10E050000F942650E2E8FCE084918F01882339F088
:10E060000F94A14F0F5F1F4FF8018491F7CF42E04B
:10E07000C701B6010F9426508AE00F94A14F2AE9F8
:10E0800039E949E15FE3C501B4010F94A9AD4B0142
:10E090005C016093EF0E7093F00E8093F10E9093FD
:10E0A000F20E9B01AC010F94A3B9A70196010F9446
:10E0B00091BA6093EB0E7093EC0E8093ED0E9093FB
:10E0C000EE0EA5019401C701B6010F94A9AD20E0A1
:10E0D00030E040E05EE30F94A9AD6093E70E7093EB
:10E0E000E80E8093E90E9093EA0EE4E7FCE0849159
:10E0F0008F01882339F00F94A14F0F5F1F4FF80154
:10E100008491F7CF8AE00F94A14FEEE6FCE0849172
:10E110008F01882339F00F94A14F0F5F1F4FF80133
:10E120008491F7CF6091EF0E7091F00E8091F10E17
:10E130009091F20E42E00F9426508AE00F94A14F86
:10E14000E8E6FCE084918F01882339F00F94A14F19
:10E150000F5F1F4FF8018491F7CF6091EB0E709124
:10E16000EC0E8091ED0E9091EE0E42E00F94265051
:10E170008AE00F94A14FE2E6FCE084918F018823AE
:10E1800039F00F94A14F0F5F1F4FF8018491F7CF23
:10E190006091E70E7091E80E8091E90E9091EA0E81
:10E1A00042E00F9426508AE00F94A14F0C941A5B22
:10E1B0008093B10F0C94355BE8961FAEE8970C94F2
:10E1C0005A5B84E690E00F94C1440C94D25C312CED
:10E1D0000C94F060E12CF12C80910101846080931B
:10E1E0000101E114F10409F04EC080910A079091F9
:10E1F0000B070097F1F10197D1F19FEFE91AF90AA6
:10E20000A1E0DA1609F452C0DA1608F04AC084E038
:10E2100090E00F94C1440F94D653950184010054AB
:10E22000184D264F3F4F061717072807390710F0DC
:10E230000C94146288E690E10E94FBFB1F8E18A2EA
:10E2400019A21AA2CE014F960F94257B0F94038931
:10E25000149ADD24D3940F94378281E00F946140A7
:10E26000F4EFEF16F1E0FF0609F0B6CFB3CFCC2004
:10E2700021F29FB7F894809102018460809302019B
:10E280009FBFC12CBACF84E1E816F10409F0B5CFE5
:10E290009FB7F894809102018B7F809302019FBF0A
:10E2A000ACCFB2E0DB16E1F00C94146284E090E0B5
:10E2B0000F94C1440F948F0F882369F2E091070DEA
:10E2C000F0E0EE0FFF1FEB58FA4E64962EAD3FAD17
:10E2D0006497318320830E9426C502E0D02EBBCFF5
:10E2E0000091070D10E0F801EE0FFF1FEB58FA4EFA
:10E2F00060817181072E000C880B990B0F9442B43A
:10E30000000F111F000F111FF801E55EF04F208173
:10E310003181428153810F94A2B92B013C0120E04D
:10E3200030E0A9010F94EEBB18165CF420E030E059
:10E3300040E85FE3C301B2010F943CB487FF16C00D
:10E340000AC020E030E040E85FEBC301B2010F9467
:10E35000EEBB18165CF483E990E10E94FBFB0F947E
:10E36000D6534B015C01D12C0C94176264E081E020
:10E370000F949711E091070D34E0E39FF001112411
:10E38000E55EF04F80819181A281B3818F8F98A348
:10E39000A9A3BAA3CE014F960E948AB60F94341057
:10E3A000F4E1EF2EF12C57CF0F94AFAC0F9408BBD4
:10E3B00060933A025BC82DEC3CEC4CEC5DE3C5018C
:10E3C000B4010F94EEBB18160CF46DCB2BCBA5014A
:10E3D0009401F101662D772D8F2F922D0F943CB46F
:10E3E000181614F40C945B3B0C946B3B0F944CACE0
:10E3F00080933A0202C9C958DF4F0FB6F894DEBFC6
:10E400000FBECDBFDF91CF911F910F91FF90EF9085
:10E41000DF90CF90BF90AF909F908F907F906F9044
:10E420005F904F903F902F9008952F923F924F9280
:10E430005F926F927F928F929F92AF92BF92CF9294
:10E44000DF92EF92FF920F931F93CF93DF93CDB79D
:10E45000DEB7C95CD1090FB6F894DEBF0FBECDBFE1
:10E46000782E81E00F94ED66711025C010920C0D8E
:10E4700010920B0D19821A821B821C82CE0101960A
:10E480000F94257B61E080EC9FE00F9429B960E058
:10E490008FEB9FE00F9429B960E08EEB9FE00F9423
:10E4A00029B960E08DEB9FE00F9429B960E08CEB17
:10E4B0009FE00F9429B980E00F944E160F9459767F
:10E4C0000F94260C1092060D1092050D83E0E8E0E3
:10E4D000FDE0DF011D928A95E9F781E00F94535E1C
:10E4E000C855DF4F99838883C85AD0408FEB9BE192
:10E4F0000E94FBFB0F94825E40E050E061E080E010
:10E5000090E00F942E6740E050E061E081E090E001
:10E510000F942E67E0905410F09055100091561013
:10E52000109157102091501030915110409152107D
:10E530005091531060914C1070914D1080914E107D
:10E5400090914F100F94FB710E947BD51092240282
:10E5500020E030E040EA50E460914C1070914D10A2
:10E5600080914E1090914F100F94A3B91B012C0174
:10E5700060934C1070934D1080934E1090934F10F9
:10E5800020E030E040EA50E460915010709151106A
:10E5900080915210909153100F94A3B99B01AC013C
:10E5A00060935010709351108093521090935310B9
:10E5B000E0905410F09055100091561010915710A3
:10E5C00087E09DE09F938F93812C912CB0EAAB2E36
:10E5D000B1E4BB2E88E5C82E80E1D82EC201B1017E
:10E5E0000F94EF2C0F9403890F948C5E0F900F9073
:10E5F000882311F40C94298685E89BE10E94ACFCE9
:10E60000772089F085E59BE10E94FBFB63E080E0D9
:10E610000F94971161E070E080E090E00F94191082
:10E620008FE49BE110C08FE29BE10E94FBFB62E064
:10E6300080E00F94971161E070E080E090E00F942B
:10E64000191089E29BE10F94BE100F94236771109B
:10E650002EC084E090E0909326028093250240E053
:10E6600060E08EE09BE10E9408FC882321F086EEAA
:10E670009AE10E94ACFC80E59AE10E94ACFC82E049
:10E6800090E090932602809325028FE29BE10E9406
:10E69000FBFB62E080E00F94971161E070E080E0A6
:10E6A00090E00F94191089E29BE10F94BE106090E6
:10E6B00024021092240220E030E040E85FE3609101
:10E6C00054107091551080915610909157100F94DE
:10E6D000A2B97B018C016093541070935510809304
:10E6E0005610909357102091501030915110409136
:10E6F00052105091531060914C1070914D108091B8
:10E700004E1090914F10E7E04E2EEDE05E2E5F929E
:10E710004F92812C912CF0EAAF2EF1E4BF2EA8E5A8
:10E72000CA2EA0E1DA2E0F94EF2C0F94038980E01B
:10E7300090E0A0EAB0E48093541090935510A09319
:10E740005610B093571081E08093240284E00E9419
:10E750008FAFE0905410F09055100091561010912A
:10E7600057102091501030915110409152105091FB
:10E77000531060914C1070914D1080914E109091FB
:10E780004F105F924F920F94EF2C0F9403890E94C9
:10E79000F8AE6092240282E00F94F0880F900F9000
:10E7A0000F900F9020E030E040EA50E40F943CB42A
:10E7B00081110C9425867720E9F0C855DF4F8881B8
:10E7C0009981C85AD0400F94325E0F94150E0F9461
:10E7D000280A0F94C511882311F40C94D5850F9441
:10E7E0008D65803F11F00C94218681E00F942E629C
:10E7F0000C9421868AEF0F942E6260E070E088EF1F
:10E800009FE00F9443B90F94236784ECE3E8F5E1AC
:10E81000DF011D928A95E9F7E6E6FEE184918F011A
:10E82000882339F00F94A14F0F5F1F4FF801849197
:10E83000F7CF61E070E080E090E00F9491650F9475
:10E840009F50BE016F5A7F4F8FE29BE10E94E9FB10
:10E8500062968FAD6297843020F083E062968FAF2E
:10E86000629780E090E0A0EAB0E480935410909327
:10E870005510A0935610B093571026E43EE1C657AA
:10E88000DF4F39832883CA58D04082E895E1CE57BC
:10E89000DF4F99838883C258D040A0969FAF8EAF38
:10E8A000A097A8963FAF2EAFA89781E090E0A0E098
:10E8B000B0E0AE968CAF9DAFAEAFBFAFAE970F944A
:10E8C000236762966FAD629780E00F949711AE96C2
:10E8D0006CAD7DAD8EAD9FADAE970F94191089E2F2
:10E8E0009BE10F94BE1065E575E585E591E40F9415
:10E8F000BA09A896EEADFFADA89785919591A5911F
:10E90000B49180934C1090934D10A0934E10B093FF
:10E910004F10A896EEADFFADA897349685919591CE
:10E92000A591B4918093501090935110A0935210E0
:10E93000B093531060E070E088E492E40F94BA0959
:10E9400000914410109145102091461030914710CD
:10E9500040914010509141106091421070914310CD
:10E9600080913C1090913D10A0913E10B0913F10CD
:10E970003F932F931F930F937F936F935F934F93C7
:10E98000BF93AF939F938F9382ED9DE19F938F935E
:10E990000F9447B30F94038940913C1050913D1060
:10E9A00060913E1070913F10809140109091411005
:10E9B000A0914210B0914310C0904410D0904510E7
:10E9C000E0904610F090471021E00FB6F894DEBFBB
:10E9D0000FBECDBF413157420CF420E08131974248
:10E9E00014F00C942B86822F90E0880F991FFC0165
:10E9F000E653F24EA590B490FC01EE53F24E859092
:10EA00009490DF92CF929F928F92BF92AF921F927B
:10EA10002F9389EA9DE19F938F930F9447B389ECDD
:10EA20009BE19F938F930F9447B30F945D4980911F
:10EA300070008B7F80937000EF9880916F008D7FC6
:10EA400080936F000FB6F894A8958091600088615C
:10EA500080936000109260000FBE1092040D10921F
:10EA6000030D80EA91E09093020D8093010D88E4FC
:10EA700091E09093000D8093FF0C00E028EC30E0D3
:10EA8000A601B401C5010F945C22009144101091BD
:10EA90004510209146103091471040914010509100
:10EAA0004110609142107091431080913C10909100
:10EAB0003D10A0913E10B0913F103F932F931F93B4
:10EAC0000F937F936F935F934F93BF93AF939F93F6
:10EAD0008F9389E69CE19F938F930F9447B3809126
:10EAE0003C1090913D10A0913E10B0913F10782EB7
:10EAF000692E8091401090914110A0914210B091E8
:10EB00004310582E492EC0904410D0904510E090EC
:10EB10004610F09047100FB6F894DEBF0FBECDBF81
:10EB200040EE242E4BE1342E95E0C91697EFD9061E
:10EB30000CF46EC01A8219821F921F92A3E0AF9349
:10EB4000B4E8BF931F92E4E6EF93DF92CF924F9227
:10EB50005F926F927F923F922F920F9447B30FB6BE
:10EB6000F894DEBF0FBECDBF89819A81803D92406F
:10EB700030F089819A81803A954050F512C0CE01DB
:10EB800001967C0100E010E024E833E0A601652D49
:10EB9000742D872D962D0F94257881110C94308635
:10EBA000E8CFDE0111967D0100E010E02CE73CEF9C
:10EBB000A60144565109652D742D872D962D0F946D
:10EBC0002578882329F089819A8180539D4F1CC024
:10EBD00089819A818037984008F04AC0FE013196B9
:10EBE0007F0104EB10E024E833E0A601485C510902
:10EBF000652D742D872D962D0F9425788823C1F1CE
:10EC000089819A8180569A4F9A8389830C943086A1
:10EC100000914410109145102091461030914710FA
:10EC200040914010509141106091421070914310FA
:10EC300080913C1090913D10A0913E10B0913F10FA
:10EC40003F932F931F930F937F936F935F934F93F4
:10EC5000BF93AF939F938F9388E19CE19F938F9392
:10EC60000F9447B30FB6F894DEBF0FBECDBFD8C325
:10EC700089819A8180349B40A0F49E012F5F3F4F91
:10EC8000790104EB10E02CE73CEFA6014C52514017
:10EC9000652D742D872D962D0F94257881110C9458
:10ECA000178780E0E981FA81882311F40C94338678
:10ECB00080913C1090913D10A0913E10B0913F107A
:10ECC000409140105091411060914210709143105A
:10ECD000009144101091451020914610309147103A
:10ECE000FF93EF931F930F935F934F939F938F9394
:10ECF00085E49CE19F938F930F9447B34091441018
:10ED000050914510609146107091471000E028EC3A
:10ED100030E0B401C5010F945C2285E08F9380E759
:10ED20008F9389E79DE19F938F930F9447B384E07E
:10ED30008F9388E38F9387E69DE19F938F930F9442
:10ED400047B380913C1090913D10A0913E10B0913E
:10ED50003F106A968CAF9DAFAEAFBFAF6A97689613
:10ED6000CEACDFAC68978091401090914110A0919B
:10ED70004210B0914310E2968CAF9DAFAEAFBFAFE3
:10ED8000E2978091441090914510A0914610B09167
:10ED900047106E968CAF9DAFAEAFBFAF6E971C01A4
:10EDA00098E4291A310889E08F9380E68F933F9287
:10EDB0002F92E096AFADE097AF93AF96BFADAF9710
:10EDC000BF936896EFAD6897EF936796FFAD67972F
:10EDD000FF9382E99CE19F938F930F9447B34091F7
:10EDE00044105091451060914610709147107A017F
:10EDF00020E931E0E0966EAD7FADE09768968EAD8C
:10EE00009FAD68970F945C22E0962EAD3FADE097E2
:10EE10003450EC963FAF2EAFEC970FB6F894DEBFB0
:10EE20000FBECDBF812C912CD601B450E896BFAF58
:10EE3000AEAFE897F601FC5FC258DF4FF983E88375
:10EE4000CE57D040382D3170A3963FAFA39780FCAA
:10EE500002C00C943986EF968FADEF97C158DF4F03
:10EE60009881CF57D04000E020E931E0A701EC962F
:10EE70006EAD7FADEC970F945C22C0904010D090A7
:10EE80004110E0904210F090431080913C1090911E
:10EE90003D10A0913E10B0913F1001E028EC30E011
:10EEA000A101B6010F945C22C0904010D090411097
:10EEB000E0904210F090431080913C1090913D10F2
:10EEC000A0913E10B0913F100FEF28EC30E040E6EB
:10EED00059E0B6010F945C22809144109091451046
:10EEE000A0914610B09147107C01A3966FADA397F7
:10EEF00080910B01662311F40C944186816080930C
:10EF00000B010000840125E0000F111F2A95E1F795
:10EF1000A3968FADA397882311F40C94448690ECAC
:10EF2000492E55245A94652C752CC12CD12C90E473
:10EF3000E3969FAFE397A12CB12C93B1A70142199F
:10EF40005309292F207194FF02C00C944B8688EE40
:10EF50009FEF840F951F97FD02C00C944F8680E0B1
:10EF600090E0A80EB91E80910B0121110C945986D6
:10EF7000846080930B01000021110C945C862E1498
:10EF80003F0434F484E00F94DA54A1E0EA1AF10863
:10EF900081E00F94DA548BE599E00197F1F7E3965D
:10EFA000FFADE397F150E396FFAFE397F111C5CFC3
:10EFB000B6E0B694A794BA95E1F7A3962FADA397C0
:10EFC000222311F40C946B868FE190E08C199D093B
:10EFD000800F911FFC01E157F84FA08280913C10F7
:10EFE00090913D10A0913E10B0913F10840D951D61
:10EFF000A61DB71D80933C1090933D10A0933E102A
:10F00000B0933F10C7010F2C000CAA0BBB0B8093D1
:10F01000441090934510A0934610B09347103FEFD3
:10F02000C31AD30A60E2C616D10409F080CF015793
:10F03000184FF0E2BF2EADE8CA2EACE1DA2ED801AF
:10F040008D918D011F928F93DF92CF920F9447B3D2
:10F05000BA940F900F900F900F90B110F0CF8BE8F3
:10F060009CE19F938F930F9447B3BFEF8B1A9B0A3A
:10F07000EC96EEADFFADEC97E05CFF4FEC96FFAF8A
:10F08000EEAFEC970F900F90F0E28F16910409F01D
:10F09000D9CEEFE8AE2EEBE0BE2E8FEA9BE0F50175
:10F0A000119211928E179F07D9F780E090E0DC0152
:10F0B00075E0AA0FBB1F7A95E1F7A157B84F40E260
:10F0C000ED91F0E054E0F595E7955A95E1F7EE0FF4
:10F0D000FF1FE157F44F208131812F5F3F4F318374
:10F0E0002083415069F701968032910501F72FE89E
:10F0F000C22E2BE0D22E00E010E03AECE32E3CE1F1
:10F10000F32ED6018C9111969C91B2E0CB0ED11CBE
:10F110009F938F931F930F93FF92EF920F9447B398
:10F120000F5F1F4F0F900F900F900F900F900F9049
:10F130000031110531F78091910B9091920BE1E92B
:10F14000FBE031E021E0419151918417950710F4E3
:10F15000322FCA012F5F2031B1F7032F1F923F9347
:10F160009F938F9381EF9CE19F938F930F9447B36D
:10F17000EDEAFBE00F900F900F900F900F900F9023
:10F180008EE0329122912A30310510F40C946E8673
:10F190008295807F20918F0B3091900B20373340E8
:10F1A00010F00C947586000F000F000F182F101B25
:10F1B0001F921F931F928F931F920F938AED9CE1D2
:10F1C0009F938F930F9447B39FE8492E97E0592E52
:10F1D0000FB6F894DEBF0FBECDBFF201202F30E096
:10F1E000012F10E0808190E02817390710F00C946F
:10F1F0007886821B930B982F80E0B8010F9441BE54
:10F200006F3F710519F010F06FEF70E06193AE166B
:10F21000BF0641F700E010E0B5EDAB2EBCE1BB2E20
:10F2200083EDC82E8CE1D82EC801A5E0880F991F68
:10F23000AA95E1F7DC01A157B84F7D01912CF701A8
:10F2400081917F011F928F93BF92AF920F9447B32A
:10F2500093940F900F900F900F90F0E29F12EFCFCA
:10F26000DF92CF920F9447B30F5F1F4F0F900F9015
:10F2700000321105C9F68FE49DE127EE3BE0AFECCB
:10F28000BBE0FC01459154914D935D9302962A1782
:10F290003B07B9F7612C712CE12CF12C10E000E058
:10F2A000A12C40E050E0EB964FAFEB972FEC3BE00A
:10F2B000E8963FAF2EAFE897A0E0B0E080E090E0A6
:10F2C000B12C4A01860C971C20E030E014012A0E74
:10F2D0003B1E6EEF6B0DE3966FAFE397B1100C948E
:10F2E0007C866EEF620F683010F40C9483862F5F7B
:10F2F0003F4F2C30310591F7B3949096E896EEADE0
:10F30000FFADE8973296E896FFAFEEAFE897FCE0E6
:10F31000BF12DACFE816F9062CF47C010A2DEB9621
:10F320001FADEB974F5F5F4F4431510509F0BBCFE5
:10F33000A39420E2620E711C34E1A312B2CFFF92BB
:10F34000EF921F920F931F921F9385E09DE19F9371
:10F350008F930F9447B30FB6F894DEBF0FBECDBFA7
:10F3600093E4E916F10414F40C94B9861F920F93F8
:10F370001F921F9386E39DE19F938F930F9447B352
:10F380001A5FE12EF12CA0E1EA1AF108E6E0EE0C9A
:10F39000FF1CEA95E1F76896EEADFFAD6897EE0EBB
:10F3A000FF1E0A5FC02ED12CF0E1CF1AD108F6E083
:10F3B000CC0CDD1CFA95E1F7E0962EAD3FADE09761
:10F3C000C20ED31E6C963FAD6C973F936B966FAD9C
:10F3D0006B976F93DF92CF92FF92EF9285E29DE160
:10F3E0009F938F930F9447B300E028EC30E06C9626
:10F3F0004EAD5FAD6C97B601C7010F945C220FB69E
:10F40000F894DEBF0FBECDBF81E0D2011D922D0169
:10F41000BFEF4B16BCE05B06C1F781110C94BC86B4
:10F4200010E082E99DE19F938F930F9447B30F946F
:10F430002D3B80917000846080937000EF9A8091E2
:10F440006F00826080936F0098E288E10FB6F894B5
:10F45000A895809360000FBE909360001092040DF9
:10F460001092030D1092020D1092010D1092000DDA
:10F470001092FF0C0F900F90112311F40C945C85E7
:10F4800020E030E0A901A096EEADFFADA09761812C
:10F490007281838194810F94A9AD20914C10309199
:10F4A0004D1040914E1050914F100F94A3B9A0965B
:10F4B000AEADBFADA09711966D937D938D939C9348
:10F4C0001497C0905010D0905110E0905210F090CE
:10F4D000531020E030E0A90115966D917D918D913A
:10F4E0009C9118970F94A9ADA70196010F94A3B909
:10F4F000A096EEADFFADA097658376838783908756
:10F5000020E030E040E850ECC701B6010F943CB475
:10F5100087FF0CC080E090E0A0E8B0EC8093501032
:10F5200090935110A0935210B093531020E030E00C
:10F5300040E450E460915410709155108091561041
:10F54000909157100F94A3B9609354107093551075
:10F550008093561090935710AE968CAD9DADAEAD86
:10F56000BFADAE970196A11DB11DAE968CAF9DAFFC
:10F57000AEAFBFAFAE97A896AEADBFADA897189689
:10F58000A896BFAFAEAFA897A096EEADFFADA0977F
:10F590003896A096FFAFEEAFA097AE968CAD9DAD1E
:10F5A000AEADBFADAE970597A105B10509F087C90E
:10F5B00080E090E00F94C14420E030E040E950EC5E
:10F5C00060918715709188158091891590918A15A1
:10F5D0000F943CB487FF43C0E5E4FEE184918F01C2
:10F5E000882339F00F94A14F0F5F1F4FF8018491CA
:10F5F000F7CF8AE00F94A14FE3E1FEE184918F0100
:10F60000882339F00F94A14F0F5F1F4FF8018491A9
:10F61000F7CF609187157091881580918915909129
:10F620008A1542E00F942650EFE0FEE184918F01AD
:10F63000882339F00F94A14F0F5F1F4FF801849179
:10F64000F7CF42E060E070E080E990EC0F94265044
:10F650000F949F50F2E0AF96FFAFAF9703C0AF9605
:10F660001FAEAF971092B3151092B4151092B51546
:10F670001092B6151092B7151092B8151092B915D0
:10F680001092BA1524E6EB962FAFEB97A2961CAE1C
:10F690001DAE1EAE1FAEA2976A961CAE1DAE1EAE6C
:10F6A0001FAE6A97CE01019664969FAF8EAF6497A6
:10F6B000DE01AF5BBF4F6696BFAFAEAF66976A968F
:10F6C0006CAD7DAD8EAD9FAD6A970F948EBAAA9644
:10F6D0006CAF7DAF8EAF9FAFAA976A966CAD7DADD4
:10F6E0008EAD9FAD6A970F941CBDC457DF4F6883E2
:10F6F00079838A839B83CC58D040A2966CAD7DAD34
:10F700008EAD9FADA2970F948EBAC057DF4F68831E
:10F7100079838A839B83C059D040A2966CAD7DAD1E
:10F720008EAD9FADA2970F941CBDCC56DF4F688362
:10F7300079838A839B83C459D0406496EEADFFAD34
:10F74000649720E411922A95E9F76696AEADBFADB5
:10F750006697E0E11D92EA95E9F780E090E00F946A
:10F76000C1448091B3159091B415A091B515B09195
:10F77000B615C655DF4F88839983AA83BB83CA5ABF
:10F78000D0408091B7159091B815A091B915B0915E
:10F79000BA15C255DF4F88839983AA83BB83CE5A9B
:10F7A000D040DE01AF5BBF4FC856DF4FB983A8839F
:10F7B000C859D040FE013196AC96FFAFEEAFAC9782
:10F7C00000E0CC56DF4F88819981AA81BB81C45962
:10F7D000D040B058E6968CAF9DAFAEAFBFAFE697C6
:10F7E000C057DF4F88819981AA81BB81C059D04021
:10F7F000B058EA968CAF9DAFAEAFBFAFEA97C45793
:10F80000DF4F88819981AA81BB81CC58D040B05804
:10F81000C258DF4F88839983AA83BB83CE57D040D9
:10F82000AC962EAC3FACAC9710E062E8462E65E19A
:10F83000562E74E0772EC12CD12C7601013011F4B4
:10F840000C943F87113011F40C944B87002311F175
:10F85000023081F4D20111962D913D914D915C9130
:10F860001497C258DF4F688179818A819B81CE5776
:10F87000D0400BC0F2012581368147815085EA9640
:10F880006CAD7DAD8EAD9FADEA970F94A9AD4B01E8
:10F890005C0106C0812C912C50E8A52E5FE3B52EAB
:10F8A000112301F1123081F4D20111962D913D9175
:10F8B0004D915C911497C258DF4F688179818A819C
:10F8C0009B81CE57D0400BC0F20125813681478104
:10F8D0005085EA966CAD7DAD8EAD9FADEA970F94E5
:10F8E000A9AD04C060E070E080E89FE39B01AC013B
:10F8F000C501B4010F94A9AD9B01AC01C701B601CC
:10F900000F94A3B96B017C010023E1F11123D1F124
:10F91000023011F00C941F87D20111962D913D9168
:10F920004D915C911497AA966CAD7DAD8EAD9FAD57
:10F93000AA970F94A9AD4B015C01113011F40C94FE
:10F940003987123011F00C942C87D20111962D9129
:10F950003D914D915C911497AA966CAD7DAD8EADA5
:10F960009FADAA970F94A9AD9B01AC01C501B4014D
:10F970000F94A9AD9B01AC01C701B6010F94A3B9C7
:10F980006B017C017A94F8E04F0E511C711056CF38
:10F99000D101CD92DD92ED92FD921D011F5F1430D9
:10F9A00009F043CF32E8232E35E1332EE6E4FEE1C1
:10F9B0006C96FFAFEEAF6C97CA57DF4F1882C658F0
:10F9C000D040C456DF4F1882CC59D040C056DF4FCC
:10F9D0001882C05AD04010E0002321F1013049F1D3
:10F9E000023081F4D10111962D913D914D915C91A0
:10F9F0001497C258DF4F688179818A819B81CE57E5
:10FA0000D0400BC0F1012581368147815085EA96AF
:10FA10006CAD7DAD8EAD9FADEA970F94A9AD4B0156
:10FA20005C010AC0812C912C20E8A22E2FE3B22E7B
:10FA300003C0812C912C5401D10111964D905D9001
:10FA40006D907C901497A3019201AA966CAD7DAD48
:10FA50008EAD9FADAA970F94A9AD6B017C01D1012A
:10FA600015968D919D910D90BC91A02DA6968CAF71
:10FA70009DAFAEAFBFAFA6976C96EEADFFAD6C97E6
:10FA800085919591A591B491CC55DF4F8883998349
:10FA9000AA83BB83C45AD040A6962CAD3DAD4EADD3
:10FAA0005FADA697CC56DF4F688179818A819B81B3
:10FAB000C459D0400F94A9AD9B01AC01C701B60158
:10FAC0000F94A2B9C655DF4F288139814A815B81E5
:10FAD000CA5AD0400F94A3B9CC55DF4F2881398141
:10FAE0004A815B81C45AD0400F94A2B9A501940108
:10FAF0000F94A9ADCA57DF4F2881C658D040C456CD
:10FB0000DF4F3881CC59D040C056DF4F4881C05AB2
:10FB1000D040512F0F94A3B9CA57DF4F6883798320
:10FB20008A839B83C658D0400023A9F00130B9F0E6
:10FB30000230D9F0A6962CAD3DAD4EAD5FADA69787
:10FB4000E6966CAD7DAD8EAD9FADE6970F94A9ADF9
:10FB50006B017C010AC0C12CD12C760106C0C12CDE
:10FB6000D12C90E8E92E9FE3F92E6C96EEADFFAD17
:10FB70006C97349685909590A590B490A3019201CE
:10FB8000C457DF4F688179818A819B81CC58D040EE
:10FB90000F94A9AD2B013C01A6962CAD3DAD4EAD09
:10FBA0005FADA697C057DF4F688179818A819B81BD
:10FBB000C059D0400F94A9AD9B01AC01C301B20163
:10FBC0000F94A3B9C255DF4F288139814A815B81E7
:10FBD000CE5AD0400F94A3B9A50194010F94A2B9B5
:10FBE000A70196010F94A9ADCA57DF4F288139812B
:10FBF0004A815B81C658D0400F94A3B9CA57DF4FE2
:10FC00006883C658D040C456DF4F7883CC59D04063
:10FC1000C056DF4F8883C05AD040192F6C96AEADC6
:10FC2000BFAD6C9718966C96BFAFAEAF6C97B8E04F
:10FC30002B0E311CE2EA2E16E5E13E0609F0CCCE91
:10FC4000DC01CB01B058C856DF4FE881F981C859B3
:10FC5000D04081939193A193B193C856DF4FF9831C
:10FC6000E883C859D0400F5FAC962EAD3FADAC973E
:10FC7000205F3F4FAC963FAF2EAFAC97043009F0FA
:10FC8000CFCD25968CAD9DADAEADBFAD2597AA96D7
:10FC90008CAF9DAFAEAFBFAFAA978D819E81AF8174
:10FCA000B885AE968CAF9DAFAEAFBFAFAE9789852E
:10FCB0009A85AB85BC85A6968CAF9DAFAEAFBFAF26
:10FCC000A6978D859E85AF85B889E6968CAF9DAF4A
:10FCD000AEAFBFAFE69789819A81AB81BC81EA96CE
:10FCE0008CAF9DAFAEAFBFAFEA9729968CAD9DADFF
:10FCF000AEADBFAD2997C258DF4F88839983AA83E1
:10FD0000BB83CE57D04089899A89AB89BC89C457B7
:10FD1000DF4F88839983AA83BB83CC58D040898DD9
:10FD20009A8DAB8DBC8DC057DF4F88839983AA8392
:10FD3000BB83C059D0408D8D9E8DAF8DB8A1CC5660
:10FD4000DF4F88839983AA83BB83C459D0408D89B0
:10FD50009E89AF89B88DC856DF4F88839983AA835F
:10FD6000BB83C859D0402D968CAD9DADAEADBFAD17
:10FD70002D97CA57DF4F88839983AA83BB83C658C0
:10FD8000D04089A19AA1ABA1BCA1C456DF4F888302
:10FD90009983AA83BB83CC59D0408DA19EA1AFA1EA
:10FDA000B8A5C056DF4F88839983AA83BB83C05A06
:10FDB000D0408DA59EA5AFA5B8A9CC55DF4F8883AF
:10FDC0009983AA83BB83C45AD04089A59AA5ABA5C1
:10FDD000BCA5CE54DF4F88839983AA83BB83C25BC3
:10FDE000D04061968CAD9DADAEADBFAD6197CA54AC
:10FDF000DF4F88839983AA83BB83C65BD04089A9E0
:10FE00009AA9ABA9BCA9C654DF4F88839983AA835A
:10FE1000BB83CA5BD0408DA99EA9AFA9B8ADC2541F
:10FE2000DF4F88839983AA83BB83CE5BD04089ADA3
:10FE30009AADABADBCADCE53DF4F88839983AA8317
:10FE4000BB83C25CD04021968CAD9DADAEADBFAD45
:10FE50002197CA53DF4F88839983AA83BB83C65CEB
:10FE6000D04014E6C12CD12C760146015701260161
:10FE70003701A3019201AE966CAD7DAD8EAD9FAD05
:10FE8000AE970F94A9AD9B01AC01AA966CAD7DAD68
:10FE90008EAD9FADAA970F94A2B92B013C01A5018D
:10FEA0009401A6966CAD7DAD8EAD9FADA6970F94D7
:10FEB000A9AD9B01AC01C301B2010F94A2B92B0102
:10FEC0003C01A7019601E6966CAD7DAD8EAD9FAD70
:10FED000E6970F94A9AD9B01AC01C301B2010F9449
:10FEE000A2B9EA962CAD3DAD4EAD5FADEA970F9449
:10FEF00091BA6E966CAF7DAF8EAF9FAF6E97C457C1
:10FF0000DF4F288139814A815B81CC58D0400F94E2
:10FF1000A9AD9B01AC01C258DF4F688179818A810C
:10FF20009B81CE57D0400F94A2B92B013C01A50173
:10FF30009401C057DF4F688179818A819B81C059C4
:10FF4000D0400F94A9AD9B01AC01C301B2010F9445
:10FF5000A2B94B015C01A7019601CC56DF4F688125
:10FF600079818A819B81C459D0400F94A9AD9B01AE
:10FF7000AC01C501B4010F94A2B9C856DF4F288166
:10FF800039814A815B81C859D0400F9491BA2B01C5
:10FF90003C01C456DF4F288139814A815B81CC59AD
:10FFA000D0406E966CAD7DAD8EAD9FAD6E970F94CB
:10FFB000A9AD9B01AC01CA57DF4F688179818A8165
:10FFC0009B81C658D0400F94A2B94B015C01C0562A
:10FFD000DF4F288139814A815B81C05AD040C301FB
:10FFE000B2010F94A9AD9B01AC01C501B4010F94FE
:10FFF000A2B94B015C01A7019601CC55DF4F688186
:020000021000EC
:1000000079818A819B81C45AD0400F94A9AD9B010C
:10001000AC01C501B4010F94A2B9CE54DF4F2881C1
:1000200039814A815B81C25BD0400F9491BA4B0108
:100030005C01C654DF4F288139814A815B81CA5BEC
:10004000D0406E966CAD7DAD8EAD9FAD6E970F942A
:10005000A9AD9B01AC01CA54DF4F688179818A81C7
:100060009B81C65BD0400F94A2B96B017C01C25446
:10007000DF4F288139814A815B81CE5BD040C3014B
:10008000B2010F94A9AD9B01AC01C701B6010F9459
:10009000A2B96B017C01CE53DF4F288139814A819F
:1000A0005B81C25CD040C501B4010F94A9AD9B0136
:1000B000AC01C701B6010F94A2B9CA53DF4F288122
:1000C00039814A815B81C65CD0400F9491BA6B0143
:1000D0007C01115009F0CDCE6E962CAD3DAD4EADEC
:1000E0005FAD6E97C655DF4F688179818A819B81AC
:1000F000CA5AD0400F94A3B96093B3157093B41546
:100100008093B5159093B615A3019201C255DF4FA8
:10011000688179818A819B81CE5AD0400F94A3B99E
:100120006093B7157093B8158093B9159093BA156D
:10013000A50194016A966CAD7DAD8EAD9FAD6A97B9
:100140000F94A3B96A966CAF7DAF8EAF9FAF6A97DD
:10015000A7019601A2966CAD7DAD8EAD9FADA29725
:100160000F94A3B9A2966CAF7DAF8EAF9FAFA2974D
:10017000EB969FADEB979150EB969FAFEB9791115C
:100180009ECA6A966CAD7DAD8EAD9FAD6A970F9499
:100190008EBA6093A3157093A4158093A5159093C0
:1001A000A6156A966CAD7DAD8EAD9FAD6A970F9426
:1001B0001CBD6093A7157093A8158093A915909303
:1001C000AA15A2966CAD7DAD8EAD9FADA2970F9492
:1001D0001CBDDC01CB01B0588093AB159093AC15DE
:1001E000A093AD15B093AE15A2966CAD7DAD8EAD5E
:1001F0009FADA2970F948EBA6093AF157093B01510
:100200008093B1159093B2156A962CAD3DAD4EAD6D
:100210005FAD6A97A2966CAD7DAD8EAD9FADA29796
:100220000F94A2B96B017C01E894F7F8B701A6011D
:1002300080E69FE00F943BB92FE132E449E05BE3B5
:10024000C701B6010F94EEBB18166CF425E33AEF24
:100250004EE85BE3C701B6010F94EEBB181634F00D
:1002600001E010E005C000E010E002C002E010E094
:1002700025E33AEF4EE85BE36A966CAD7DAD8EAD5B
:100280009FAD6A979F770F94EEBB18167CF025E31D
:100290003AEF4EE85BE3A2966CAD7DAD8EAD9FADBF
:1002A000A2979F770F94EEBB181614F402E010E0AB
:1002B0008091A3159091A415A091A515B091A615B4
:1002C000AE968CAF9DAFAEAFBFAFAE978091AB1582
:1002D0009091AC15A091AD15B091AE15A6968CAFCE
:1002E0009DAFAEAFBFAFA6978091B3159091B415F7
:1002F000A091B515B091B615EE968CAF9DAFAEAF8F
:10030000BFAFEE978091A7159091A815A091A91560
:10031000B091AA15E6968CAF9DAFAEAFBFAFE69792
:100320008091AF159091B015A091B115B091B21513
:10033000EA968CAF9DAFAEAFBFAFEA978091B7158D
:100340009091B815A091B915B091BA15C258DF4F68
:1003500088839983AA83BB83CE57D040A6E4BEE1AD
:100360006C96BFAFAEAF6C9782E8282E85E1382E31
:10037000F10181809280A380B48085819681A781DC
:10038000B085AA968CAF9DAFAEAFBFAFAA976C9663
:10039000EEADFFAD6C97C590D590E590F490A501BA
:1003A0009401AE966CAD7DAD8EAD9FADAE970F94C2
:1003B000A9AD2B013C01AA962CAD3DAD4EAD5FAD74
:1003C000AA97A6966CAD7DAD8EAD9FADA6970F9406
:1003D000A9AD9B01AC01C301B2010F94A3B9EE9684
:1003E0002CAD3DAD4EAD5FADEE970F94A3B99B0123
:1003F000AC01C701B6010F94A2B96B017C016C96E8
:10040000EEADFFAD6C973496459055906590749025
:10041000E6962CAD3DAD4EAD5FADE697C501B4019E
:100420000F94A9AD4B015C01EA962CAD3DAD4EADEC
:100430005FADEA97AA966CAD7DAD8EAD9FADAA97E4
:100440000F94A9AD9B01AC01C501B4010F94A3B9F0
:10045000C258DF4F288139814A815B81CE57D04015
:100460000F94A3B99B01AC01C301B2010F94A2B9CF
:100470004B015C01A7019601C701B6010F94A9AD1C
:100480006B017C01A5019401C501B4010F94A9ADD4
:100490009B01AC01C701B6010F94A3B90F9427BD0E
:1004A0002DEC3CEC4CE45FE30F94EEBB181614F417
:1004B0000EEF1FEFB8E02B0E311C6C96EEADFFADCA
:1004C0006C9738966C96FFAFEEAF6C9722EA35E1E9
:1004D0002215330509F04CCF0115110509F07AC139
:1004E000A2962CAD3DAD4EAD5FADA2976A966CADB8
:1004F0007DAD8EAD9FAD6A970F94A3B920E030E03B
:1005000040E05FE30F94A9AD6B017C010F948EBABC
:100510002B013C016093A3157093A4158093A5153E
:100520009093A615C701B6010F941CBDA2966CAF9F
:100530007DAF8EAF9FAFA2976093A7157093A8155C
:100540008093A9159093AA15DC01CB01B058AA9607
:100550008CAF9DAFAEAFBFAFAA978093AB15909312
:10056000AC15A093AD15B093AE154092AF15509257
:10057000B0156092B1157092B2151092B315109229
:10058000B4151092B5151092B6151092B7151092B9
:10059000B8151092B9151092BA156E961CAE1DAE14
:1005A0001EAE1FAE6E976A961CAE1DAE1EAE1FAE7F
:1005B0006A97CE57DF4FA881B981C258D0401196B3
:1005C0008D909D90AD90BC90149715968D919D91B6
:1005D0000D90BC91A02DAE968CAF9DAFAEAFBFAFCE
:1005E000AE97C657DF4FE881F981CA58D040C59011
:1005F000D590E590F490A5019401C301B2010F9448
:10060000A9ADA6966CAF7DAF8EAF9FAFA697AE9605
:100610002CAD3DAD4EAD5FADAE97AA966CAD7DAD48
:100620008EAD9FADAA970F94A9AD9B01AC01A69684
:100630006CAD7DAD8EAD9FADA6970F94A3B99B0118
:10064000AC01C701B6010F94A2B92091B315309146
:10065000B4154091B5155091B6150F94A3B96B011F
:100660007C016093B3157093B4158093B515909386
:10067000B61520E030E040E85FE36A966CAD7DADF2
:100680008EAD9FAD6A970F94A3B96A966CAF7DAF9C
:100690008EAF9FAF6A97C657DF4FE881F981CA587E
:1006A000D040349685919591A591B491A6968CAF42
:1006B0009DAFAEAFBFAFA697A5019401A2966CAD5A
:1006C0007DAD8EAD9FADA2970F94A9AD4B015C019E
:1006D000AE962CAD3DAD4EAD5FADAE97C301B20150
:1006E0000F94A9AD9B01AC01C501B4010F94A3B94E
:1006F0009B01AC01A6966CAD7DAD8EAD9FADA6976E
:100700000F94A2B92091B7153091B8154091B91541
:100710005091BA150F94A3B94B015C016093B715C2
:100720007093B8158093B9159093BA1520E030E016
:1007300040E85FE36E966CAD7DAD8EAD9FAD6E977C
:100740000F94A3B96E966CAF7DAF8EAF9FAF6E97CF
:10075000CE57DF4FA881B981C258D0401896CE57E6
:10076000DF4FB983A883C258D040C657DF4FE88116
:10077000F981CA58D0403896C657DF4FF983E883CD
:10078000CA58D0402A163B0609F013CF6A962CAD02
:100790003DAD4EAD5FAD6A97C701B6010F9491BAFA
:1007A0006093B3157093B4158093B5159093B615F7
:1007B0006E962CAD3DAD4EAD5FAD6E97C501B401EB
:1007C0000F9491BA6093B7157093B8158093B915CB
:1007D0009093BA154090A3155090A4156090A5155C
:1007E0007090A615C090AF15D090B015E090B115DF
:1007F000F090B2158091A7159091A815A091A91518
:10080000B091AA15A2968CAF9DAFAEAFBFAFA29725
:100810008091AB159091AC15A091AD15B091AE152E
:100820006A968CAF9DAFAEAFBFAF6A97A701960136
:10083000C301B2010F94A9AD4B015C016A962CADC6
:100840003DAD4EAD5FAD6A97A2966CAD7DAD8EAD00
:100850009FADA2970F94A9AD9B01AC01C501B40156
:100860000F94A2B94B015C019B01AC01C701B60119
:100870000F9491BA6B017C016A966CAD7DAD8EAD23
:100880009FAD6A979058A50194010F9491BA6A960A
:100890006CAF7DAF8EAF9FAF6A97A2966CAD7DAD0A
:1008A0008EAD9FADA2979058A50194010F9491BA77
:1008B000CE57DF4F688379838A839B83C258D040A9
:1008C000A5019401C301B2010F9491BA4B015C01DF
:1008D0004090B3155090B4156090B5157090B61552
:1008E0008091B7159091B815A091B915B091BA152E
:1008F000A2968CAF9DAFAEAFBFAFA297C092A3152B
:10090000D092A415E092A515F092A615CE57DF4F10
:1009100088819981AA81BB81C258D0408093A71554
:100920009093A815A093A915B093AA156A968CADBB
:100930009DADAEADBFAD6A978093AB159093AC15EE
:10094000A093AD15B093AE158092AF159092B015EF
:10095000A092B115B092B215C701B6019058A3018B
:1009600092010F94A9AD6B017C01A2962CAD3DAD17
:100970004EAD5FADA2976A966CAD7DAD8EAD9FAD6D
:100980006A970F94A9AD9B01AC01C701B6010F9402
:10099000A2B96093B3157093B4158093B515909375
:1009A000B615CE57DF4F688179818A819B81C25805
:1009B000D0409058A30192010F94A9AD6B017C0126
:1009C000A2962CAD3DAD4EAD5FADA297C501B40171
:1009D0000F94A9AD9B01AC01C701B6010F94A2B958
:1009E0006093B7157093B8158093B9159093BA15A5
:1009F00080E090E00F94C14417FD53C043EB55E1F4
:100A00006BEA75E183EA95E10F94A30A4091B3156F
:100A10005091B4156091B5157091B61585EE9FE0B3
:100A20000F943BB94091B7155091B8156091B91525
:100A30007091BA1589EE9FE00F943BB94091A315D0
:100A40005091A4156091A5157091A6158DED9FE0AC
:100A50000F943BB94091A7155091A8156091A91525
:100A60007091AA1581EE9FE00F943BB94091AB15B0
:100A70005091AC156091AD157091AE1585ED9FE06C
:100A80000F943BB94091AF155091B0156091B115DD
:100A90007091B21589ED9FE00F943BB90F94280A2D
:100AA00009C00E3F9FEF190729F4AF96AFADAF977E
:100AB000A23049F038010BC0AF961FAEAF97662445
:100AC0006A94762C04C0BEEF6B2E77247A94C855B6
:100AD000DF4F88819981C85AD0400F94325E80E000
:100AE00090E0A0EAB0E48093541090935510A09346
:100AF0005610B093571020915010309151104091E2
:100B000052105091531060914C1070914D10809183
:100B10004E1090914F10E7E0FDE0FF93EF93812C92
:100B2000912CE0EAAE2EE1E4BE2EF8E5CF2EF0E106
:100B3000DF2EE12CF12C00EA10E40F94EF2C0F943F
:100B400003890F900F9077FC22C020E030E046E14F
:100B500053E460915410709155108091561090910B
:100B600057100F94A3B9609354107093551080934D
:100B700056109093571065E575E585E591E40F945F
:100B8000BA098EE899E10E94ACFC0F94C51181E08E
:100B90000F944E1682E00F94BE0EBFEF6B167B06CD
:100BA00031F481E599E10E94ACFC10E04BC0EEEF1E
:100BB0006E16EFEF7E0681F4AF96FFADAF97FF2381
:100BC00029F0F23031F08AE098E1EDCF8FE898E13A
:100BD000EACF8FE498E1E7CFAF962FADAF97211121
:100BE00007C033E06316710498F08FE898E117C0EE
:100BF000AF966FADAF97623019F48CE099E102C007
:100C000082EC98E10E94ACFC1614170454F309C05E
:100C1000F301EE0FFF1FE353FD4F808191810E948E
:100C2000ACFC6720609409F286EE0F942E628FE58B
:100C30009FE00F9417B9813021F083EB99E10E9476
:100C4000ACFC11E00E94F8AE2BC182E79EE10E944D
:100C5000ACFC10E025C183E0821B282F0C94F374B8
:100C600081E00C945276F0E9CF1AF1E0DF0A0C949F
:100C70009475E7968FADE797E8969FADE8970C944B
:100C800033778E7F0C947F7780E4482E512C612C33
:100C9000712C0C94957787E190E00C94A9778F3FA5
:100CA000910509F014F40C94B1778FEF90E00C9457
:100CB000B1778B7F0C94B977B0E6EB16B9E0FB0601
:100CC00014F00C94C87784E00F94DA54EFEFEE1A26
:100CD000FE0A0C94C877C6010C94E87781508830DE
:100CE00011F00C94C1780C94C87800E00C94D6787C
:100CF00080E090E00C94FB78EBE0BE1611F40C94CD
:100D00007179222311F02B3039F4E396FFADE3978C
:100D1000F83010F00C947779B101620F731F6157AE
:100D2000784FFB01F081A396FFAFA397E896EEAD55
:100D3000FFADE897C080D18061E070E0022E02C074
:100D4000660F771F0A94E2F76C217D21672B31F043
:100D5000A396FFADA397F13148F005C0A3966FAD00
:100D6000A397613118F401960C94777901970C944C
:100D7000777980E00C94057A84EF91E00F94A223B8
:100D8000882311F40C94107A14E0812C912C5401D6
:100D9000C12CD12C760188EE93E00F94A2238823F6
:100DA00011F40C94107A80913C1090913D10A09118
:100DB0003E10B0913F10092E000CAA0BBB0BC80EC1
:100DC000D91EEA1EFB1E8091401090914110A09107
:100DD0004210B0914310092E000CAA0BBB0B880ED9
:100DE000991EAA1EBB1E1150B1F64090441050909F
:100DF00045106090461070904710C501B40122E084
:100E000096958795779567952A95D1F732E0F69470
:100E1000E794D794C7943A95D1F700E028EC30E0F6
:100E2000A201C6010F945C2211E00C94117A298171
:100E30003A812059374F3A8329830C945276F20134
:100E40002581368147815085E6966CAD7DAD8EADAE
:100E50009FADE6970C94997CF201258136814781FC
:100E60005085E6966CAD7DAD8EAD9FADE6970C944A
:100E7000B27C60E070E080E89FE30C94B47C1123C6
:100E800011F40C94C27C812C912C40E8A42E4FE3E9
:100E9000B42E0C949D7C01110C94887C0C94C27C23
:100EA00081E00F944E1680E00F94ED66812FC753BA
:100EB000DF4F0FB6F894DEBF0FBECDBFDF91CF91ED
:100EC0001F910F91FF90EF90DF90CF90BF90AF9068
:100ED0009F908F907F906F905F904F903F902F905A
:100EE000089561E0FC0180810D94A8218EBD0DB4B0
:100EF00007FEFDCF08958FEF8EBD0DB407FEFDCF29
:100F00008EB508958F929F92AF92BF92EF92FF920B
:100F10001F93CF93DF93EC01162F49015A019A8159
:100F2000892F806A86958CBD90FD03C081E0963044
:100F300009F480E08DBD60E088810F94A8216CE207
:100F400071E0CE010E94DBEB812F8064CFDF88E16E
:100F5000E82EF12CD501C4010E2C04C0B695A7953E
:100F6000979587950A94D2F7C1DF88E0E81AF108CF
:100F700088EFE8168FEFF80669F7112391F0183023
:100F800011F487E801C08FEFB1DF1C3009F4B3DF43
:100F900010E0B1DF8B8387FF07C01F3F29F01F5F81
:100FA000F8CF85E9A3DFF4CFDF91CF911F91FF90B8
:100FB000EF90BF90AF909F908F9008952F923F92A7
:100FC0004F925F926F927F928F929F92AF92BF9259
:100FD000CF92DF92EF92FF920F931F93CF93DF9305
:100FE000CDB7DEB728970FB6F894DEBF0FBECDBFE2
:100FF0001B012C017090310D7092070DC0902D0DCA
:10100000D0902E0DE0902F0DF090300D20E030E0CC
:10101000A901C701B6010F943CB48823D9F071101F
:1010200008C0C701B6010F9402BB70937615609398
:10103000751581E090E09093510D8093500D0F94C1
:10104000D653472D0F946F4382E090E09093510D5B
:101050008093500D8091290D90912A0DA0912B0D18
:10106000B0912C0D80935B0290935C02A0935D0283
:10107000B0935E028091280D8093380D8091260DEB
:101080009091270D9093C1198093C019A2019101ED
:101090006091220D7091230D8091240D9091250D6A
:1010A0000F94A2B96D837E838F839887CE010596B6
:1010B0000E9440D6A20191016091220D7091230DF2
:1010C0008091240D9091250D0F94A2B969837A83A4
:1010D0008B839C83E0905410F09055100091561033
:1010E0001091571020911A0D30911B0D40911C0D3D
:1010F00050911D0D6091160D7091170D8091180D76
:101100009091190DE7E06E2EEDE07E2E7F926F92AA
:10111000F2E68F2EF7E29F2EF6E7AF2EF2E4BF2E17
:10112000FE0131966F010F94EF2C0F940389A201F9
:1011300091016091220D7091230D8091240D909169
:10114000250D0F94A2B969837A838B839C83E090E9
:101150001E0DF0901F0D0091200D1091210D20917A
:101160001A0D30911B0D40911C0D50911D0D609179
:10117000160D7091170D8091180D9091190D7F9299
:101180006F920F94EF2C0F940389E0901E0DF09056
:101190001F0D0091200D1091210D20911A0D3091FD
:1011A0001B0D40911C0D50911D0D6091160D7091FD
:1011B000170D8091180D9091190D7F926F92812CCF
:1011C000912CACE0AA2EA2E4BA2EB2E2CB2EBDE066
:1011D000DB2E0F94EF2C0F94038980E1E6E1FDE014
:1011E000ACE4B0E101900D928A95E1F780E1ECE486
:1011F000F0E1A8E0BFE001900D928A95E1F78091BF
:10120000110D0F900F900F900F900F900F90811174
:101210002AC04090120D5090130D6090140D7090E4
:10122000150D4092511950925219609253197092B3
:101230005419B301A2018CE998E10E949DEE4092FD
:101240005C0D50925D0D60925E0D70925F0D81E0BD
:101250008093761685E590E29F938F930F9447B322
:101260000F900F9018C08130B1F48091120D9091C1
:10127000130DA091140DB091150D8093620D9093F4
:10128000630DA093640DB093650D109280131092BE
:101290007F130F94E3448EE194E10F942326109280
:1012A0007F0E28960FB6F894DEBF0FBECDBFDF913C
:1012B000CF911F910F91FF90EF90DF90CF90BF9053
:1012C000AF909F908F907F906F905F904F903F90E6
:1012D0002F9008958F929F92AF92BF92CF92DF92FC
:1012E000EF92FF92CF93DF930F94D6536B017C0163
:1012F00020912F02222309F47BC0409125025091B6
:1013000026024130510509F473C080912B0290915F
:101310002C02A0912D02B0912E0246015701881A8D
:10132000990AAA0ABB0A30E0A8EEB3E00F9493B979
:1013300086169706A806B9060CF462C0443051051B
:1013400059F14CF4423051050CF452C0E9EBFDE583
:101350008491EF0109C04530510509F049C0E9EB1E
:10136000FDE58491EF0130C0882331F00F94A14F47
:101370002196FE018491F8CFE4E4F0E28491EF013C
:10138000882331F00F94A14F2196FE018491F8CF6C
:101390008AE00F94A14F2CC0E9EBFDE58491EF01A9
:1013A000882331F00F94A14F2196FE018491F8CF4C
:1013B000EEE2F0E28491EF01882351F30F94A14F04
:1013C0002196FE018491F8CF882331F00F94A14F2C
:1013D0002196FE018491F8CFE7E1F0E28491EF01DC
:1013E0008823B1F20F94A14F2196FE018491F8CF8A
:1013F000C0922B02D0922C02E0922D02F0922E028B
:10140000DF91CF91FF90EF90DF90CF90BF90AF90A2
:101410009F908F9008958F929F92AF92BF92CF929C
:10142000DF92EF92FF920F931F93CF93DF93CCE461
:10143000D0E120E030E048EC51E46C857D858E857C
:101440009F850F94A3B96C877D878E879F87E884DB
:10145000F9840A851B852C813D814E815F816881DD
:1014600079818A819B81E7E0FDE0FF93EF93E3E3DD
:101470008E2E982CE3E5AE2EE0E4BE2EF8E5CF2EBE
:10148000F0E1DF2E0F94EF2C0F900F90DF91CF91B2
:101490001F910F91FF90EF90DF90CF90BF90AF9092
:1014A0009F908F9008954F925F926F927F928F924C
:1014B0009F92AF92BF92CF92DF92EF92FF920F93E3
:1014C0001F93CF93DF93CDB7DEB7E0970FB6F894B5
:1014D000DEBF0FBECDBFE0917F0EE11144C12901F7
:1014E0003A014B015C01F894809176168823F9F05B
:1014F000C0905C0DD0905D0DE0905E0DF0905F0DA2
:101500000E94B2D5C81AD90AE108F1080E94F7B6BC
:10151000C81AD90AE108F108C092120DD092130D31
:10152000E092140DF092150D1092110D2BC08091C8
:101530004507882321F1C090620DD090630DE090A3
:10154000640DF090650D0E94B2D5C81AD108E1086B
:10155000F1088091841390918513092E000CAA0B39
:10156000BB0BC81AD90AEA0AFB0AC092120DD09224
:10157000130DE092140DF092150D81E001C082E090
:101580008093110D9091090780910807981799F0A1
:10159000E091080727E5E29FF0011124E157F84F99
:1015A00020E030E040E752E462A173A184A195A15C
:1015B0000F94A9AD08C060915B0270915C028091AC
:1015C0005D0290915E026093290D70932A0D8093C5
:1015D0002B0D90932C0D0F942D3B80E1ECE4F0E16A
:1015E000A6E1BDE001900D928A95E1F7E091070D2B
:1015F000E093310DF0E0EE0FFF1FEB58FA4E6081E3
:101600007181072E000C880B990B0F9442B46093E4
:101610002D0D70932E0D80932F0D9093300D809192
:10162000380D8093280D8091C0199091C119909325
:10163000270D8093260D0E94DDEA1092761681E038
:1016400080937F0EB19A109285001092840080EDF5
:1016500097E09093890080938800789420E030E0B0
:10166000A901C501B4010F943CB481110AC020E066
:1016700030E0A901C301B2010F943CB4882309F4FE
:1016800072C08091280D9E012F5F3F4F790181111B
:1016900009C063E170E2C9010F94F2B160E0C701D3
:1016A0000E9415EA6EE070E2C7010F94F2B1F701F3
:1016B00001900020E9F78F010150110923E046E075
:1016C000C301B2010F945DAE6BE070E2C7010F94ED
:1016D000E7B1F70101900020E9F78F0101501109EE
:1016E00023E048E060E070EC88E295E40F945DAEA2
:1016F00060E0C7010E9415EA66E070E2C7010F943E
:10170000F2B1F70101900020E9F78F0101501109B2
:1017100020911E0D30911F0D4091200D5091210DF3
:10172000C501B4010F94A3B923E048E00F945DAE66
:1017300063E070E2C7010F94E7B1F7010190002068
:10174000E9F78F010150110923E048E060E070E003
:1017500088E494E40F945DAE60E0C7010E9415EA4E
:1017600081E080938313E0960FB6F894DEBF0FBE3E
:10177000CDBFDF91CF911F910F91FF90EF90DF9040
:10178000CF90BF90AF909F908F907F906F905F9021
:101790004F9008953F924F925F926F927F928F92F7
:1017A0009F92AF92BF92CF92DF92EF92FF920F93F0
:1017B0001F93CF93DF93CDB7DEB7C855D1090FB6CE
:1017C000F894DEBF0FBECDBFB82E81E00F944E1649
:1017D00082E00F94BE0E8BE391E20F94232685EAFC
:1017E0009FE00F9417B9A82E8DE99FE00F941FB9C1
:1017F00060934C1070934D1080934E1090934F1047
:1018000081EA9FE00F941FB96093501070935110BC
:10181000809352109093531022E0A21209C08AEDD7
:101820009EE00F941FB96B017C0188ED9EE008C01B
:101830008DE89FE00F941FB96B017C0183E79FE067
:101840000F9424B967E074E0681B790BE4E07695A7
:101850006795EA95E1F780E090E00F9440B420911D
:101860009C1030919D1040919E1050919F100F94AC
:1018700091BA2B013C012AE037ED43E25FE3C70157
:10188000B6010F94A3B99B01AC01C301B2010F943F
:10189000A3B9609354107093551080935610909391
:1018A000571082E79FE00F9417B9882391F18EE6D5
:1018B0009FE00F941FB96093581070935910809354
:1018C0005A1090935B1088E19FE19F938F93CE0114
:1018D00001967C019F938F930F94A0B3F701019021
:1018E0000020E9F78F0101501109609158107091A3
:1018F000591080915A1090915B1023E046E00F94AC
:101900005DAE60E0C7010E9415EA0F900F900F9046
:101910000F9080E1ECE4F0E1A8E0BFE001900D92CF
:101920008A95E1F7E6EEFEE184918F01882339F094
:101930000F94A14F0F5F1F4FF8018491F7CF809153
:1019400057108F93809156108F93809155108F93DD
:10195000809154108F93809153108F9380915210E7
:101960008F93809151108F93809150108F9380911D
:101970004F108F9380914E108F9380914D108F93C5
:1019800080914C108F9380E790E29F938F930F94F8
:1019900047B30F94150E109282150FB6F894DEBF60
:1019A0000FBECDBF55E7E52E5FE0F52E912C63E02D
:1019B000762E6E013FE1C30ED11C6624639477E05E
:1019C000872E892D672D0F9434BE082F592E42E0A3
:1019D00050E0B701C6010F9407B96F8D78A161156A
:1019E000710511F060928215282D020380011124E7
:1019F000050D111D57FC1A95000F111F000F111F27
:101A00000E571A4E072E000C880B990B0F9442B4F8
:101A10002FE632E143E85AE30F94A9ADF801618360
:101A20007283838394839394F2E0EF0EF11C29E098
:101A30009212C7CF8091821581110F9471760E9406
:101A4000C1A4E0905410F0905510009156101091E0
:101A500057102091501030915110409152105091D8
:101A6000531060914C1070914D1080914E109091D8
:101A70004F100F94FB7181E08093080D17988093AD
:101A8000090D169880930A0D1598E4EBFEE18491F8
:101A90008F01882339F00F94A14F0F5F1F4FF8017A
:101AA0008491F7CF82E00F94F088962E872E782EBF
:101AB000692E81E00F94F088162F072FF82EE92E5B
:101AC00080E00F94F0886F927F928F929F92EF92B6
:101AD000FF920F931F939F938F937F936F9387E949
:101AE00090E29F938F930F9447B38CE89FE00F94FD
:101AF00017B9E091070DF0E0EE0FFF1FEB58FA4E1B
:101B000090E0918380838BE89FE00F9417B990E079
:101B100090930C0D80930B0D88EE9EE00F941FB9EF
:101B200060932702709328028093290290932A02DF
:101B30008EED9EE00F9424B99093600280935F0233
:101B40000FB6F894DEBF0FBECDBF32E0A316A9F0EA
:101B500020E030E048EC51E4609154107091551051
:101B600080915610909157100F943CB487FF05C098
:101B700061E087EF9FE10E9415EA61E08FEE9FE14F
:101B80000E9415EAE091070DF0E0EE0FFF1FEB5801
:101B9000FA4E81818F9380818F9386EE9FE19F9390
:101BA0008F93DF92CF920F94A0B360E0C6010E94A2
:101BB00015EA80910C0D8F9380910B0D8F938DED15
:101BC0009FE19F938F93DF92CF920F94A0B360E039
:101BD000C6010E9415EA61E089ED9FE10E9415EAC5
:101BE0000FB6F894DEBF0FBECDBFB11005C061E0E7
:101BF0008EEC9FE10E9415EA61E081EB9FE10E947B
:101C000015EA809153108F93809152108F93809199
